:1000000000800020BD01000089D9000041D9000016
:1000100041D9000041D9000041D9000041D9000078
:1000200041D9000041D9000041D9000089D9000020
:1000300089D9000041D9000009D000000DD100008D
:1000400089D9000089D9000089D9000089D9000028
:1000500089D9000089D9000089D9000089D9000018
:1000600089D9000089D9000089D9000089D9000008
:1000700089D9000089D9000089D9000089D90000F8
:1000800089D9000089D9000089D9000089D90000E8
:1000900089D9000089D9000089D9000089D90000D8
:1000A00045B5000051B5000089D9000089D900008C
:1000B00089D9000089D9000089D9000089D90000B8
:1000C00089D9000089D9000089D9000089D90000A8
:1000D00089D9000089D9000089D9000089D9000098
:1000E00089D9000089D9000089D9000089D9000088
:1000F00089D90000F5F9000089D9000021FB000032
:1001000089D9000061E3000089D9000089D9000085
:1001100089D9000089D9000089D9000089D9000057
:1001200089D9000089D9000089D9000089D9000047
:1001300089D9000089D9000089D9000089D9000037
:1001400089D9000089D9000089D9000089D9000027
:10015000F9D100000DD2000021D2000035D20000FC
:1001600089D900007DE6000089D9000089D9000006
:1001700089D9000089D9000089D9000089D90000F7
:1001800089D9000089D9000089D9000089D90000E7
:1001900089D9000089D9000089D9000089D90000D7
:1001A00089D9000089D9000089D9000089D90000C7
:1001B00089D9000089D9000089D90000564B4CF23A
:1001C000205210B51A804DF628121A8000BF00BFC9
:1001D0000DF0DEFB514B4FF010621A60504A9A60EE
:1001E000504ADA60504A136813F4807304D14F49BF
:1001F0000B604FF4A85313604D4B1A78110703D5C9
:100200001A7842F008021A704A4B4B492A221A7097
:100210004A4A4B4B8B4204D252F8040F43F8040B6A
:10022000F8E7484B484900228B4202D243F8042B9E
:10023000FAE74649464A002352F8230041F82300D2
:1002400001336F2BF8D1434B434A802103F8011B44
:100250009342FBD1414B3D4A1A60414B8A221A70AE
:10026000A3F5805324225A70A0221A709A7992071B
:10027000FCD59A79D406FCD43A4A937903F00C035E
:10028000082B384BF9D103221A7140225A719A79FE
:100290009006FCD5334A9179324B4906FBD5324A58
:1002A000324911600221516020221A709A7902F0BD
:1002B0000C020C2AFAD12E4B2E4A1A602E4B2F4AD2
:1002C0001A6000225A60072243F8042C2C4AC3F813
:1002D0000C2D62B60DF00CFF144B1B68DA0705D528
:1002E00028480DF0D9FC284B284A1A60284B1B7867
:1002F0005B0609D5244C254B22689A4204D121483B
:100300000DF0CAFC0023236010F0C2FE0DF046FB86
:100310000DF074FAFEE700BF0E2005403080044067
:10032000823F04000100002B10D0034014D0034092
:1003300002D0074000E00740649CFF1F744A0100A0
:100340004088FF1F649CFF1FA0A4FF1F0082FF1FA7
:100350000000000000E400E05FE400E008ED00E0E1
:100360000050064000400640448004400000030165
:1003700004800440C010050014E000E0FF76010096
:10038000000020207D6E4F5F1CE00340A5C3945AFF
:1003900000F00740FFFFFFFFFFFFFFFFFFFFFFFF32
:1003A000FFFFFFFFFFFFFFFFFFFFFFFFFFFFFFFF5D
:1003B000FFFFFFFFFFFFFFFFFFFFFFFFFFFFFFFF4D
:1003C000FFFFFFFFFFFFFFFFFFFFFFFFFFFFFFFF3D
:1003D000FFFFFFFFFFFFFFFFFFFFFFFFFFFFFFFF2D
:1003E000FFFFFFFFFFFFFFFFFFFFFFFFFFFFFFFF1D
:1003F000FFFFFFFFFFFFFFFFFFFFFFFFFFFFFFFF0D
:10040000FFFFFFFFFFFFFFFFFFFFFFFFDEF9FFFF23
:1004100010B5054C237833B9044B13B10448AFF33E
:1004200000800123237010BD649CFF1F00000000AA
:10043000784A0100084B10B51BB108490848AFF3D2
:1004400000800848036803B910BD074B002BFBD0A0
:10045000BDE81040184700BF00000000689CFF1F67
:10046000784A0100649CFF1F0000000038B5044674
:10047000104621700A491D4610F0ECFB01464FF072
:100480007E5010F09BFC074910F0E4FBE5606060D3
:10049000256165610DF0BCFDE061204638BD00BFFF
:1004A000DB0FC9400024744938B50446104621705A
:1004B00009491D4610F0CEFB01464FF07E5010F06A
:1004C0007DFC064910F0C6FBE56060602561656152
:1004D0000DF09EFDE06138BDDB0FC940002474497A
:1004E00038B503780446032B20D8DFE803F01A1848
:1004F0001002C168406910F0A3FA0D490546606812
:1005000010F05CFC0146284610F058FC38BD084944
:10051000406810F053FCE16810F09CFB38BDC068E7
:1005200038BDC168406910F08BFA38BD002038BD75
:100530000024744970B504460E460DF069FD054669
:10054000E069281A10F032FBE3682361E561666117
:10055000A0610146606810F031FC0146A0601048BF
:1005600010F02CFC0FF002FF0FF0A2FB10F014FAB9
:10057000054601464FF07E5010F062FA616910F0B6
:1005800069FB21690646284610F064FB01463046A7
:1005900010F058FAE0602046BDE87040FFF7A0BFB9
:1005A000000080BF38B50E201C4C0DF001F82188EA
:1005B0001B4B884205461A881DDA0023511AB1F5F3
:1005C000805FAABF1B03C3EB03330131142093FBED
:1005D000F1F10DF073FB134B1988F1B923889D429B
:1005E00010DAC3F57F630F33282091FBF3F1BDE8E8
:1005F00038400DF063BB9042D4BFC1EB0003C1EBA8
:100600000203DBE740F6FF718D42D4BFC3EB050167
:10061000C3EB0101C1EB0131E3E738BD609DFF1F72
:100620002C9FFF1FCC9EFF1F10B504460CF0C2FD8F
:10063000204610BD70B44C88A04220D9012301335C
:10064000DBB21CB2660031F8144084421D46F6D37A
:10065000A04211D005F10045013D965B31F815101F
:1006600032F81530401AF21A00FB02F0641A90FBBF
:10067000F4F4E01870BC7047905B70BC70470226C1
:100680000125E5E700280CDA064A434282FB0320F5
:10069000DA17C2EB600000EB4000A3EB8000C0F172
:1006A0000C007047ABAAAA2A38B5234B1B78002B45
:1006B0002CD015200CF07CFF204B1860204B1B88A1
:1006C000984203DA1F4C237863BB38BD1E4A148856
:1006D000A042A4EB0302A8BF20467F2A1CDDC01A5B
:1006E000C001541C90FBF4F4002CEBD0154B1A788D
:1006F0000AB901221A70154D2B689C4204D0144B84
:10070000E1B2187809F004F82C6038BD11200DF022
:1007100093FE0A4B1860D1E7C01AC0EBC01090FBE3
:10072000F2F4E1E70A4B0021187808F0F1FF00230A
:10073000064A2370136038BD809EFF1F909CFF1FE8
:100740000A9DFF1F5C9FFF1FF89EFF1F549FFF1F06
:10075000E09CFF1F38B50F200DF06EFE1B4A1C4BAE
:1007600012881860C0F53B600830904220DB194BBE
:100770001B889842A3EB0204A8BF1846801A7F2C5E
:10078000C6BFC0010134C0EBC01090FBF4F47CB1D3
:10079000114B1A780AB901221A70104D2B689C422D
:1007A00004D00F4BE1B2187808F0B2FF2C6038BDCE
:1007B000094C237803B938BD094B0021187808F09B
:1007C000A7FF0023054A2370136038BD649DFF1FF7
:1007D000789EFF1FE49EFF1F089FFF1F189DFF1FAD
:1007E000FE9CFF1FF0B40E8886420DD203F1004339
:1007F000013B31F81350854202D9F0BCFFF71ABF14
:1008000032F81300F0BC70471088F0BC704700BF8E
:10081000094B1B880C2B09D8084A80B252F82320B8
:1008200028B143F6FE73984203D9108C70471088A4
:1008300070470349FFF7FEBEB69CFF1F5425010019
:10084000F02601004B4B4C4A2DE9F0471E881468F6
:100850004A4BB442B3F80080494B33DB4445A8BF50
:100860004446A6421C60C8BF00202DDDC6EB080729
:10087000B7F5804F33DB80037B1C90FBF3F0FFF771
:10088000C7FF404A404B15881B88C0F3C61909FBB7
:1008900005F57F2D8246A8BF7F252BB3A64253DCEA
:1008A0004445D4BFC6EB0404C6EB08049F42CCBF4A
:1008B00003FB04445C43354BC8BF013794FBF7F797
:1008C0001F6013E034461E60C6EB0807A045D4BF86
:1008D000C6EB0800C6EB0400B7F5804FCBDAC0EBDF
:1008E000803090FBF7F0CAE7284A1360284C236851
:1008F000994508D0274B1B88002B34D1264B1B88E9
:100900006BBBC4F80090254C23689A4506D0214B58
:100910001B885A1F032A19D9C4F800A0204C236849
:100920009D420FD01F4B188848B11A4B1E4A1B8896
:10093000D35C834203D0C0B2E9B208F0E9FE25607F
:10094000BDE8F087BDE8F0870024AFE7164AD05C29
:100950002030C0B20AF07F0108F0DAFEDCE748463A
:1009600008F04AFFCDE7104A4946D05C08F0D0FEB7
:10097000C4E700BF609DFF1FC89EFF1F2C9FFF1F85
:10098000889CFF1F989CFF1F9A9CFF1F349FFF1F8E
:10099000F89CFF1FB09EFF1F529DFF1FB09CFF1FC2
:1009A000549DFF1FBE9EFF1F088AFF1F2DE9F04FB9
:1009B00001208BB00DF040FDDFF870B3DFF870A3BD
:1009C000CBF8000000200DF037FDBA4BCAF800004C
:1009D0001B880C2B00F05E82B74EB84A3188B84BAA
:1009E00052F8214000221A70B64BB74A1B88B7490B
:1009F0001288013B012A31F91330059300F0AE81D2
:100A0000B34B0193B34B0293B34FDFF8288300231A
:100A10000093B24B1B88012B00F0F481DFF8189390
:100A2000AF4B0393D9F80050AE4B04930023AE4A6A
:100A30001288013A032A00F24982DFE812F0A50089
:100A4000ED000400C9002846059310F0AFF8A7494F
:100A500010F000F9059B0546184610F0A7F8A449C8
:100A600010F0F8F8014628460FF0ECFF10F0B8FA45
:100A70000546C9F80050386810F098F89B4910F006
:100A8000E9F88146009810F091F8994910F0E2F8E1
:100A9000014648460FF0D6FF10F0A2FA3860954A9A
:100AA000954B17881988954BDBF800201B88DFF8D9
:100AB0008CE2C7EB050C3D44039FC7F800C0471A02
:100AC000084404990D6001990F600299BEF8007006
:100AD00008609A4280F2E7800025C3EB070E744558
:100AE000DAF8000080F2D380611C984205FB01F522
:100AF0000EF1010E95FBFEF5C0F25F838742A8BFA1
:100B00000746FF1A01FB07F494FBFEF49A4200F338
:100B1000A780984200F3A480794C206810F046F832
:100B2000784910F097F878490FF08CFF10F058FAD8
:100B3000A0F5FF531C3B082B98BF4FF40050D8F88A
:100B40000030184400282060C0F29F80B0F5804F2C
:100B500080F2F6806D4B1B781BB1B0F5005F40F062
:100B6000F7806B4D2B78002B40F0AB81694D2068EE
:100B70002B68634C984204D080B208F0A7FE23682B
:100B80002B600BB0BDE8F08F2846059310F00EF8EF
:100B9000614910F05FF8059B0546184610F006F80D
:100BA0005E4910F057F8014628460FF04BFF10F051
:100BB00017FA0546C9F8005038680FF0F7FF564994
:100BC00010F048F8814600980FF0F0FF53495DE7B8
:100BD000284605930FF0EAFF4A4910F03BF8059BC1
:100BE000054618460FF0E2FF4D4910F033F8014674
:100BF00028460FF027FF10F0F3F90546C9F800501A
:100C000038680FF0D3FF3F4910F024F88146009870
:100C10000FF0CCFF424939E7284605930FF0C6FF95
:100C2000404910F017F8059B054618460FF0BEFF27
:100C30003D4910F00FF8014628460FF003FF10F071
:100C4000CFF90546C9F8005038680FF0AFFF3549B5
:100C500010F000F8814600980FF0A8FF324915E720
:100C60003388002B3FF458AF2B1B002BB8BF5B42DF
:100C7000092B00F32D81D8F80030214C4FF400509F
:100C8000184400282060BFF661AF00225AE0984265
:100C900005FB04F5B8BF002195FBFEF580F28482C8
:100CA00091FBFEF432E7BA42D4BFC3EB0205C3EBBB
:100CB000070512E7FA9EFF1FEE9CFF1F8889FF1FA2
:100CC0008E9CFF1F2089FF1FCE9EFF1FA0290100C1
:100CD000589FFF1F289DFF1F809CFF1F5C9EFF1FCA
:100CE000EC9EFF1F609EFF1F5E89FF1FCDCC4C3F17
:100CF000CDCC4C3E148AFF1F5C89FF1FC49EFF1F92
:100D0000BC89FF1F9A99193FCDCC4C450EA0FF1FFF
:100D1000509DFF1F2489FF1F3333733FCDCC4C3DC3
:100D2000CDCCCC3E6666663FCDCCCC3DE89CFF1F6B
:100D3000AC9CFF1F049FFF1FE89EFF1FCC9CFF1F62
:100D400043F6FF72C04B22601B78002B3FF409AFC3
:100D500005F0B2FEBD4B01221A7007E7BC4BBD4A3D
:100D60001B88BD491278013B31F91350002A40F02D
:100D7000C78011200DF060FB0090B84B0193D3F8B1
:100D80000080009B984540F3C080B54BB54F1B8851
:100D9000B54A012B3B68B2F80090B44A0292204653
:100DA000A3EB050500F0E2800FF000FF029A52F875
:100DB00029100FF04FFF014600200FF041FE10F008
:100DC0000FF9009BC8EB05029D42B8BF1D4690423B
:100DD000C8EB050580F2DE8000FB0555013295FB6E
:100DE000F2F5A34BDFF8B4820293D8F800302B441D
:100DF00003EBD3735B10C8F800309E4B1B88012BAC
:100E00007FF40CAE9C4B03931D460F200DF014FB9A
:100E10002A6804929042034680F2CC80904A12885D
:100E2000012A00F03F81904A079012888F4D069268
:100E300020460FF0BBFE069ADFF8649255F82210A8
:100E4000D9F800500FF006FF014600200FF0F8FD22
:100E5000059BEA1A059210F0C3F8059A079B0499BE
:100E60009A42C1EB020EB8BF1A46704580F2448127
:100E7000521A00FB02220EF1010192FBF1F2D8F8A6
:100E800000107E4804900A4402EBD2725210C8F857
:100E90000020CCE57A4B1B78002B3FF49DAD794EBA
:100EA000794A3188794B52F8210001221A700FF0EB
:100EB0007DFE4FF07C510FF0CDFE10F091F804460E
:100EC00092E505F0F5FD00232B704FE63868E6E566
:100ED00005F500500130001B0FF068FE6C496D4CA9
:100EE0000FF0B8FE054620680FF060FE6A490FF06B
:100EF000B1FE014628460FF0A5FD10F071F81EE680
:100F000015200CF055FB009037E7594B0293D3F8AE
:100F10000080009B984542DA514B524F1B88524A41
:100F2000012B3B68B2F80090504A039220461D44C2
:100F300000F0E9800FF03AFE039A52F829100FF002
:100F400089FE10F04DF8009B9D42C8EB0502A8BF3A
:100F50001D46C8EB05059042BABF00FB055501329E
:100F6000454395FBF2F5DFF834813EE70FF01EFEB6
:100F7000029A52F829100FF06DFE10F031F8009B24
:100F8000C8EB05029D42B8BF1D468242C8EB05056D
:100F90003FF722AF00FB05F595FBF2F521E7DFF8FF
:100FA000FC80304FD8F8003003EBD3735B10C8F8E7
:100FB00000302EE5314A049212680692904237DDE5
:100FC000274A1288012A00F0BC80274A099011881C
:100FD000264A0891204607920FF0E8FD079A0899E3
:100FE000DFF8BC9052F82110D9F800500FF032FE13
:100FF000059B2B4405930FF0F3FF0599099B069A77
:101000009942C2EB010EA8BF1946704580F2BE801E
:10101000891A00FB01110EF1010291FBF2F2D8F8DE
:1010200000100A4402EBD2725210C8F80020FEE40D
:10103000D8F80020DFF8689002EBD2725210D9F88D
:101040000050C8F80020F2E40EA0FF1F509DFF1FC3
:10105000608AFF1F809EFF1FA8260100589FFF1F68
:101060003A9DFF1F809CFF1FD49CFF1FB8290100E1
:10107000289DFF1F5C9EFF1FEC9EFF1F609EFF1FB1
:10108000A49CFF1FEE9CFF1F8889FF1F8E9CFF1FE3
:10109000CDCCCC3EBC89FF1F9A99193F049FFF1FFE
:1010A000E89EFF1F464A08901188464A079120464D
:1010B00006920FF07BFD069A0799DFF80C9152F823
:1010C0002110D9F800500FF0C5FD059BE91A0591D4
:1010D0000FF086FF0599089B049A9942C2EB010E16
:1010E000B8BF1946704558DA891A00FB01110EF194
:1010F000010291FBF2F2C2E60499521A00FB02F2DD
:1011000092FBFEF2BBE60FF051FD039A52F8291054
:101110000FF0A0FD014600200FF092FC0FF060FFE1
:10112000009A9542C8EB0503A8BF1546C8EB050514
:101130009842BABF00FB05550133454395FBF3F5D3
:1011400011E71F491F4A089020460D8807920FF0AB
:101150002DFD079ADFF8709052F82510D9F800504D
:101160000FF078FD014600200FF06AFC059B2B4430
:1011700005930FF035FF0599089B069A9942C2EB3B
:10118000010EA8BF19467045FFF642AF069A891AAC
:1011900000FB01F191FBFEF241E7049A891A00FB82
:1011A00001F191FBFEF26AE6B842D4BFC3EB000145
:1011B000C3EB070104FB01F172E51F46A1E400BF88
:1011C000D49CFF1FB8290100E89EFF1F08B5244BDF
:1011D0001B88FBB1234B1B78FBB1234B1B78E3B17E
:1011E000224B1B78CBB1224B1B78B3B1214B224849
:1011F0001A78C2B9214A2249008812880968024433
:10120000B1EB620F09DD01221A706420BDE80840CD
:1012100005F066BC174A117801B908BD1370BDE826
:10122000084008F01DBB154A164900881288096855
:101230000244B1EB620FF0DD00221A7008F010FBDF
:10124000642005F04DFC642005F04AFC642005F0A4
:1012500047FC4FF41670BDE808400CF0FBBE00BF21
:101260006E9EFF1F289FFF1F299FFF1F2A9FFF1FA2
:101270002B9FFF1FB49CFF1FCC9CFF1FC49EFF1F12
:10128000E89CFF1FAC9CFF1F38B5114C232025782C
:101290000CF08EF90F4A42F82500131F02F1C4002A
:1012A000002253F8041F83420A44FAD123780A49E2
:1012B00007480A4C0133DBB2322B81FB025108BFD5
:1012C0000023D217C2EB21120370226038BD00BF89
:1012D0009C9CFF1F709DFF1F1F85EB51C09EFF1F31
:1012E0002DE9F04FB84CB94D2068B94F83B00FF0DD
:1012F0005DFCB8490FF0AEFC064610200DF09CF8DE
:101300000FF054FCB4490FF0A5FC31460FF09AFBE6
:101310000FF066FE2988206088423B8843DA9E46AB
:101320005B1A7F2B4FF0000247DDD2015E1C92FB5F
:10133000F6F2AA4EDFF8C882B6F800C0C8F800205E
:10134000BCF1190F00F0DF80BCF11A0F00F017811B
:10135000BCF11E0F00F020810126B146A04A128880
:10136000002A00F09D808842C0F207817045D4BFFA
:10137000C1EB0000C1EB0E009A42BABF02FB0000B5
:101380000133504390FBF3F3964A1360964B188851
:10139000C0B9964A1288AAB9954B197801B11A704A
:1013A00003B0BDE8F08F9842D4BFC1EB0002C1EB9F
:1013B00003029E465B1A7F2BB7DCC2EBC21292FB84
:1013C000F3F2B6E72988D4F800E0DFF80082DFF80E
:1013D000F8A171456CDCDFF818C29CF80020002AE7
:1013E0002ED14FF0010B04288CF800B028D1002E2C
:1013F00040F094817D4B18880028D1D0B9F1000FBE
:10140000CED023682C883A88A34280F265810023DD
:10141000141B7E2C774DD5BFC3EB8313C3EBC313D3
:101420005B00013493FBF4F42B680134A34203D036
:10143000C0B2E1B208F06CF92C6003B0BDE8F08FE7
:10144000012800F0F680022800F0EB800328D1D1BB
:10145000694B1B88092BCDD0002ECBD023682E885A
:101460003A88B34280F27B810023961B7E2EDFF800
:101470008CA1D5BFC3EB8313C3EBC3135B00013651
:1014800093FBF6F6DAF800300136B34203D0F1B23E
:101490004A2008F03DF9CAF80060ABE716469146CD
:1014A000BCF11E0F7FF472AF0022DFF858817EE09E
:1014B0004F4B1A78002A3FF473AF002401281C70A8
:1014C00000F0A480022840F00E81002E00F0A380DE
:1014D0004A4D2B68002B00F09E800420214608F026
:1014E00017F9424B2C60188800283FF459AFB9F126
:1014F000000F3FF455AFC0B2002108F009F93D4B91
:1015000000221A604CE7DFF8FC8098F80020C2B196
:10151000DFF8D890B9F800A0BAF1000F11D0DFF8C9
:10152000E89099F800B0934578D05FFA8AF07F216F
:1015300008F0EEF898F80030B6F800C089F80030EE
:1015400010E0DFF8C49099F800A0924566D0274BD0
:101550000021187808F0DCF898F80030B6F800C0E0
:1015600089F800301E4B1A88002A97D0BCF11E0F54
:1015700040F006810026B14619E00020FCE6DFF8C5
:10158000848098F80020002A0BBF012600264FF027
:1015900000094FF00109E1E6DFF86880104B98F888
:1015A00000601A88B6FA86F676094FF0000998F8B6
:1015B0000030002B3FF4E8AE2988B7F800E020683F
:1015C000C1EB0E03CFE600BFDC9CFF1F749EFF1F24
:1015D000709EFF1F9A99193FCDCCCC3EFA9EFF1FFB
:1015E000389FFF1F689DFF1FE49CFF1F0C9FFF1F7C
:1015F000009FFF1FC09CFF1FB09EFF1F6C9DFF1F21
:10160000E09EFF1FA49CFF1FA09CFF1F1EB1614D09
:101610002B68002B7BD1604B188865E70026B1460C
:101620009CE6002E3FF4E6AEDFF868A1DAF8002071
:101630002EE0002E3FF4DEAEB7F80080F045D4BFB8
:10164000C1EB0802C1EB0E02C1EB0808B8F17E0F36
:10165000DFF840A1D5BFC2EB8212C2EBC21252002A
:1016600008F1010892FBF8F8DAF8002008F1010807
:10167000424506D05FFA88F10120009308F048F84F
:10168000009B1888CAF8008002287FF4DFAE42462B
:101690002168B5F800803888414559DA0021C8EB47
:1016A0000008B8F17E0FD3BFC1EB8111C1EBC111AE
:1016B00008F10108490091FBF8F808F1010890458C
:1016C00006D05FFA88F10420009308F021F8009B0F
:1016D0001888CAF80080B9E69342D4BFC4EB03036C
:1016E000C4EB020394E6032827D12C4B1B88092B5B
:1016F00091D0002E8FD0274D2B68002B8BD04A2005
:10170000214608F005F8244B2C601888ECE62146A9
:1017100007F0FEFF204B2C601888E5E640207F2173
:101720008DE80C0007F0F4FF019B009A18885845DB
:101730001CD002287FF48AAE76E704287FF46BAFD2
:10174000002E3FF468AF2146402007F0E1FF62E73A
:101750008142D4BFC8EB0101C8EB00019FE793426F
:10176000D4BFC6EB0303C6EB02037EE6B8F8001055
:10177000DAF800E0B7F800808E45FFF665AF5DE768
:101780002988B7F800E020680026C1EB0E03B146B7
:10179000E9E500BF6C9DFF1F0C9FFF1FB09EFF1F60
:1017A00008B5114B1B88022B09D0052B07D0032B42
:1017B00015D0042B0BD00D4B01221A7008BD7F21D0
:1017C000412007F0A5FF094B01221A7008BD7F21B7
:1017D000092007F09DFF054B01221A7008BD40212A
:1017E000092007F095FFE6E7669DFF1F0E9DFF1F8E
:1017F00038B5074B074D1B88052B044606D02B68D0
:10180000834203D0C1B2052007F082FF2C6038BDAF
:10181000669DFF1F149FFF1F38B5124D124C2B8879
:10182000052B12D022684AB9022B0ED0033B012BA4
:1018300013D90E4A00231370236038BD0021052000
:1018400007F066FF2B88022B04D10021412007F00E
:101850005FFFEEE7052BE9D1F7E70021092007F04C
:1018600057FFE6E7669DFF1F149FFF1F0E9DFF1F9A
:10187000464B1B881D2B70B541D0454D0024454B70
:101880001B88022B16D0444B1B88022B54D028886F
:10189000424B002C1B780ADB8442A8BF044634B1BB
:1018A000002B3AD02046BDE87040FFF7A1BF002BC7
:1018B0002FD170BD3A4B1B78002B37D015200BF081
:1018C00077FE384B1860384A1288002ADBD0374A36
:1018D000186811888142D6DC354B2A881B888342E0
:1018E000A3EB0106A8BF03465B1AB242BABF02FBD4
:1018F00003330136534393FBF6F31C44C3E72A4BEF
:101900001C888CB12B4B224D1C78002CB7D02C8816
:10191000B5E7BDE87040FFF77FBFFFF741FF204606
:10192000BDE87040FFF764BF194DA8E711200CF027
:1019300083FD1C4B1860C6E70F200CF07DFD1A4B91
:101940001D4A1B881060002BA1D01C4AC0F53B63C8
:10195000118808338B429ADB194A288812889342EF
:10196000A2EB0105A8BF1346A842A3EB010306DAC8
:1019700000FB0333013593FBF5F31C4488E700FBC0
:1019800003F292FBF5F31C4482E700BFFA9EFF1FAF
:10199000029FFF1FCE9EFF1F5C9EFF1F0E9DFF1F1D
:1019A000809EFF1F909CFF1F669DFF1F0A9DFF1FCB
:1019B000F89EFF1FA49CFF1F789EFF1F649DFF1FC2
:1019C000E49EFF1FF8B510200CF036FDC830B0F5CE
:1019D000FA7FC0F29680B0F57A6F0146A8BF4FF447
:1019E0007A6101F51673B3F57A6FA8BF4FF47A6385
:1019F0009BB289B2914A924C11802220238008F038
:101A00000BF821888F4D904C242008F005F80E200B
:101A10000BF0CEFD40F6FF71C8308842A8BF0846E3
:101A200020EAE07000F5FA6283B28A42A8BF0A4653
:101A30000220194622802B8007F0EEFF2188042027
:101A400007F0EAFF01200CF0F7FC044600200CF040
:101A5000F3FCA042B8BF204600F1C801B1F5FA7FFF
:101A6000C0F2D180B1F57A6FA8BF4FF47A6101F569
:101A70004873B3F57A6FA8BF4FF47A639BB289B20B
:101A8000724A734C11800A20238007F0C5FF218819
:101A90000C2007F0C1FF0F200CF0CEFCC0F53F6119
:101AA0000431B1F5AF6FC0F2AB80B1F5FA6FA8BFEA
:101AB0004FF4FA6189B2674BC0F54360B0F5AF6F80
:101AC0001980C0F29A80B0F5FA6FA8BF4FF4FA609F
:101AD00083B2614CA420238007F09EFF2188A620BA
:101AE00007F09AFF15200BF063FD00F59671B1F534
:101AF0002F7F0BDB41F25C23994240F3898019462A
:101B000008E040F24C434FF4FA7173E740F214538B
:101B10004FF42F71514A1180514C524D23800620B1
:101B200007F07AFF2188504E082007F075FF002744
:101B30004FF4AF74F9B24D4809F078FD55F8043B05
:101B4000C3F5967300FB03F086FB0023C017C0EBC0
:101B50006310844207F10107A8BF0446062FE9D1AC
:101B6000434F414E0025E9B2424809F05FFD57F866
:101B7000043BC3F5967300FB03F086FB0023C017FC
:101B8000C0EB6310844205F10105A8BF04460C2D8B
:101B9000E9D1394F344E0025E9B2384809F046FD05
:101BA00057F8043B304AC3F5967300FB03F086FBFD
:101BB0000013C017C0EB6310844205F10105A8BFF4
:101BC00004460C2DE8D1A4F11401312931DD40F295
:101BD0003A73A4F5B97403FB04F482FB0432E417EE
:101BE000A4EB621289B232322548264B01801A607A
:101BF0002A20BDE8F84007F00FBF4FF4AF6368E755
:101C00004FF4AF6157E740F214534FF4FA7137E7DE
:101C1000124A00F5617089B2B0F52F7F1180B8BF0C
:101C20004FF42F73FFF678AF8342A8BF03469BB2F1
:101C300072E740F26C723221D6E700BF749EFF1F3C
:101C4000709EFF1F609DFF1F2C9FFF1FC49EFF1FE4
:101C5000CC9CFF1F649DFF1FE49EFF1F0A9DFF1F7A
:101C6000F89EFF1F488AFF1FB5814E1BB89CFF1FBF
:101C7000188AFF1FEC9CFF1F2C89FF1F589DFF1F18
:101C8000269FFF1F048AFF1F2DE9F84F0C200BF041
:101C90005BFC0C200CF010F9C44914200CF01CF96A
:101CA000C349C44809F054F9022103200CF0AAF9F1
:101CB000022104200CF0A6F9022105200CF0A2F963
:101CC000022106200CF09EF901210A200CF09AF95D
:101CD000012109200CF096F901210D200CF092F958
:101CE000012128200CF08EF9012114200CF08AF932
:101CF000012116200CF086F9172001210CF082F941
:101D000004200CF071F9002844D005200CF06CF987
:101D1000002849D00023A84D06202B700CF064F950
:101D2000B0FA80F35B090024A44A137006F06CFA41
:101D30002E785EBB204607F099FEA14BA1491B8877
:101D40000F88A14ADFF8E4E2A04DA3F5AF7140F29D
:101D50003A7303FB01F382FB0312DB17A3EB62135D
:101D6000323301210D20CEF800302F700CF036F9FF
:101D700064200CF06FF94FF416710A200BF09EFFEF
:101D80005D21934809F08EFCA8B9FEE7BDE8F84F45
:101D900008F0EEBF06200CF027F90028B5D1864DDB
:101DA000034628700124BFE703200CF01DF9B0FAA8
:101DB00080F35B09AFE764200CF04CF931460A2050
:101DC0000BF07CFF4FF4967109200BF077FF5C213C
:101DD000804809F067FC00B9FEE764200CF03AF98E
:101DE000314609200BF06AFF4FF4967116200BF074
:101DF00065FF5B21784809F055FC00B9FEE76420D7
:101E00000CF028F9314616200BF058FF4FF496716C
:101E100017200BF053FF64200CF01CF931461720FB
:101E20000BF04CFF64200CF015F931460D200CF03E
:101E3000D5F86A4A6A481268DFF8F4B1DFF8A8A159
:101E4000684FDFF8F091DFF8F08100230121FEF701
:101E50002BFB0123CAF800603E60C9F800608BF8D4
:101E6000003004260F200CF0E7FAD9F800300344C4
:101E70000E20C9F800300BF09BFBDAF800309BF81D
:101E800000200344CAF800301520002A7DD00BF052
:101E90008FFB3B681844386006F0010080F00100B9
:101EA00004F00EFEB8F80030002B14BF4B20DC20ED
:101EB0000CF0D0F8013ED5D1D9F80030DAF8002086
:101EC00049493868DFF874E1484E002BB8BF033346
:101ED000002AB8BF033292100A604549454A098872
:101EE00012880028B8BF03309B10801038605F1A3A
:101EF00019443160CEF800703F4E404F4049C9F858
:101F00000030C2EB000E0244C7F800E032600B6004
:101F10000CB1FFF757FDB8F800305BB94FF4FA7019
:101F200004F0DEFD04F0C8FD06F096FC4FF4AF604F
:101F30000CF090F8334B012404201C600CF054F892
:101F400010B9314B28701C70304B1B881C2B23D0D0
:101F50002F4C04F1C80523200BF02AFB44F8040F92
:101F600001200CF077F8A542F5D12A4A2A4B1078C7
:101F7000187007F085FC04F09BFD45F6BF52274919
:101F80002748BDE8F84F0BF0CBB811200CF054FAFD
:101F90003B68184438607FE7224B18880028D7D068
:101FA000214BC0B2197807F0B3FBD1E7001B3746CD
:101FB00040420F007091FF1FBC9CFF1F649EFF1FDB
:101FC000269FFF1FFC9EFF1FB5814E1B249DFF1FF8
:101FD000B89CFF1F589DFF1FEC9CFF1F2889FF1F07
:101FE0008C9EFF1F809CFF1F949CFF1F609EFF1F05
:101FF000148AFF1F5C89FF1F289DFF1F589FFF1F2A
:10200000409FFF1FF49EFF1FA59CFF1FFA9EFF1F0E
:102010006C9DFF1F7C9EFF1F5B9EFF1FA5050000A0
:102020001C9FFF1F2C9DFF1FD89CFF1F048AFF1FB2
:10203000809EFF1FE89EFF1FBA9EFF1FEC9EFF1FA2
:102040002DE9F04FAD4C2678012E95B000F0558269
:10205000C0F00B82022E00F0D880A949A94A91F85D
:1020600000801178A84ADFF83CE3A84DA84FA948A2
:10207000A94B0392A94A0192A94A9EF800B0009286
:102080002D78A84A3F7890F800E01B78DFF818A375
:10209000DFF818C3DFF818930292012E84BF0022E4
:1020A0002270A14AA1481370A14A80F800B01570AF
:1020B000A048A14A077082F80080A048A04A037097
:1020C0009CBF013626701170BEF1000F40F0748184
:1020D0009C4A10880D2800F0B9819B4C002020708C
:1020E000024604462DB197480088002840F0BA8186
:1020F0000546964806882544002E40F0678194489E
:10210000944C009E0078367824780130A0EB46008D
:10211000002C40F05682029C94F800E0CEEB0004C4
:10212000BEF1000F40F076820026DFF874E20398DB
:102130009EF800E00078A41BA4EB4E043C44CBEBDB
:10214000040410B1B7FA87F040099CF80060271822
:10215000BC1B1EB11EF1000618BF0126019F99F895
:10216000000097F800909AF800C07B4FC6EB040E71
:10217000C0EB0E00A0EB49008044C3EB0803A3EBC7
:1021800041010C2313FB0C113960744B744F754CD7
:1021900075481B880088D7F800C0744E2788744C97
:1021A0003688D4F800E0033BC0EBC00403EB4303E4
:1021B000C7EBC70001EB830364446E4F33447044A4
:1021C0006D4E57F8244056F820000C3B1D44254422
:1021D00005440AB1694B1960694A13689D4200F0D1
:1021E0003181684B684819680791079901601B683D
:1021F00008936648089B008815605B1A834284BF79
:10220000634B1D6015B0BDE8F08FDFF8A881614E0B
:1022100008AF0025E9B2604809F008FA58F8043B15
:10222000C3F5967300FB03F086FB00230135C0174E
:10223000C0EB63100C2D47F8040BEBD1574B384D16
:102240000095384DB3F800C00295109D09980F997C
:10225000404EDFF8C0A0DFF8B490DFF8BC806545E1
:1022600011AA8CCAAE46ACBF4FF0000E4FF0010E63
:102270008445D4BF0020012030708C4528480B9D38
:102280001F4E8AF800E0D4BF00210121017094455F
:102290002449DFF814A1D4BF002201220A709C4512
:1022A0003F4AD4BF00230123BC45AB46D4BF00271F
:1022B00001271370AC45164B0C9D1F70D4BF4FF017
:1022C000000B4FF0010B374B0F4A0392AC45DFF880
:1022D00034C0124A83F800B0D4BF0025012589F824
:1022E000005098F800309CF8001096F80080DFF855
:1022F000BCC02678DFF8B8900192CEE65A9EFF1F48
:10230000AC9EFF1FAE9EFF1F3C9DFF1FB39EFF1F95
:102310000C9DFF1F649FFF1FAD9EFF1FFE9EFF1FB2
:10232000119FFF1F129FFF1F5E9FFF1F5F9FFF1FD9
:10233000609FFF1F619FFF1F629FFF1F639FFF1F23
:10234000FF9EFF1F669FFF1FA49CFF1F8C9CFF1F0B
:10235000168AFF1F4C9FFF1FB49EFF1FD29EFF1FB8
:10236000689DFF1F109DFF1FF09EFF1F9E9CFF1F7B
:10237000349FFF1FB4270100F0210100449FFF1F7D
:10238000049DFF1F4CA0FF1FF09CFF1F0A9FFF1F13
:10239000509FFF1FB5814E1B589DFF1F269FFF1F9B
:1023A000139FFF1F0D9DFF1F659EFF1F5D9FFF1F5A
:1023B000249FFF1F2C89FF1FAF4AB04814880122B9
:1023C000182C027040F2058100248BE6012E00F0EB
:1023D0008F81022E00F0EE81032EA94B00F01F81A9
:1023E0001E78019B9CF800E01C78009B99F800C0C7
:1023F0001878039B93F80080029B1F78A6EB4E038E
:10240000A4EB8404CCEB030CC0EB80760CEB040350
:10241000C0EB8600034403EB480303EB810327B1C1
:1024200098490978002940F0608201269AF8001046
:102430009548C1F1060101EB4101334403EB8101F1
:102440000160A2E69149924B0968D0E6002D3FF465
:1024500044AE894A894E14880122182C327040F209
:10246000B8807446A0F10D0543E6DFF87092894FFD
:102470000DF120080025E9B2874809F0D7F859F88E
:10248000043BC3F5967300FB03F087FB0023013583
:10249000C017C0EB6310062D48F8040BEBD17F4B3F
:1024A000DFF83CA219880D9B00228B428AF800209D
:1024B00080F2A2807A4B8AF800507A497A4A7B48A7
:1024C00091F8008011787A4A1D7003920378794A56
:1024D000DFF810C2DFF810920192774A774E784DFC
:1024E000784892F800E0784A0092784A96F800B06E
:1024F0002D78077826780292CFE5DFF8F081654ED7
:1025000008AF0025E9B2724809F090F858F8043B8A
:10251000C3F5967300FB03F086FB00230135C0175B
:10252000C0EB63100C2D47F8040BEBD15B4B0C9DFB
:102530001F885F4B03935F4B01930B9B0A98099A8B
:10254000DFF8A0C1089EDFF8A0910F99BB429E461C
:10255000ACBF4FF0000E4FF0010EAF42D4BF0025CC
:1025600001258742109B8CF80050D4BF0020012029
:10257000504D89F800009742D4BF00220122B74293
:10258000D4BF4FF000084FF001082A709F42474A1D
:102590004448474E80F80080D4BF002301231370C5
:1025A000129A414886F800E08F42D4BF00210121F1
:1025B000974201701ADC00224648DFF824A102701D
:1025C0008BE7029C46B12678002E40F06081441EC5
:1025D000ABE50C3C012285E594F800E00138CEEB38
:1025E0000004BEF1000F7FF4A0AD9DE5119A974263
:1025F000D4BF00220122DFE70C9A374B9142CCBFB7
:10260000012200221A7040F3458105258AF8005006
:10261000234B52E7002E3FF487AD012685E51C7859
:10262000019B039893F80080009B9CF800601B7846
:1026300090F800C099F800700298A4EB4604E71BDC
:1026400090F800E0C3EB8374A8EB88003844C3EB38
:102650008403034403EB4C0303EB8103BEF1000F3F
:1026600040F0488101269AF80010074833440C24B2
:1026700014FB0131016088E5FA9EFF1FA49CFF1F37
:10268000168AFF1F139FFF1FB49EFF1FF09CFF1FA2
:102690004CA0FF1FB5814E1BB89CFF1F269FFF1F3C
:1026A000729EFF1FAC9EFF1FAE9EFF1FAD9EFF1FC1
:1026B0003C9DFF1FFE9EFF1F649FFF1F0D9DFF1F80
:1026C000B39EFF1F0C9DFF1F119FFF1F129FFF1F37
:1026D000EC9CFF1FD29CFF1F2B9FFF1F488AFF1FF0
:1026E000659EFF1F5D9FFF1F249FFF1F188AFF1F0E
:1026F000A34CDFF89CE2207805909EF800400098FB
:102700000494059C007800900134A4EB40040498E4
:10271000002840F0AF80029890F800E00498261A54
:10272000CEEB06000490BEF1000F40F09E80744690
:102730000398944E00780290049836780396041B10
:10274000A4EB460402983C44CBEB0404002800F0C0
:102750008780B7FA87F040099CF800602044871B07
:102760001EB10398061C18BF0126019C99F80000B1
:102770002478BE1B301AA0EB440080440098C3EBC1
:102780000803A3EB4103002867D1BEF1000F40F01E
:10279000BB807344002C5ED100290CBF00206FF079
:1027A00009009AF80010784C03440C2010FB01310A
:1027B0002160EAE4029E009C36780296019E24780D
:1027C000009434786F4E714899F800E0019496F8BF
:1027D00000906F4C9DF8086086709DF80060067050
:1027E00080F806E09DF8046080F803909CF800C033
:1027F0002478DFF8B491DDF800E080F808800771F4
:1028000080F805C0C671417244704FF00008012085
:10281000019500215D4C0D465FFA88FC4F467646D7
:1028200007E0022809D00A290BD014F8016F17F825
:10283000010F864201F10101F3D101350A29EDB200
:10284000F3D1092D72D808F10108B8F1100F36D074
:1028500019F80A0FDDE70020A3E74FF0000E98E714
:10286000029879E7CEEB040004900098041C18BF8E
:1028700001245DE7009800284ED0029890F800E00F
:10288000BEF1000FEED1601E0490744650E7841B29
:1028900001264AE40B9A3F4B9142CCBF0122002211
:1028A0001A703EDC0A9A3C4B9142CCBF01220022B6
:1028B0001A7052DD03258AF80050384BFDE5304888
:1028C00037490478C86B0399019D09780134204485
:1028D000CBEB0000084400219AF800402A4B401A34
:1028E0000C2111FB040119604FE41BF1000618BF15
:1028F00001269BE52349097800293FF4B3AE1BF17B
:10290000000618BF0126AEE6039800280CBF4FF062
:10291000000E4FF0090E3CE7029890F800E03046B8
:10292000FDE604258AF800501C4BC6E514481C49F6
:10293000047851F828000399019D09780134204456
:10294000CBEB000066460844002BC4D0002EC2D159
:10295000BBF1000FBFD00121BEE7099A114B914294
:10296000CCBF012200221A7004DD02258AF8005033
:102970000A4BA2E5089B994218DD01259AE500BFA4
:10298000168AFF1F139FFF1FB49EFF1F309DFF1F5E
:102990004C9FFF1F2A9FFF1F299FFF1F729EFF1F33
:1029A000C489FF1F289FFF1F14270100134B1D78A8
:1029B000012D21D9124A8AF800501288002A3FF4CA
:1029C0007CAD104A1288013A92B2062A3FF675ADE4
:1029D0000D4A1278002A3FF470AD0C4A1268012AA1
:1029E0007FF46BAD0A4A0B4E10680C2290FBF2F19B
:1029F00002FB1102328060E535465EE5729EFF1FE4
:102A0000DC9EFF1F7E9EFF1F629DFF1FF49EFF1F27
:102A1000509FFF1FB89EFF1F2DE9F04F3A4B1B78C8
:102A20008BB0002B6BD10E200AF0C2FD0EF0BEF869
:102A300001463648364E374DFDF77CFD3348FDF7ED
:102A40004FFD0EF0CDFA80F30C003060FFF7F8FA7E
:102A50002C68012C7AD0022C00F0A782032C00F005
:102A6000B9832D4E2D4C33682D4A2E4E0993099B68
:102A7000316812882360591A013A9142274F00F2B7
:102A80008F82294E32689A1A0D2A00F27882274ED8
:102A900032689A1A132A00F26D82254E32689A1A09
:102AA000252A1AD9234B1B88002B40F05481224B36
:102AB0001B78002B40F04F81FEF7E6FB1F4B1B8875
:102AC0001B3B9BB2022B04D81D4B1B78002B40F004
:102AD000458104F017F8236833601A4D2A689B1A61
:102AE000502B00F20382184B1B88012B00F01B8235
:102AF00006F0A2FE06F0D0FC0BB0BDE8F08F07F0A8
:102B0000BFFF0BB0BDE8F08FBC9CFF1F8C9EFF1F6A
:102B1000C89EFF1FF49EFF1F4CA0FF1F889EFF1F33
:102B2000C089FF1F5C9DFF1F449DFF1F1C9DFF1F51
:102B3000209DFF1F6E9EFF1FB49CFF1FFA9EFF1F6C
:102B4000A49CFF1F689EFF1FCC9EFF1FDFF80C9305
:102B50009C4AB9F800001378834204D0C3B21846E7
:102B6000137006F0A5FDDFF8F082974AB8F8003040
:102B70001178994204D0954F3978002940F0E886C1
:102B8000934A33681288934E9A42C0F2F180924A77
:102B90001278002A40F0EC80DFF8C4A2BAF80030C6
:102BA00023B98E4B1B88002B00F0FB848C4A8D4B85
:102BB00011881B888C4A0B4412685B1093428B4A25
:102BC000126880F29D8400219342B4BF01230B461A
:102BD00004910093ACBF4FF0010B8B4605910E2082
:102BE0000AF0E6FC824B834A1B68176803930133A3
:102BF000A7F25232002B8446029240F3D086802BFB
:102C0000A8BF80237C4A7D4912780191002A00F0F8
:102C1000B9800978914200F0B580B8F80010DFF86B
:102C200038E2994201F0ED806849AEF80030744B0B
:102C30004FF0010E81F800E01978DFF828E2019BDF
:102C40008EF800101A70009B002B00F00D81BAF86E
:102C50000030002B00F008816A4B1B685A1C002AC8
:102C600040F3A186802A00F39D86674C6749684837
:102C70002488098800682144B0EB610FC1F23683D3
:102C8000A3F148020F2A02D8473BA9F800300E20D2
:102C90000AF08EFC6FF454731F44874202DC5D4BD4
:102CA00000221A705C4B1B88002B00F021845B4BC8
:102CB0005B4A1B781178994240D0002B3ED059498D
:102CC0000C78002C00F03387574991F800C0BCF114
:102CD000000F40F02A87554F0097554F55480297EF
:102CE000524F007887F800C0514F4FF0010E87F81F
:102CF00000C081F800E0002841F0DA804E490978F0
:102D0000002900F0F6874D4903910C460978002907
:102D100040F0EC874A48464F00783970012102970D
:102D2000217058B141484049009000200870009936
:102D3000029F0870039901243C7008701370414B86
:102D40001B88A3F11B02012A40F2C6851D2B00F04F
:102D500010863D4C87E6FEF739FAADE63B4B1B7813
:102D6000002B3FF4B6AE2B68012B7FF4B2AEB2E677
:102D70003168374A069106983649106002220B6086
:102D80002A6009E71E49DFF8DCE0097800293FF4F2
:102D900056AF9EF8000081423FF451AF03984B2894
:102DA00040F3F6871833802BB8F80000A8BF8023C3
:102DB00098423FF444AF284803800448012303703D
:102DC0003DE700BF5B9EFF1F249DFF1FA59CFF1FCB
:102DD000609DFF1F4CA0FF1FB49CFF1F4A9DFF1F5B
:102DE000CC9CFF1FC49EFF1FE89CFF1FAC9CFF1FD5
:102DF000449FFF1F949CFF1F3A9FFF1FFC9CFF1FD7
:102E00003B9FFF1FB49EFF1F749EFF1F709EFF1FFE
:102E1000DC9CFF1FC69CFF1F7E9EFF1FD29CFF1FD6
:102E2000849CFF1F619FFF1FBC9EFF1F109FFF1F01
:102E3000629DFF1F629FFF1F5E9FFF1F009DFF1F80
:102E4000A49CFF1FFA9EFF1F889EFF1FFF9EFF1F6F
:102E5000149DFF1F849EFF1FFC9EFF1F7C9EFF1F73
:102E6000089DFF1FFD9CFF1F029B9C45BFF60FAFF7
:102E70008B4B1B88002B3FF40AAFBBF1000F7FF494
:102E8000EBAE884B1B881BB1059B002B7FF4E4AE97
:102E9000049B002B3FF4FBAE834B1A78002A7FF48F
:102EA000F6AEDFF8809299F8004001221A70002CEB
:102EB00040F044837D4B1B78002B02F0D8807C4B84
:102EC0001B78002B02F09B837A4B1B78002B7FF43E
:102ED000DEAE794B1B78002B3FF4D9AEB8F800304A
:102EE00076490A3BA8F800300A70D0E605F0D4F91C
:102EF000734B1B7873B9734B1B785BB9724B1B78A0
:102F000043B9724B1B782BB9714B1B7813B903F083
:102F1000CFFD01E003F0D8FD23682B606D4B1B88CB
:102F2000012B7FF4E5AD6C4A6C4B11686C481A7844
:102F3000A1F118032A2101FB03F10160002A00F02E
:102F4000C182684C2368994200F36A8310DA6648AC
:102F50000278002A40F09287644A1068D0F17F001E
:102F600048BF0330801001301B1A994242F3D086CB
:102F70002160A9E2FEF77CFC236833608DE5FDF754
:102F800015FDFEF7ADF95A4B1B88032B00F02B857E
:102F9000584B1B88032B00F022852368336076E5AD
:102FA000FDF750FC3B6833606BE5534A3468118889
:102FB000A14204DB464B1B78002B00F061834F4E8F
:102FC0004F48336807934F4B079A00681B88121AC3
:102FD0009A4200F2AD80002B00F0AA804A4B1A887A
:102FE000002A3FF4B6AE494B49481B680088A3420B
:102FF000B8BF2346994241F37281464B1960DFF80E
:10300000288188F80020344FFDF71CFC38687F28A1
:1030100040F37D85404B7F3883FB0032C317C3EB01
:10302000620303EB4303A0EB830073303B4B01933C
:103030001B883860002B40F0D686234B00931B780A
:10304000002B00F0CA83364C2378002B00F0C58398
:10305000DFF8D890DFF8C0A04FF0000B0CE003F1D0
:103060007300C0B298F8001006F07AFB23780BF1D9
:10307000010B5B4540F3B1833B6859F8040F1844DA
:10308000A0F17F038AFB0321DA17C2EB610202EB96
:1030900042027F28A3EB8203E1DCFDF7F3FAE0E7CD
:1030A0004A9DFF1F829EFF1FC69CFF1F5E9FFF1F42
:1030B0005F9FFF1F609FFF1F619FFF1FA59CFF1F5A
:1030C000629DFF1FBC9EFF1F109FFF1F009DFF1FE3
:1030D000B49CFF1FCC9EFF1F509FFF1F0E9DFF1F24
:1030E000309FFF1F4C9DFF1F189FFF1F149FFF1F46
:1030F000CE9EFF1F5C9EFF1F609DFF1F4CA0FF1F09
:10310000149DFF1F489DFF1FA29CFF1F849EFF1F51
:103110002C9FFF1F889CFF1FABAAAA2AE29CFF1FBF
:103120008489FF1F659EFF1F3D9DFF1F5C89FF1F58
:10313000554B564A1B681088554AA342B8BF2346D0
:10314000994200F38482534C12888342A8BF0346FD
:103150002360002A7FF453AF9942C8BF134640F35F
:103160007D82401AB0F5804FAABF9B03C3EB833327
:10317000013093FBF0F0FDF74BFBC0F3C6100DF0F0
:1031800015FD454B044618880DF010FD43490746D0
:1031900020460DF05FFD014638460DF05BFD2146EF
:1031A0000DF050FC4FF07E5104460DF0F1FE00286A
:1031B00041F079803A4920460DF008FF002840F0A0
:1031C000718620460DF032FFC0B2DFF8F48088F837
:1031D000000018E7334B34681988A14274DD324B84
:1031E0001B78002B70D1DFF8DC9099F800007F2865
:1031F00040F34086A3F155337F3803F1004383FB4E
:103200000032C317C3EB620303EB4303A0EB83005D
:103210007330264B01931B88C0B289F80000002B45
:1032200041F03380224B00931B78002B00F0AC84DC
:10323000204C2378002B00F0A7841F4FDFF87C8000
:103240004FF0000A0AE003F17300C0B206F0B0FAD2
:1032500023780AF1010A534540F3968457F8043F56
:1032600099F800001844A0F17F0388FB0321DA17C6
:10327000C2EB610202EB42027F28A3EB8203E2DC95
:10328000FDF700FAE1E700BF849EFF1F2C9FFF1FA0
:10329000A29CFF1F889CFF1F3C9FFF1FCDCCCC3DF5
:1032A0000000FE42609DFF1FB49CFF1FE29CFF1FB9
:1032B000109FFF1F8489FF1F5C89FF1FABAAAA2AEA
:1032C0003D9DFF1FB29EFF1FB84F38687F2840F317
:1032D000CC81B74B7F3883FB0032C317C3EB62034B
:1032E00003EB4303A0EB83007330DFF8249399F8DA
:1032F00000A0824500F01782AE4B1B88002B43D103
:10330000AD4AAE4812680088914205DC8242D4BFC3
:10331000C1EB0203C1EB0003411AB1F5804FA6BF18
:103320009B030131C3EB833393FBF1F0FDF770FA9C
:10333000C0F3C6100DF03AFCA14B044618880DF0FE
:1033400035FCA049804620460DF084FC01464046ED
:103350000DF080FC21460DF075FB4FF07E510446C8
:103360000DF016FE002840F00A87974920460DF020
:103370002DFE002840F0938520460DF057FEC0B288
:10338000DFF8908288F80000BAF17F0F40F3B8832D
:103390008748AAF17F0A80FB0A304FEAEA73C3EB41
:1033A000600000EB4000AAEB80007330874B009375
:1033B0001B78C0B289F80000002B40F01883844BC2
:1033C00003931B78002B40F04985824B02931B78B6
:1033D000002B40F07C87804B0193029B1B78FBB154
:1033E0007E4B1B88012B00F0C185022B01F04D8024
:1033F000032B01F08C81042B01F09783052B01F046
:103400003884062B01F0FF85072B01F0BB87082BC2
:1034100002F0BA80092B02F0BF810A2B02F09283DE
:10342000009B1B78002B00F07484019B6A4C198868
:10343000002900F0FB8438687F2840F365835C4BEB
:103440007F3883FB0032C317C3EB620303EB4303F4
:10345000A0EB830073303860002940F0AA84009B01
:103460001B78002B00F06B815D4C2378002B00F063
:103470006681DFF8A4A1DFF89C814FF0000B0CE01F
:1034800003F17300C0B298F8001006F069F92378D0
:103490000BF1010B5B4540F352813B685AF8040F76
:1034A000434A1844A0F17F0382FB0321DA17C2EBE1
:1034B000610202EB42027F28A3EB8203E0DCFDF70E
:1034C000E1F8DFE7474B1960474B1B68A92202FB75
:1034D00003F3002BBCBF03F57F533F339B13543BD7
:1034E000194481F30C0128200AF0E8FBFFF700BB28
:1034F000384C3E483549364A237003700B701DE442
:1035000093424FF0000B80F2B3800123CDF800B05E
:10351000CDF814B00493FFF762BB354B1B78002B3A
:103520007FF4B5AB039B334A243B83F34703D9B203
:103530005B20136006F0ECF899F80040032C30D1C2
:10354000DFF8D88098F80030002B42F05E822A4FD6
:103550003B78002B42F04C82254C2378002B42F024
:103560003A82264B1B78002B42F02882244A138093
:10357000244B1B78002B42F014820E4B7F221A80C2
:1035800098F800306BB93B785BB923784BB91E4A89
:103590007F210720138006F0BBF87F210B2006F067
:1035A000B7F81A4B1F68FFF772BB00BF509FFF1F91
:1035B000ABAAAA2AA29CFF1F889CFF1F2C9FFF1F5B
:1035C0003C9FFF1FCDCCCC3D0000FE42109FFF1F53
:1035D000009DFF1F629DFF1FE29CFF1F7E9EFF1F3D
:1035E0008489FF1F4C9DFF1FBC89FF1FBC9EFF1FCE
:1035F000619FFF1FC89CFF1F609FFF1F5F9FFF1FF2
:10360000529DFF1F629FFF1FB09EFF1F949CFF1FD4
:10361000B29EFF1F3D9DFF1F5C89FF1F5E9FFF1F26
:10362000B64A1078002840F05783B54A1268D2F1A4
:103630007F0248BF033203EBA202531CB14A23604E
:103640009942B8BF1160FFF63FAF19463CE7AE4B59
:1036500012881960002A7FF4D2AC0B469842D4BF7E
:10366000C1EB0003C1EB03037BE5FDF70BF83CE680
:103670000123CDF810B0CDF800B00593FFF7AFBA35
:1036800001232B60A14EA24CFFF7EDB9029B1B78E2
:10369000FBB1A04B1B88012B00F0EA84022B00F049
:1036A0007386032B01F0A980042B01F06382052BA4
:1036B00001F05683062B01F0AF84072B01F0AF8594
:1036C000082B01F01987092B02F02F800A2B02F03A
:1036D000C381019B1B88002B00F07483009B1B7827
:1036E0003BB9039B1B7823B9029B1B78002B01F08D
:1036F0000480894B1B78002B00F0FE8087490B78F3
:10370000082B00F2F98086483A680068854C01333E
:10371000DBB25F1E101A44F827000B70824B34682E
:10372000198889F800208C42784E7FF712AB3268F6
:103730007E4B0892089A764C1A60FFF794B9039B67
:103740001B78002BA2D03B68A3F10C007F2840F32C
:10375000828377488B3B80FB0320DA17C2EB600043
:1037600000EB4000A3EB800303F17300DFF8D4818A
:10377000C0B298F8001005F0F3FF009B1B78002BF7
:1037800084D0664C2378002B80D0DFF8BCA14FF0AA
:10379000000B0CE003F17300C0B298F8001005F0C4
:1037A000DFFF23780BF1010B5B457FF76FAF3B68C1
:1037B0005AF8040F5E4A1844A0F18B0382FB0321E0
:1037C000DA17C2EB61020C3802EB42027F28A3EB4E
:1037D0008203DFDCFCF756FFDEE74F4B1B78002B44
:1037E00040F0F6823B68534A1278002A45D0A3F194
:1037F0000C007F2840F33B834D4A8B3B82FB032127
:10380000DA17C2EB610202EB4202A3EB820303F17F
:103810007300C0B298F8001005F0A2FF009B1B785F
:1038200053B33E4C23783BB3DFF81C91DFF800A183
:103830004FF0000B0BE003F17300C0B298F80010DA
:1038400005F08EFF23780BF1010B5B4514DD3B681F
:1038500059F8040F1844A0F18B038AFB0321DA17EF
:10386000C2EB61020C3802EB42027F28A3EB820319
:10387000E1DCFCF707FFE0E73B682F4A1278FAB17A
:10388000244A1288012A00F07D84022A00F07B86F7
:10389000032A01F02F80042A01F09381052A01F008
:1038A000CC82062A01F0D083072A01F01384082A6B
:1038B00001F0D386092A01F090870A2A02F00A81D2
:1038C000019A1288002A00F095821C4A104C13704D
:1038D00003232B60FFF7C7B8DFF8708098F800303B
:1038E000002B40F01881164F3B78002B40F01485D8
:1038F000074C3B70FFF7B7B83A680FE7189FFF1FF8
:10390000149FFF1F4C9DFF1F889CFF1F4CA0FF1F93
:10391000889EFF1F7E9EFF1FBC9EFF1F8489FF1F86
:10392000A89CFF1F6089FF1F609DFF1FF89FFF1F5E
:10393000ABAAAA2A009DFF1F629DFF1FB29EFF1F18
:10394000A09CFF1F3D9DFF1F5C89FF1FA49CFF1FC4
:10395000DBB21846137005F0B9FEB04BB0491A46F9
:10396000B04B184600230B703B7013700370FFF7C9
:1039700007B9DFF8CC8298F80030002B40F0D781EF
:10398000A94F3B78002BB3D0A84BA94C1988A22093
:1039900006F042F898F800303B70FFF764B8012356
:1039A000FFF730B98024A349A34BA44A09881B8898
:1039B00012680B44B2EB630FBFF669A9A04B1B78EA
:1039C000002B40F02482B8F800309E4AA3423FF416
:1039D0005EA99D4B148001221A70FFF758B9FCF7BD
:1039E000B9FEFFF7DABAFCF75FFEFFF7D1BA974BE3
:1039F00001931B88002B42F085818A4B0393944BE3
:103A00000293944C23786BB3DFF85C82DFF848A212
:103A10004FF0000B09E003F17300C0B205F0C8FEDF
:103A200023780BF1010B5B451CDD58F8043F99F836
:103A300000001844A0F17F038AFB0321DA17C2EBD0
:103A4000610202EB42027F28A3EB8203E3DCFCF776
:103A500019FEE2E77E4B029305F0AAFE009B1B785D
:103A6000002BCED1039B1B78002B3FF4B6AC99F80A
:103A70000030A3F10C007F2840F3EA8176488B3BAD
:103A800080FB0320DA17C2EB600000EB4000A3EBE1
:103A9000800303F17300C0B205F08AFE009B1B781F
:103AA000002B00F0CA816B4C2378002B01F0C582FB
:103AB000DFF8B481DFF8A0A14FF0000B0AE003F1BA
:103AC0007300C0B205F074FE23780BF1010B5B4567
:103AD0007FF783AC58F8043F99F800001844A0F130
:103AE0008B038AFB0321DA17C2EB61020C3802EB6D
:103AF00042027F28A3EB8203E1DCFCF7C3FDE0E791
:103B00005046FCF7BFFD51E4FCF7BCFDA3E4FCF715
:103B1000B9FDFFF78BBA514A1278002A40F0D581DF
:103B2000414F434C3B70FEF79EBF002008704C494C
:103B3000087840B1394900910978002900F0B58131
:103B4000009F002139704749097800297FF4DBA8DC
:103B5000002C40F0CE80002840F0CB80384C2F4F16
:103B600094F800E02F4C0394394C02942D4C2C49CE
:103B70002070374C0097087038702070BEF1000F2D
:103B80007FF4D3A8FFF7DAB8264B1B78002B6DD053
:103B900099F80030A3F10C007F2840F3C8832E4A27
:103BA0008B3B82FB0321DA17C2EB610202EB42027C
:103BB000A3EB820303F17300C0B205F0F9FD009B93
:103BC0001B78002B52D0234C2378002B4ED0264F4D
:103BD000DFF884804FF0000A09E003F17300C0B2FF
:103BE00005F0E6FD23780AF1010A53453EDD57F85A
:103BF000043F99F800001844A0F18B0388FB0321CF
:103C0000DA17C2EB61020C3802EB42027F28A3EB09
:103C10008203E2DCFCF736FDE1E700BF109FFF1FE7
:103C2000BC9EFF1F009DFF1FA09CFF1F029FFF1F48
:103C3000889EFF1F749EFF1F709EFF1FDC9CFF1F4E
:103C4000A49CFF1FFC9EFF1FA59CFF1FE29CFF1F63
:103C5000629DFF1F8489FF1FABAAAA2AFF9EFF1F38
:103C6000629FFF1F5E9FFF1F5C89FF1FA84B1B7891
:103C7000FBB1A84B1B88012B00F0D086022B00F073
:103C8000CB87032B01F04281042B01F0CD81052B62
:103C900001F01784062B01F0D884072B01F0E7858B
:103CA000082B01F07087092B01F0D5870A2B01F052
:103CB000A287019B1B88002B00F0F082964B1B789B
:103CC000002B40F0E682954B954A19883468002015
:103CD000012310602B6026E50130C0B2022886BFA8
:103CE0000021117010701946FFF7EEBB03980021F8
:103CF00001708C49097800293FF420A88449029179
:103D00000978002900F0AE87029800210170FFF7C2
:103D100015B8039B1B78002B7FF487AB029B1B78A5
:103D2000002B7FF482AB019B1988FFF784BB7E4A8E
:103D30001278002A3FF4F4AE7C4F387802F04CFF42
:103D40007B4B1B78002B00F0B78439887E2900F26A
:103D5000B384784CDFF80C922368D9F800209B1AC2
:103D60000F2B40F29680744B01311B8889B2398049
:103D70002BB1052B03D0C9B2052005F0C9FC6F4F4C
:103D8000226898F80030C9F800203B70FEF76BBE3F
:103D9000243B002BB8F8000040F3748498423EF4B2
:103DA0004EAF9BB26648A8F8003001230370FEF7BF
:103DB00046BFDFF89081C0B298F8001005F0D0FC43
:103DC000FFF74DBB5F4B3878197805F0C9FC85E4E7
:103DD0007F21402005F09CFC5B495C4A3B680B60FE
:103DE00000211170FFE4C0B298F8001005F0B8FC93
:103DF000FFF723B9D8B298F8001005F0B1FC3B6882
:103E000063E5534BDFF860E11978FEF718BF4B2CE0
:103E100040F34C821834802CB8F800304D4AA8BFCB
:103E20008024A3427FF4D5ADFEF731BF99F800009E
:103E300005F0BEFC2188FFF7FEBA029B1B78002B21
:103E40007FF4CEAA039B1B78002B7FF4EEAA6AE7CF
:103E5000FCF718FC1FE6FCF715FC87E43E4B0193CA
:103E60001B88002B7FF4F6AD294B0293FFE5FCF78E
:103E700009FCCEE4FCF706FCFFF7CBB90132D2B265
:103E8000022A40F25A82002202701946FFF71CBB38
:103E9000284C2A4F98F800303B70FEF7E4BD7F2095
:103EA000FFF76EBA7F20FFF790B9194F1A490297B2
:103EB0004FF0000C81F800C0009F02994FF0010EF6
:103EC00087F800E081F800C03DE6244F387802F022
:103ED00083FE174B1B78002B00F0368239887E2931
:103EE00000F23282134CDFF87C902368D9F800206E
:103EF0009B1A0F2BCDD91A4B0131188889B2398002
:103F0000002800F03D82C9B2C0B205F001FC36E7DE
:103F1000629DFF1F7E9EFF1FBC9EFF1F609DFF1FB7
:103F2000889CFF1FA49CFF1FFF9EFF1F029FFF1F77
:103F3000639FFF1F889EFF1F669DFF1FA09CFF1FA2
:103F4000A59CFF1F3D9DFF1FA89CFF1F8489FF1F8D
:103F50003B9FFF1FFC9EFF1FE29CFF1FD89CFF1F83
:103F60002C9DFF1F489FFF1FFD9CFF1FDFF89CA398
:103F700099F80000BAF80030DF4AE04CC31A82FB1F
:103F8000031ED917C1EB6E0101EB4101A3EB8103C5
:103F900003EB430354F8233018447F2840F3A684EE
:103FA0007F3882FB0032C317C3EB620303EB43038A
:103FB000A0EB83007330DFF858B3C0B205F0F8FB14
:103FC000BBF80030022B7FF62BAA99F80010BAF844
:103FD0000030C94ACB1A82FB030ED817C0EB6E0023
:103FE00000EB4000A3EB800303EB430304EB8303EC
:103FF000586808447F2840F318877F3882FB0032D6
:10400000C317C3EB620202EB4202A0EB82007330E3
:10401000C0B205F0CDFBBBF80030032B7FF600AA41
:1040200099F80010BAF80030B34ACB1A82FB030E9D
:10403000D817C0EB6E0000EB4000A3EB800303EB4E
:10404000430304EB8304A06808447F2840F35181B4
:104050007F3882FB0032C317C3EB620202EB4202DD
:10406000A0EB82007330C0B205F0A2FBFFF7D8B915
:10407000DFF898A23868BAF800309F4A9F4CC31AFC
:1040800082FB031ED917C1EB6E0101EB4101A3EBCB
:10409000810303EB430354F8233018447F2840F393
:1040A000A0847F3882FB0032C317C3EB620303EBAB
:1040B0004303A0EB83007330DFF85882DFF850B27F
:1040C00098F80010C0B205F04BFBBBF80030022B93
:1040D0007FF6FFAA3968BAF80030874ACB1A82FB0C
:1040E000030ED817C0EB6E0000EB4000A3EB80037B
:1040F00003EB430304EB8303586808447F2840F331
:1041000098867F3882FB0032C317C3EB620202EB52
:104110004202A0EB82007330C0B298F8001005F0A4
:104120001FFBBBF80030032B7FF6D3AA3968BAF81F
:104130000030714ACB1A82FB030ED817C0EB6E0019
:1041400000EB4000A3EB800303EB430304EB830489
:10415000A06808447F2840F3F4807F3882FB003257
:10416000C317C3EB620202EB4202A0EB8200733082
:1041700098F80010C0B205F0F3FAFFF7AABA0120D0
:10418000FFF7FEB8DFF884A15B49BAF800205B4C6A
:104190009A1A81FB020ED017C0EB6E0000EB4000B4
:1041A000A2EB800202EB420254F8220018447F285E
:1041B00040F31B84A0F17F0381FB0321DA17C2EBDC
:1041C000610000EB4000A3EB80007330DFF840B1EA
:1041D00098F80010C0B205F0C3FABBF80030022B0B
:1041E00050D93968BAF80030434ACB1A82FB030E23
:1041F000D817C0EB6E0000EB4000A3EB800303EB8D
:10420000430304EB8303586808447F2840F3E186A6
:104210007F3882FB0032C317C3EB620202EB42021B
:10422000A0EB82007330C0B298F8001005F098FA45
:10423000BBF80030032B25D93868BAF800302E4A75
:10424000C31A82FB031ED917C1EB6E0101EB4101BA
:10425000A3EB810303EB430304EB8304A36818443B
:104260007F2867DD7F3882FB0032C317C3EB620211
:1042700002EB4202A0EB82007330C0B298F800104B
:1042800005F06EFA3B68FFF71BBB05F091FAFEF7ED
:10429000C9BF0021402005F03BFA14E599F8000061
:1042A00005F086FA0AE50120FEF78FBF243C002CBA
:1042B000B8F8003040F32486A3423EF4E8ACA4B240
:1042C0000F4BA8F8004001221A70FEF7E0BC0D4B1E
:1042D00001931B88002B7FF4BFABFFF77EB80A4920
:1042E0008342A8BF03460B60FEF789BE1446FFF762
:1042F00065BBFCF7C7F9B6E6ABAAAA2A18260100E7
:10430000A59CFF1FE29CFF1F889CFF1FB89EFF1FFC
:10431000BA9CFF1F3D9DFF1FDD4BDE4C19886A20B4
:1043200005F07AFB98F800303B70FEF79CBBFCF779
:10433000A9F941E4FCF7A6F99FE702701946FFF7D7
:10434000C3B8FCF79FF913E7D34B1B78002B3FF45E
:104350009FAD3B88CE4F002B3FF49AADCD4CDFF89C
:1043600048932268D9F80010521A0F2A7FF691ADAF
:10437000CA4A013B108899B2398000287FF4C3AD46
:10438000C8B205F039FAFAE4DFF820A33868BAF8C1
:104390000030C34AC34CC31A82FB031ED917C1EBBA
:1043A0006E0101EB4101A3EB810303EB430354F8DE
:1043B000233018447F2840F328847F3882FB003262
:1043C000C317C3EB620303EB4303A0EB830073301B
:1043D000DFF8DC82DFF8DCB298F80010C0B205F03C
:1043E000BFF9BBF80030022B7FF673A93968BAF821
:1043F0000030AB4ACB1A82FB030ED817C0EB6E001D
:1044000000EB4000A3EB800303EB430304EB8303C7
:10441000586808447F2840F326867F3882FB0032A4
:10442000C317C3EB620303EB4303A0EB83007330BA
:10443000C0B298F8001005F093F9BBF80030032BD8
:104440007FF647A93868BAF80030954AC31A82FB4C
:10445000031ED917C1EB6E0101EB4101A3EB8103F0
:1044600003EB430304EB8304A36818447F287FF71E
:1044700068AF7F3882FB0032C317C3EB620303EBE4
:104480004303A0EB8300733072E6DFF820A299F8B3
:104490000000BAF80030824A824CC31A82FB031E25
:1044A000D917C1EB6E0101EB4101A3EB810303EBD3
:1044B000430354F8233018447F2840F37F837F3828
:1044C00082FB0032C317C3EB620303EB4303A0EB91
:1044D00083007330DFF8DCB1C0B205F069F9BBF8D6
:1044E0000030022B7EF69CAF99F80010BAF800302D
:1044F0006B4ACB1A82FB030ED817C0EB6E0000EBA1
:104500004000A3EB800303EB430304EB83035868F1
:1045100008447F2840F39F857F3882FB0032C31711
:10452000C3EB620303EB4303A0EB83007330C0B221
:1045300005F03EF9BBF80030032B7EF671AF99F819
:104540000010BAF80030564ACB1A82FB030ED81777
:10455000C0EB6E0000EB4000A3EB800303EB4303D2
:1045600004EB8304A06808447F287FF7C2AE7F383D
:1045700082FB0032C317C3EB620303EB4303A0EBE0
:10458000830073306FE5DFF824A14549BAF80020B5
:10459000444C9A1A81FB020ED017C0EB6E0000EB60
:1045A0004000A2EB800202EB420254F822001844C1
:1045B0007F2840F32E83A0F17F0381FB0321DA17CC
:1045C000C2EB610000EB4000A3EB80007330DFF82A
:1045D000E4B098F80010C0B205F0C2F8BBF80030A3
:1045E000022B7FF64FAE3968BAF800302C4ACB1A4E
:1045F00082FB030ED817C0EB6E0000EB4000A3EB6C
:10460000800303EB430304EB8303586808447F28CB
:1046100040F325857F3882FB0032C317C3EB62036A
:1046200003EB4303A0EB83007330C0B298F8001093
:1046300005F096F8BBF80030032B7FF623AE386800
:10464000BAF80030164AC31A82FB031ED917C1EB11
:104650006E0101EB4101A3EB810303EB430304EB88
:104660008304A36818447F287FF764AE7F3882FBF9
:104670000032C317C3EB620303EB4303A0EB8300D9
:104680007330FAE501283EF4DAAA0123FFF78ABB6A
:10469000D89CFF1F889EFF1F629FFF1F2C9DFF1F3E
:1046A000ABAAAA2A5C280100489FFF1FB89EFF1FE3
:1046B0003D9DFF1FBA9CFF1FCE4B1B78002B3FF484
:1046C000E7AB3B88CC48002B3FF4E2ABCB4CDFF8A8
:1046D0003C932268D9F80010521A0F2A7FF6D9AB02
:1046E000C74A013B128899B20180002A3FF447ABC8
:1046F000052A7FF440ABFFF742BB4FF47A43013BFE
:10470000FDD199F8000005F053F8FEF7F2BFDFF88D
:1047100000A399F80000BAF80030BA4ABA4CC31A9C
:1047200082FB031ED917C1EB6E0101EB4101A3EB24
:10473000810303EB430354F8233018447F2840F3EC
:10474000E8817F3882FB0032C317C3EB620202EBC1
:104750004202A0EB82007330DFF8B8B2C0B205F0BD
:1047600027F8BBF80030022B7EF65AAE99F800000D
:10477000BAF80030A34AC31A82FB0321DA17C2EB4E
:10478000610202EB4202A3EB820303EB430304EB5F
:1047900083035B6818447F2840F325847F380C220C
:1047A00090FBF2F302FB13007330C0B205F000F887
:1047B000BBF80030032B7EF633AE99F80000BAF850
:1047C0000030904AC31A82FB0321DA17C2EB610260
:1047D00002EB4202A3EB820303EB430304EB8304EB
:1047E000A36818447F287FF784AD7F380C2290FBA4
:1047F000F2F302FB1300733035E4DFF814A23868DB
:10480000BAF800307F4A804CC31A82FB031ED917C6
:10481000C1EB6E0101EB4101A3EB810303EB430309
:1048200054F8233018447F2840F370817F3882FB8E
:104830000032C317C3EB620202EB4202A0EB82001C
:104840007330DFF8D481DFF8CCB198F80010C0B233
:1048500004F086FFBBF80030022B7EF63AAF3868D2
:10486000BAF80030674AC31A82FB0321DA17C2EB99
:10487000610202EB4202A3EB820303EB430304EB6E
:1048800083035B6818447F2840F3B4837F380C228D
:1048900090FBF2F302FB13007330C0B298F80010E3
:1048A00004F05EFFBBF80030032B7EF612AF3868D1
:1048B000BAF80030534AC31A82FB0321DA17C2EB5D
:1048C000610202EB4202A3EB820303EB430304EB1E
:1048D0008304A36818447F287FF733AD7F380C2208
:1048E00090FBF2F302FB1300733041E4FBF7CAFEC6
:1048F000FFF761BBDFF818A14249BAF80020424C2B
:104900009A1A81FB020ED017C0EB6E0000EB40003C
:10491000A2EB800202EB420254F8220018447F28E6
:1049200040F3FA80A0F17F0381FB0321DA17C2EB89
:10493000610101EB4101A3EB81007330DFF8D4B0DA
:1049400098F80010C0B204F00BFFBBF80030022B47
:104950007FF698AC3868BAF800302A4AC31A82FB4E
:104960000321DA17C2EB610202EB4202A3EB8203DE
:1049700003EB430304EB83035B6818447F2840F395
:104980003C837F380C2290FBF2F302FB1300733060
:10499000C0B298F8001004F0E3FEBBF80030032B1F
:1049A0007FF670AC3868BAF80030164AC31A82FB3A
:1049B0000321DA17C2EB610202EB4202A3EB82038E
:1049C00003EB430304EB8304A36818447F287FF7B9
:1049D000B1AC7F380C2290FBF2F302FB1300733072
:1049E0004BE4FBF74FFEFFF767BBFBF74BFEFFF710
:1049F000EDBB00BF629FFF1F029FFF1F889EFF1F2E
:104A0000669DFF1FABAAAA2AEC280100489FFF1F42
:104A1000B89EFF1FBA9CFF1F3D9DFF1FDFF838A304
:104A200099F80000BAF80030C34AC44CC31A82FB9C
:104A30000317D917C1EB670101EB4101A3EB810318
:104A400003EB430354F8233018447F286ADD7F3892
:104A500082FB0032C317C3EB620202EB4202A0EBFF
:104A600082007330DFF8F4B2C0B204F0A1FEBBF8EC
:104A70000030022B7FF61DA999F80000BAF800302B
:104A8000AD4AC31A82FB0321DA17C2EB610202EBC3
:104A90004202A3EB820303EB430304EB83035B6853
:104AA00018447F2840F3AC827F380C2290FBF2F34D
:104AB00002FB13007330C0B204F07AFEBBF8003082
:104AC000032B7FF6F6A899F80000BAF800309A4A4E
:104AD000C31A82FB0321DA17C2EB610202EB420226
:104AE000A3EB820303EB430304EB8304A3681844A2
:104AF0007F2814DD7F380C2290FBF2F302FB1300B9
:104B00007330C0B204F054FEFFF7D3B8FBF7BAFD20
:104B100097E6FBF7B7FD1FE6FBF7B4FD0EE7FBF7E3
:104B2000B1FDEEE7FBF7AEFD9CE7DFF82CA299F8AC
:104B30000000BAF80030804A814CC31A82FB031E81
:104B4000D917C1EB6E0101EB4101A3EB810303EB2C
:104B5000430354F8233018447F28DADD7F3882FB82
:104B60000032C317C3EB620303EB4303A0EB8300E4
:104B70007330F1E5DFF8E0A13868BAF800306E4A2A
:104B80006F4CC31A82FB031ED917C1EB6E0101EBF8
:104B90004101A3EB810303EB430354F82330184492
:104BA0007F28B3DD7F3882FB0032C317C3EB62037B
:104BB00003EB4303A0EB8300733042E6FBF762FD97
:104BC00088E4DFF894A15C49BAF800205C4C9A1A9A
:104BD00081FB020ED017C0EB6E0000EB4000A2EB91
:104BE000800202EB420254F8220018447F2893DD31
:104BF000A0F17F0381FB0321DA17C2EB610000EB18
:104C00004000A3EB8000733098E6FBF73BFDFFF715
:104C1000DFBBFBF737FDDAE4DFF83CA199F80000D1
:104C2000BAF80030444A474CC31A82FB0317D9171D
:104C3000C1EB670101EB4101A3EB810303EB4303EC
:104C400054F8233018447F287FF76CAF7F3882FBFD
:104C50000032C317C3EB620303EB4303A0EB8300F3
:104C60007330FFE638480090384839490390FEF722
:104C70005CB8DFF8E4A099F80000BAF800302E4ADA
:104C8000344CC31A82FB0321DA17C2EB610202EB38
:104C90004202A3EB820303EB430354F8233018448E
:104CA0007F2840F3A4817F380C2290FBF2F302FBB3
:104CB00013007330DFF8A4B0C0B204F079FDBBF884
:104CC0000030022B19D999F80000BAF800300C22F4
:104CD000C11A91FBF2F302FB131302FB03435B685F
:104CE00018447F2840F384847F3890FBF2F302FB62
:104CF00013007330C0B204F05BFDBBF80030032B2F
:104D00007EF68EABBAF8003099F800000C22C11A7A
:104D100091FBF2F302FB131302FB0344A368184454
:104D20007F287FF7E6AA7F3890FBF2F302FB13009F
:104D30007330FFF798B900BFABAAAA2A1826010062
:104D4000842201005C280100109FFF1F009DFF1FAF
:104D5000BC9EFF1F3C210100B89EFF1FBA9CFF1F95
:104D6000DFF864A33868BAF80030CE4ACE4CC31AD4
:104D700082FB0321DA17C2EB610202EB4202A3EBD2
:104D8000820303EB430354F8233018447F2840F395
:104D900024817F380C2290FBF2F302FB1300733066
:104DA000DFF82883DFF828B398F80010C0B204F0C9
:104DB000D7FCBBF80030022B1AD93868BAF800309B
:104DC0000C22C11A91FBF2F302FB131302FB034303
:104DD0005B6818447F2840F3D4837F3890FBF2F35C
:104DE00002FB13007330C0B298F8001004F0B8FC56
:104DF000BBF80030032B7EF66CACBAF80030386894
:104E00000C22C11A91FBF2F302FB131302FB0344C1
:104E1000A36818447F287FF794AA7F3890FBF2F3A9
:104E200002FB13007330FFF7A3B9FBF72BFCFFF76E
:104E3000EFB8FBF727FCFFF76FB9DFF88CA29949B1
:104E4000BAF80020984C9A1A81FB0210D117C1EBD6
:104E5000600101EB4101A2EB810202EB420254F836
:104E6000220018447F2840F3BB80A0F17F030C2070
:104E700093FBF0F200FB12307330DFF854B298F875
:104E80000010C0B204F06CFCBBF80030022B1AD941
:104E90003868BAF800300C22C11A91FBF2F302FB19
:104EA000131302FB03435B6818447F2840F39D8380
:104EB0007F3890FBF2F302FB13007330C0B298F816
:104EC000001004F04DFCBBF80030032B7FF6DAA98C
:104ED000BAF8003038680C22C11A91FBF2F302FBD9
:104EE000131302FB0344A36818447F287FF722AA08
:104EF0007F3890FBF2F302FB13007330FFF7BDB96C
:104F0000012B3DF4C4AE0124FFF7DAB9DFF8B8A1F4
:104F100099F80000BAF80030624A644CC31A82FB68
:104F20000321DA17C2EB610202EB4202A3EB820318
:104F300003EB430354F8233018447F2846DD7F38C1
:104F40000C2290FBF2F302FB13007330DFF880B108
:104F5000C0B204F02DFCBBF80030022B19D999F82F
:104F60000000BAF800300C22C11A91FBF2F302FBE8
:104F7000131302FB03435B6818447F2840F38F80C0
:104F80007F3890FBF2F302FB13007330C0B204F0E1
:104F90000FFCBBF80030032B7EF68BAEBAF8003066
:104FA00099F800000C22C11A91FBF2F302FB1313D3
:104FB00002FB0344A36818447F287FF7B0AD7F3815
:104FC00090FBF2F302FB130073309AE5FBF75AFBF8
:104FD000BCE7FBF757FBFFF726B9FBF753FBDFE610
:104FE000FBF750FB49E7FBF74DFBFFF7DEBBFBF799
:104FF00049FB5FE6FBF746FB4FE4FBF743FBC7E4E7
:10500000FBF740FB57E5DFF8C0A099F80000BAF8BD
:105010000030244A264C34E6DFF8ACA03868BAF8F1
:105020000030204A224CA2E6DFF89CA099F800004C
:10503000BAF800301B4A1F4C70E7029B1B78002B0C
:105040007EF4CEA9FEF7F1B9DFF87CA01549BAF8D5
:105050000020174CF7E6FBF715FBFFF768BAFBF7E4
:1050600011FBFFF7E2BAFBF70DFBFFF7E1B9124BBB
:105070001B78002B00F0D682104B1B78002B7DF4A0
:1050800006AE0F4B1B78002B3DF401AEB8F8003094
:105090000C490A33A8F800300A70FDF7F8BDFBF799
:1050A000F1FA73E7ABAAAA2A3C210100EC2801001F
:1050B000E0290100842201005F9FFF1F609FFF1F06
:1050C000619FFF1FA59CFF1FB89EFF1F3D9DFF1FF7
:1050D000BA9CFF1FA44C2288002A00F02383A34916
:1050E000DFF89CB20988BBF800000331884227DD55
:1050F0009F48A0490088B1F800E0DFF87CC2181A88
:105100000C2190FBF1F901FB19004FF0900909FB0C
:105110000EFE01FB00E06FF00B0E5CF80000034494
:105120000EFB02307F2840F3CE847F3890FBF1F3F2
:1051300001FB13007330C0B298F8001004F010FBAC
:10514000BBF8002023881344022B23DD884B894AB7
:1051500038681B88B2F800C0DFF81CE2C31A0C21C3
:1051600093FBF1F201FB1232902303FB0CF301FBE2
:10517000023373445B6818447F2840F3A7857F3867
:1051800090FBF1F301FB13007330C0B298F80010EC
:1051900004F0E6FABBF8002023881344032B23DD38
:1051A000734B744A38681B88B2F800C0DFF8C8E156
:1051B000C31A0C2193FBF1F201FB1232902303FB83
:1051C0000CF301FB023373449B6818447F2840F3BF
:1051D0000B857F3890FBF1F301FB13007330C0B2F5
:1051E00098F8001004F0BCFABBF8002023881344A0
:1051F000042B7FF747A85D4B1B88012B7FF442A847
:105200003A68A2F10C007F287FF794A88B3A0C2013
:1052100092FBF0F300FB13207330FFF72EB8524CD3
:105220002388002B40F00D83DFF854B15049514AD8
:105230000988D7F80080B2F800E04F48C1EB080CAD
:105240000C229CFBF2F102FB11C14FF0900C0CFB05
:105250000EFE02FB01E16FF00B0E405880440EFB86
:1052600003807F2840F36A84A0F17F0393FBF2F070
:1052700002FB10307330414BC0B2197804F070FA61
:10528000BBF8002023881344022B23DD384A394B16
:1052900011883868B3F800C0DFF8DCE0411A0C224E
:1052A00091FBF2F302FB1311902303FB0CF302FBBF
:1052B000013373445B6818447F2840F3F1847F38DE
:1052C00090FBF2F302FB130073302C4BC0B2197841
:1052D00004F046FABBF8002023881344032B23DD97
:1052E000234A244B11883868B3F800C0DFF888E0FF
:1052F000411A0C2291FBF2F302FB1311902303FBE2
:105300000CF302FB013373449B6818447F2840F37D
:10531000CF847F3890FBF2F302FB13007330174BFE
:10532000C0B2197804F01CFABBF80020238813449B
:10533000042B7EF7CEA90D4B1B88012B7EF4C9A947
:105340003A68A2F10C007F2840F356818B3A0C207A
:1053500092FBF0F300FB13207330084BC0B21978B6
:1053600004F0FEF9FEF7B5B9409DFF1FD69CFF1F64
:10537000B89EFF1F669EFF1F142301003D9DFF1F67
:10538000BA9CFF1FCF4C2388002B40F06582DFF8CA
:1053900068B3CD49CD4A098899F80000B2F800E019
:1053A000DFF85883C1EB000C0C229CFBF2F102FBEE
:1053B00011C14FF0900C0CFB0EFE02FB01E16FF0EF
:1053C0000B0E58F8011008440EFB03007F2840F331
:1053D0007E83A0F17F0393FBF2F002FB1030733069
:1053E000C0B204F0E5F9BBF8002023881344022B77
:1053F00022DDB54AB54B118899F80000B3F800C01A
:10540000DFF8F8E2411A0C2291FBF2F302FB1311D0
:10541000902303FB0CF302FB013373445B681844D5
:105420007F2840F341847F3890FBF2F302FB1300A6
:105430007330C0B204F0BCF9BBF8002023881344D9
:10544000032B22DDA04AA14B118899F80000B3F884
:1054500000C0DFF8A8E2411A0C2291FBF2F302FB34
:105460001311902303FB0CF302FB013373449B687D
:1054700018447F2840F320847F3890FBF2F302FB2E
:1054800013007330C0B204F093F9BBF800202388F6
:105490001344042B7DF7C4AF8D4B1B88012B7DF487
:1054A000BFAF99F80020A2F10C007F287EF721AF52
:1054B0008B3A0C2092FBF0F300FB13207330FEF7C5
:1054C000D2BDDFF804A299F80000BAF80030814C90
:1054D000C11A0C2291FBF2F302FB131302FB03F33C
:1054E000E35818447F287FF771AD7F3890FBF2F3C3
:1054F00002FB1300733029E5774B1A88182A13D062
:105500003B681344A3F118007F2840F3C6830C20A6
:10551000973B93FBF0F200FB123303F173006F4BE8
:10552000C0B2197804F01CF96D4B6E491A78022A42
:1055300094BF013200221A701A7831F8120018282C
:1055400010D10424022A02F10100C2B288BF002255
:1055500031F81200182804D1013CF3D11A70FEF77B
:10556000B8B81A703B680344A3F118007F2843DDE4
:105570000C20973B93FBF0F200FB123303F1730016
:10558000EBE6FBF77FF82EE4534B1B88182B12D069
:1055900099F800201344A3F118007F2840F3938367
:1055A0000C20973B93FBF0F200FB123303F17300E6
:1055B000C0B204F0FDF84A4A4A4B127833F8123070
:1055C000182B3DF42DAF99F800201344A3F11800D7
:1055D0007F287EF78EAE0C20973B93FBF0F200FB0A
:1055E000123303F17300FEF73EBDFBF74BF865E4A1
:1055F000FBF748F8FFF77EBBFBF744F8ADE63A4B04
:105600001B78002B7DF443AB384B1B78002B3DF40B
:105610003EABB8F800303649013BA8F800300A70BC
:10562000FDF735BB304B1B78002B7DF476AF2F4B4D
:105630001B78002B3DF42BABB8F800302C4901331C
:10564000A8F800300A70FDF722BBDFF87CA099F8BB
:105650000000BAF80030274C3AE71F4A1288182A8F
:1056600012D01344A3F118007F2840F3C1820C200C
:10567000973B93FBF0F200FB123303F17300C0B2CF
:1056800098F8001004F06CF8154B16491A78022AA5
:1056900094BF013200221A701A7831F812001828CB
:1056A0002FD10424022A02F10100C2B288BF0022D5
:1056B00031F81200182823D1013CF3D11A703B684D
:1056C000FEF7FEB8409DFF1FB89EFF1F669EFF1F9E
:1056D000D69CFF1F3C2101000E9FFF1F3D9DFF1F19
:1056E0003E9DFF1FD49EFF1F609FFF1F619FFF1FF6
:1056F000A59CFF1FE0290100BA9CFF1F1423010095
:105700001A703B680344A3F118007F287EF712AE9D
:105710000C20973B93FBF0F200FB123303F1730074
:10572000FEF7ABBDDFF82CB3E2E4BE4B1A88182AB3
:1057300013D03B681344A3F118007F2840F37A820A
:105740000C20973B93FBF0F200FB123303F1730044
:10575000B54BC0B2197804F003F8B44BB4491A78C9
:10576000022A94BF013200221A701A7831F812000E
:1057700018287FF4F7AE0424022A02F1010294BF34
:10578000D2B2002231F8120018287FF4EAAE013CB0
:10579000F2D11A70FDF79DBFA24B1B88182B12D0B7
:1057A00099F800201344A3F118007F2840F3728277
:1057B0000C20973B93FBF0F200FB123303F17300D4
:1057C000C0B203F0F5FF994A994B127833F81230C2
:1057D000182B7FF4F8AEFDF723BE924A1288182AE0
:1057E00012D01344A3F118007F2840F369820C20E3
:1057F000973B93FBF0F200FB123303F17300C0B24E
:1058000098F8001003F0ACFF884B89491A78022AF7
:1058100094BF013200221A701A7831F81200182849
:105820007FF46FAF0424022A02F1010294BFD2B2C6
:10583000002231F8120018287FF462AF013CF2D147
:105840003CE77C4ADFF80CB21288BBF80010033248
:1058500091427FF715ADE9E4764ADFF8F8B1128896
:10586000BBF80010033291427FF7BDAD91E5724C59
:105870002388002B40F0E481DFF8D8B16F4999F814
:1058800000006F4A09881788DFF8B8E1411A0C2236
:1058900091FBF2FC02FB1C114FF0900C0CFB07F784
:1058A00002FB01716FF00B075EF80110014407FB6A
:1058B00003107F2840F3C1817F3890FBF2F302FB95
:1058C00013007330C0B203F073FFBBF800202388CD
:1058D0001344022B21DD594B594A99F800001B88CB
:1058E000B2F800E0574FC31A0C2193FBF1F201FB11
:1058F0001232902303FB0EF301FB02333B445B683F
:1059000018447F2840F3F8817F3890FBF1F301FBC6
:1059100013007330C0B203F04BFFBBF800202388A4
:105920001344032B21DD454B454A99F800001B88A1
:10593000B2F800E0434FC31A0C2193FBF1F201FBD4
:105940001232902303FB0EF301FB02333B449B68AE
:1059500018447F2840F3C1817F3890FBF1F301FBAD
:1059600013007330C0B203F023FFBBF8002023887C
:105970001344042B7EF79DA92E4B1B88012B7EF42C
:1059800098A999F80020A2F10C007F287FF7C7A8FA
:105990008B3A0C2092FBF0F300FB13207330FFF7DF
:1059A000B0B8294B00227F2107201A8003F0B0FEF7
:1059B0007F210B2003F0ACFEFDF7E2BD234B01225B
:1059C0007F2107201A8003F0A3FE7F210B2003F024
:1059D0009FFEFDF7CDBD1E4B04227F2107201A80BC
:1059E00003F096FE00210B2003F092FEFDF7B9BDF7
:1059F000174B02227F2107201A8003F089FE7F21A6
:105A00000B2003F085FEFDF7A7BD114B00210720F9
:105A10001C8003F07DFE7F210B2003F079FEFDF753
:105A200096BD00BFCE9CFF1F3D9DFF1F3E9DFF1FEB
:105A3000489EFF1FD69CFF1F409DFF1FB89EFF1F63
:105A4000669EFF1F14230100A29CFF1F529DFF1F93
:105A5000B09EFF1FBA9CFF1FAF4B1A88182A13D0A5
:105A60003B681344A3F118007F2840F33F810C20CA
:105A7000973B93FBF0F200FB123303F17300A74B4B
:105A8000C0B2197803F06CFEA54BA6491A78022A19
:105A900094BF013200221A701A7831F812001828C7
:105AA0007FF460AD0424022A02F1010294BFD2B255
:105AB000002231F8120018287FF453AD013CF2D1D6
:105AC0001A70FDF706BEFAF7DDFDFFF734BBFAF7F3
:105AD000D9FD85E4904A1288182A12D01344A3F104
:105AE00018007F2840F3F6800C20973B93FBF0F2E0
:105AF00000FB123303F17300C0B298F8001003F0FA
:105B00002FFE874B87491A78022A94BF0132002260
:105B10001A701A7831F8120018287FF4F2AD0424B4
:105B2000022A02F1010294BFD2B2002231F812001F
:105B300018287FF4E5AD013CF2D1BFE5FAF7A2FDEC
:105B4000FFF799BB744B1B88182B12D099F80020D3
:105B50001344A3F118007F2840F3C5800C20973B25
:105B600093FBF0F200FB123303F17300C0B203F0B9
:105B70001FFE6B4A6B4B127833F81230182B7FF4F0
:105B800022ADFDF74DBC684B1B88182B12D099F83D
:105B900000201344A3F118007F2840F3B0800C20AC
:105BA000973B93FBF0F200FB123303F17300C0B29A
:105BB00003F0FEFD5A4A5D4B127833F81230182B71
:105BC0003EF477A899F800201344A3F118007F2829
:105BD0007EF7A5AF0C20973B93FBF0F200FB12334E
:105BE00003F17300FEF78DBFFAF74CFDFFF7F7BA2C
:105BF000FAF748FD43E5484B1B88182B11D099F85C
:105C000000201344A3F118007F2872DD0C20973B7D
:105C100093FBF0F200FB123303F17300C0B203F008
:105C2000C7FD3F4A3F4B127833F81230182BC9D1C9
:105C3000FEF73FB8FAF726FD8AE5FAF723FD41E6BD
:105C40003B4ADFF800B11288BBF8001003329142E2
:105C50007FF73BAE12E6374B1B88182B11D099F813
:105C600000201344A3F118007F2839DD0C20973B56
:105C700093FBF0F200FB123303F17300C0B203F0A8
:105C800097FD274A2C4B127833F81230182B99D1F4
:105C9000FEF70FB8FAF7F6FC92E5FAF7F3FC3EE4EC
:105CA000FAF7F0FCFFF711BBFAF7ECFCFFF7C1BB0A
:105CB000FAF7E8FCFFF733BBFAF7E4FCFFF7E2BBC7
:105CC000FAF7E0FC9BE5FAF7DDFC71E4FAF7DAFCA1
:105CD000FFF75BBAFAF7D6FC0EE7FAF7D3FC41E61A
:105CE000FAF7D0FCCAE7FAF7CDFC3FE7FAF7CAFCAF
:105CF000C5E6FAF7C7FC91E7FAF7C4FC0AE6FAF73B
:105D0000C1FC54E70D4B03930D4B0293FDF7A4BE6A
:105D100023601946FDF7D8BBD09CFF1F3D9DFF1F98
:105D20003E9DFF1F509EFF1F0E9FFF1FD49EFF1F13
:105D3000D69CFF1FCE9CFF1F489EFF1F009DFF1F8C
:105D4000629DFF1FBA9CFF1F38B507F0CDFC0E48BF
:105D500005F004FC0D4805F001FC0D4805F0FEFBC4
:105D600000234FF07E5201210A48FAF77FFB0A4BCD
:105D70000A4A0B49802400251C7118461D60BDE8A5
:105D800038400BF073B900BFB89CFF1FEC9CFF1F9D
:105D9000589DFF1F8C9EFF1F1C9FFF1F1C89FF1F0C
:105DA0002906000010B50446A4206368198803F092
:105DB00033FEE368A6201988BDE8104003F02CBE2E
:105DC00043682A20198803F027BE00BF10B5044697
:105DD00022206368198803F01FFEE36824201988D5
:105DE000BDE8104003F018BE10B504460A206368F1
:105DF000198803F011FEE3680C201988BDE81040F3
:105E000003F00ABE10B5044606206368198803F043
:105E100003FEE36808201988BDE8104003F0FCBDCC
:105E200010B5044602206368198803F0F5FDE368A5
:105E300004201988BDE8104003F0EEBD70B50E4C8B
:105E400084B01225042201230646039002932046C3
:105E50008DE824001423102106F084FD0622092376
:105E6000029303960195204600921423102106F018
:105E700079FD04B070BD00BF909FFF1FF8B5B04C16
:105E8000B4F90030032B00F01281002B6AD0022BF2
:105E900000F08A80052B00F0B580012B00F0DD803A
:105EA000042B00D0F8BDA74FA74E00254FF4AF74C8
:105EB000E9B2A64805F0BAFB57F8043BC3F5967360
:105EC00000FB03F086FB0023C017C0EB6310844285
:105ED00005F10105A8BF0446062DE9D19C4F9A4E55
:105EE0000025E9B29B4805F0A1FB57F8043BC3F538
:105EF000967300FB03F086FB0023C017C0EB631012
:105F0000844205F10105A8BF04460C2DE9D1924F4A
:105F10008D4E0025E9B2914805F088FB57F8043B07
:105F2000894AC3F5967300FB03F086FB0013C01784
:105F3000C0EB6310844205F10105A8BF04460C2D97
:105F4000E8D1A4F11401312900F3A38040F26C726E
:105F500032218348834B01801A602A20BDE8F84033
:105F600003F05ABD0E2007F023FB40F6FF71C83046
:105F70008842A8BF084620EAE07000F5FA6283B2C2
:105F80008A42794D794EA8BF0A46022019463380CD
:105F90002A8003F041FD2988042003F03DFDB4F977
:105FA0000030022B7FF476AF012008F045FA054659
:105FB000002008F041FAA842B8BF284600F1C80105
:105FC000B1F5FA7FC0F2B480B1F57A6FA8BF4FF493
:105FD0007A6101F54873B3F57A6FA8BF4FF47A631D
:105FE0009BB289B2624A634D11800A202B8003F074
:105FF00013FD29880C2003F00FFDB4F90030052BA8
:106000007FF44BAF0F2008F017FAC0F53F6304335D
:10601000B3F5AF6FC0F28980B3F5FA6FA8BF4FF444
:10602000FA6399B2544BC0F54360B0F5AF6F198075
:1060300061DBB0F5FA6FA8BF4FF4FA6083B24F4D41
:10604000A4202B8003F0E8FC2988A62003F0E4FCC0
:10605000B4F90030012B7FF423AF152007F0A8FA24
:1060600000F59671B1F52F7F4DDB41F25C2399422B
:1060700063DC434A00F5617089B2B0F52F7F11806F
:10608000B8BF4FF42F7344DB8342A8BF03469BB2D3
:106090003FE040F23A73A4F5B97403FB04F482FBC9
:1060A0000432E417A4EB621289B2323251E71020B5
:1060B00008F0C2F9C830B0F5FA7F1FDBB0F57A6F8F
:1060C0000146A8BF4FF47A6101F51673B3F57A6FF4
:1060D000A8BF4FF47A639BB289B22A4A2A4D118035
:1060E00022202B8003F098FC2988242003F094FCC4
:1060F000B4F90030C9E64FF4AF63A0E740F24C4377
:106100004FF4FA71E9E740F214534FF42F711C4A2F
:1061100011801E4D06202B8003F07EFC298808206C
:1061200003F07AFCB4F90030BAE64FF4AF6179E7D6
:1061300040F214534FF4FA7154E71946E7E700BFF1
:106140006E9FFF1F488AFF1FB5814E1BB89CFF1F23
:10615000188AFF1FEC9CFF1F2C89FF1F589DFF1FF3
:10616000269FFF1F048AFF1F2C9FFF1F609DFF1F9C
:10617000C49EFF1FCC9CFF1F649DFF1FE49EFF1F5A
:106180000A9DFF1F749EFF1F709EFF1FF89EFF1F3A
:106190002DE9F041224D82B0012602B284B2009274
:1061A000284601967823192106F022FB04F10C02FF
:1061B00012B28DE844002846A7197823192104F16A
:1061C000020806F015FB3FB20FFA88F819233A4689
:1061D000284619460196CDF8008006F009FB782381
:1061E0003A4628461946CDF80080019604F10A0780
:1061F0000B3406F0FDFA3FB224B278233A46284623
:1062000019468DE8500006F0F3FA192300943A4637
:1062100001962846194606F0EBFA02B0BDE8F08177
:10622000909FFF1F30B583B000230C4605B200934A
:1062300026225B231C210C4806F02AF8294601235C
:106240002622094805F034FB002C24B205DB214648
:1062500001232622044805F02BFB044A044B158039
:106260001C8003B030BD00BF909FFF1F628AFF1FDC
:10627000648AFF1F2DE9F041B44C237882B01BB132
:10628000B34B4FF6FF721A80B24BB3F90030CBB963
:10629000B14AAF4B1068B3F9002080F30C005B23C8
:1062A00003FB00F000131C30824244D04FF0FF315A
:1062B000FFF7B8FFA94806F04FF80023237002B09B
:1062C000BDE8F081012B1BD0022B53D0032B38D01B
:1062D000042B00F08C80052BEFD10F2008F0ACF8D8
:1062E000C0F53B600830B0F5AF6F41DBB0F5FA6F39
:1062F000A8BF4FF4FA60A0F5AF625B2398482EE088
:10630000984B1A68B2F52F7F32DB41F25C2393423F
:10631000A8BF1346A3F52F735B22934802FB03F338
:1063200080FB0320DB17C3EBA0201C30884BB3F9A4
:1063300000308342BAD18D4BB3F900300133B5D16F
:10634000BBE78B4B1B68B3F5FA7F11DBB3F57A6FB4
:10635000A8BF4FF47A638748A3F5FA725B2303FB67
:1063600002F380FB0320DB17C3EB20201C30DDE7AA
:106370001C20DBE7804B1B68B3F5FA7F33DBB3F5FA
:106380007A6FA8BF4FF47A63A3F5FA7279485B235A
:1063900003FB02F380FB0320DB17C3EB20201C3040
:1063A000764B1B68B3F5FA7F1FDBB3F57A6FA8BF96
:1063B0004FF47A63A3F5FA726E495B2303FB02F391
:1063C00081FB0321DB17C3EB21211C31604BB3F9A7
:1063D000003083427FF46CAF644BB3F900308B42E2
:1063E0007FF466AF69E71C20DAE71C21EEE725227F
:1063F00000258DE8240076231C215848604E614F0B
:10640000DFF8988106F0F4F916E0B0F5AF7FA8BF89
:106410004FF4AF70323802FB00F088FB0031C01738
:10642000C0EB61111C3109B201231D4425224B48E8
:1064300005F03EFA0C2D14D0E9B2534805F0F6F8F9
:1064400056F8043BC3F5967300FB03F087FB00137B
:10645000C017C0EB631031284FF05B02D5DC1C2164
:10646000E2E7262200258DE8240076231C213B4804
:10647000464E444FDFF8248106F0BAF916E0B0F535
:10648000AF7FA8BF4FF4AF70323802FB00F088FB3B
:106490000031C017C0EB61111C3109B201231D444A
:1064A00026222E4805F004FA0C2D14D0E9B2384803
:1064B00005F0BCF856F8043BC3F5967300FB03F0F7
:1064C00087FB0013C017C0EB631031284FF05B024D
:1064D000D5DC1C21E2E7272200258DE82400762365
:1064E0001C211E482B4E274FDFF8B08006F080F9A4
:1064F00017E0B0F5AF7FA8BF4FF4AF70323802FBA2
:1065000000F088FB0031C017C0EB61111C3109B2EB
:1065100001231D442722114805F0CAF9062D3FF436
:10652000C9AEE9B21C4805F081F856F8043BC3F542
:10653000967300FB03F087FB0013C017C0EB6310DA
:1065400031284FF05B02D4DC1C21E1E7689FFF1F7C
:10655000628AFF1F6E9FFF1FC89EFF1F909FFF1F35
:1065600037800B6D909CFF1FD3058541648AFF1F08
:10657000DC9CFF1F011FB812E89CFF1FAC9CFF1F93
:10658000188AFF1FB5814E1BEC9CFF1F2C89FF1F33
:10659000589DFF1F488AFF1FB89CFF1F4B48371BA1
:1065A0002DE9F041044682B056482768E56805F0B9
:1065B000C7FD1120FFF7ECFD012619234FF0280835
:1065C000194624224F480196CDF8008006F010F9B4
:1065D0007823194624224B480196CDF8008006F016
:1065E00007F93146474806F099FC0222192145482F
:1065F00006F090FC38460BF003FB39460246414852
:1066000006F022FE3F4806F035FE142200213D48E8
:1066100006F080FC03223C493A4806F015FE394852
:1066200006F028FE23220021364806F073FC0322E0
:106630003649344806F008FE324806F01BFE7DB1AC
:106640002F20FFF7A5FD322200212E4806F062FC24
:1066500003222F492B4806F0F7FD2A4806F00AFED0
:1066600001232C4A18461370FFF7E8FB2189638940
:1066700062685B1A5C2B128832DD521A02EB42020E
:10668000C2EB4212013392FBF3F31B33224A1D4843
:10669000138001261A221BB28DE8440019461422E9
:1066A00006F0A6F8CDB1218A638AE2685B1A5C2BFA
:1066B00012881DDC511A5C2202FB01F292FBF3F3FB
:1066C0001B33164A0F481380012438221BB28DE871
:1066D00014001946322206F08BF802B0BDE8F081B2
:1066E000511A5C2202FB01F292FBF3F31B33CDE75C
:1066F000521A02EB4202C2EB4212334492FBF3F312
:106700001B33DEE7909FFF1F482B01004C2B01003D
:10671000502B01000DA0FF1F6A9FFF1F6C9FFF1FE2
:106720002DE9F0411E4682B014461AB3052A0546EB
:1067300000F09C80099B6F4A00EBC305012C6F8918
:1067400029896868A7EB010382FB03E21A444FEA38
:10675000E373C3EBA213028829D0042C69D0664AE4
:10676000022CB2F9001060D0082C65D0012002B0D4
:10677000BDE8F081614D624A2B681268CB1A9342E2
:106780000F466FD95F4A338811785F48012918BFD7
:1067900001241470089A06321BB212B28DE814005C
:1067A0001946BDF9202006F023F82F60DEE79BB2E2
:1067B000D31A994203DC9F423946A8BF1946089A6A
:1067C0000180B6F90030BDF920804F48971D4FF089
:1067D000000E3FB2194642460097CDF804E006F09D
:1067E00007F829896A896B68521A1B885C2AA3EB0F
:1067F000010377DD03EB43030132C3EB431393FB48
:10680000F2F303F11B0213B2012032801946424613
:10681000019000973C4805F0EBFF3A4B00221A70BC
:10682000354A022CB2F900109ED14B1C1BB21380CA
:1068300004E012FA83F3BCE700231380994295D059
:10684000089AB6F9003030480632012412B200929C
:1068500019460194BDF9202005F0CAFF204602B078
:10686000BDE8F081204602B0BDE8F0810724002693
:106870005A2323228DE850001A21234805F086FF71
:106880000121214806F04AFB01211F4806F04CFB7C
:10689000232235211C4806F03DFB22461B491A489D
:1068A00006F0D2FC184806F0E5FC174805F054FD48
:1068B0004FF4FA6007F0CEFBFFF7E0FA5A232322E9
:1068C0001A218DE85000104805F060FF0E4805F0D1
:1068D00043FD2846FFF764FE0D4B01221A70FFF7B7
:1068E000C9FC43E75C2101FB03F393FBF2F21B328B
:1068F00089E700BFC94216B2729FFF1FF89FFF1FB2
:10690000143B01000DA0FF1F909FFF1F542B01009F
:10691000689FFF1F2DE9F04F5A4E5B4DB6F900708E
:106920004C7855F8277085B08146984604B10C78AC
:10693000DFF874A11AB99AF80030002B39D0534D02
:10694000002338462B808AF80030FFF729FE504A92
:10695000504BB5F90000012111704FF6FF721A80FB
:1069600060B301285ED001203223224601900093BB
:106970004946494B3846FFF7D3FE00240346B5F994
:106980000020022A39DD00222A80B6F900203D4984
:10699000002A3BDB052AC4BF00220A80B8F1000FA1
:1069A00039D1002C0CBF18464FF0FF3005B0BDE8C0
:1069B000F08F364DB5F900000028D2D1DFF8ECB0E9
:1069C000364ADBF800301268C3EB0903934227D93B
:1069D000334B1A78012A18BF01201870FFF72EFADE
:1069E0000123CBF80090012C2AD0042C35D0022CA6
:1069F0003AD0082C3ED00024C1E7C6D1FA68002A5C
:106A0000C1D0B6F900201F49002AC3DA05220A8046
:106A1000B8F1000FC5D00393FFF72CFC039BC0E730
:106A20000346E0E74FF0000E142322468DE80840AD
:106A300049461C4B38467446FFF772FE03469EE7F4
:106A400032888AF80040013232807A6982B10024AB
:106A5000384603939047039B91E732880121013A1E
:106A600032808AF80010F0E701222A8000248CE7A7
:106A7000144684E77A69002129804FF0FF34002A08
:106A8000E6D182E76E9FFF1F688AFF1F729FFF1F7C
:106A9000689FFF1F628AFF1F6C9FFF1F143B01004E
:106AA0000DA0FF1F6A9FFF1F709FFF1FF89FFF1F12
:106AB00001210D2007F092BA00210D2007F08EBAB7
:106AC00001460D2007F08ABA08B50D2007F08CFAB0
:106AD000B0FA80F149090D20BDE8084007F07EBA00
:106AE00010B5002144080D2007F078FA204607F081
:106AF000B1FA0D20012107F071FA2046BDE81040DF
:106B000007F0A8BA2D4A2E4B10881B68984210B582
:106B100049DA2C4A1288141A9A42A8BF1A46B4F5C8
:106B2000157F36DA121A40F2532303FB02F393FB6C
:106B3000F4F105310A2007F0C1F8234B1978C9B3E5
:106B4000224B23491B6840F2271283F3070302FB01
:106B500003F381FB03211944DB17C3EBA1110531BA
:106B6000092007F0ABF81B4B1968F1B181F307015D
:106B700040F22712164802FB01F380FB032119445F
:106B8000DB17C3EBA11105311620BDE8104007F05B
:106B900095B8131A4FF41572611C02FB03F393FBB3
:106BA000F1F10531C6E70021C4E71620BDE8104029
:106BB00007F084B8092007F081F8D4E7609DFF1F33
:106BC000889CFF1F2C9FFF1F0E9DFF1F149FFF1F00
:106BD00009040281E09EFF1F7F2838B5A8BF7F20EF
:106BE0000F4C4FF4167202FB00F284FB0231114489
:106BF000D2170546C2EBA1110A2007F05FF87F3DCE
:106C00004FF4967303FB05F384FB03211944DB1750
:106C1000A3EBA1110920BDE8384007F04FB800BF31
:106C200009040281C368B3F9003030B583EAE37424
:106C3000A4EBE374002BA0B218DB012300E01346A1
:106C400003EB830252009442F9DA0A4D90FBF3F20F
:106C500085FB03E403FB1200DB173032D3EBA40304
:106C600080B201F8012BF1D10B7030BD2D230B70D8
:106C70000131E2E76766666638B5094D8224204631
:106C800002F0E4FE35F8021B00B28842204601D033
:106C900002F0C2FE0234A4B28A2CF0D138BD00BF8B
:106CA000509EFF1F024B8020198802F0B5BE00BF26
:106CB000D09CFF1F38B5094D7824204602F0C6FE4F
:106CC00035F8021B00B28842204601D002F0A4FE33
:106CD0000234A4B2802CF0D138BD00BF489EFF1F03
:106CE000024B7620198802F097BE00BFCE9CFF1F92
:106CF00038B5094D4624204602F0A8FE35F8021B9F
:106D000000B28842204601D002F086FE0234A4B2CE
:106D10004E2CF0D138BD00BFD49EFF1F024B442043
:106D2000198802F079BE00BF0E9FFF1F024B4E2054
:106D3000198802F071BE00BFE29CFF1F024B9A202F
:106D4000198802F069BE00BF409DFF1F024B9820CA
:106D5000198802F061BE00BFD69CFF1F024B8C2039
:106D6000198802F059BE00BF669EFF1F024B9C208F
:106D7000198802F051BE00BFBA9CFF1F024BA02031
:106D8000198802F049BE00BFDC9EFF1F024B96200F
:106D9000198802F041BE00BFB89EFF1F024B8A2037
:106DA000198802F039BE00BF7E9EFF1F08B5034B55
:106DB0001020198802F030FE012008BD7C9EFF1FC4
:106DC000024B1020198802F027BE00BF7C9EFF1FD7
:106DD000024B2C20198802F01FBE00BFB69CFF1F7B
:106DE000024B1E20198802F017BE00BFD49CFF1F63
:106DF000C3680E20198802F00FBE00BF024B282086
:106E0000198802F009BE00BFD29EFF1F024B64200A
:106E1000198802F001BE00BFCC9EFF1F024B5A2012
:106E2000198802F0F9BD00BF989CFF1F024B162085
:106E3000198802F0F1BD00BFA29CFF1F024B2E205B
:106E4000198802F0E9BD00BF489DFF1F024B3020AA
:106E5000198802F0E1BD00BF3C9FFF1F024B9E203E
:106E6000198802F0D9BD00BFC089FF1F024BAC20BA
:106E7000198802F0D1BD00BFCE9EFF1F024BAE208D
:106E8000198802F0C9BD00BFE09CFF1F024BB02073
:106E9000198802F0C1BD00BF5C9EFF1F024BB220EB
:106EA000198802F0B9BD00BFFE9CFF1F024B1820DD
:106EB000198802F0B1BD00BF669DFF1F024BA220E2
:106EC000198802F0A9BD00BF029FFF1F024B1A20C4
:106ED000198802F0A1BD00BFEE9CFF1F024B1C20D1
:106EE000198802F099BD00BFE49CFF1F024B662089
:106EF000198802F091BD00BF0C9FFF1F024B72204A
:106F0000198802F089BD00BF389FFF1F024B202067
:106F1000198802F081BD00BF0A9FFF1F024B32207B
:106F2000198802F079BD00BFFA9EFF1F024B68204E
:106F3000198802F071BD00BF2C9DFF1F024B6C2011
:106F4000198802F069BD00BF8C9CFF1F024B6E20A8
:106F5000198802F061BD00BF669FFF1F024B5220DF
:106F6000198802F059BD00BF5E89FF1F024B5020F7
:106F7000198802F051BD00BF2089FF1F024B542029
:106F8000198802F049BD00BF148AFF1F024B5C2024
:106F9000198802F041BD00BF608AFF1F024B5E20CE
:106FA000198802F039BD00BF5C89FF1F024B5620D3
:106FB000198802F031BD00BF3A9DFF1F244B1B888A
:106FC0000B2B43D8DFE803F00B10151A1F24292ED2
:106FD00033383D06084604221E490AF0CFBE084653
:106FE00004221D490AF0CABE084604221B490AF0C1
:106FF000C5BE084604221A490AF0C0BE084604224B
:1070000018490AF0BBBE0846042217490AF0B6BE6A
:107010000846042215490AF0B1BE08460422144964
:107020000AF0ACBE0846042212490AF0A7BE084680
:10703000042211490AF0A2BE084604220F490AF0B0
:107040009DBE084604220E490AF098BE704700BF54
:10705000B89EFF1FC83701001C35010088330100AE
:10706000B83401008C330100D438010090330100A2
:10707000943301006036010098330100D4370100D9
:107080009C330100064B074A10B41C88064B084687
:10709000002C14BF11461946042210BC0AF06EBE23
:1070A000089DFF1FA0330100A4330100064B074ACF
:1070B00010B41C88064B0846002C14BF1146194614
:1070C000042210BC0AF05ABE4A9DFF1FA0330100E3
:1070D000A4330100064B074A10B41C88064B08462F
:1070E000002C14BF11461946042210BC0AF046BEFB
:1070F0006E9EFF1FA0330100A4330100064B074A18
:1071000010B41C88064B0846002C14BF11461946C3
:10711000042210BC0AF032BEBA9EFF1FA033010049
:10712000A4330100064B074A10B41C88064B0846DE
:10713000002C14BF11461946042210BC0AF01EBED2
:10714000529DFF1FA0330100A43301001B4B1B887D
:107150000A2B0AD8DFE803F00A0E12161A1E22269E
:107160002A2E0600164B186808607047154B1868E1
:1071700008607047144B186808607047134B186814
:1071800008607047124B186808607047114B186808
:1071900008607047104B1868086070470F4B1868FC
:1071A000086070470E4B1868086070470D4B1868F0
:1071B000086070470C4B1868086070477E9EFF1F80
:1071C000CC330100A4330100A8330100AC3301002B
:1071D000B0330100B4330100B8330100BC33010007
:1071E000C0330100C4330100C8330100F0B52B4E99
:1071F0002B4FDFF8C4E005460FCE87B06C460FC4B6
:1072000096E803003B68274A274F44F8040B40F6F2
:10721000CC308342C8BF3A46BEF800602180012EC0
:1072200011889278ADF80D108DF80F202AD032D346
:1072300040F6CA02022E18BF00229A4226DAA3F6AE
:1072400098031A491A4AC3EB031381FB030119443B
:10725000DB17C3EB6123243382FB0321DA17C2EB74
:10726000A10202EB8201A3EB4103303330328DF8EF
:1072700013308DF811206946284616220AF07EFD4B
:1072800007B0F0BD40F698029A42D8DB094B186867
:10729000CDF81100EFE740F6FC02CEE7E033010045
:1072A000C09EFF1FD4330100D03301003B773B98D1
:1072B00067666666D8330100589EFF1FF8B5174C05
:1072C000174E2278174D33782F888E46003218BF1C
:1072D000012201467046FFF71DFB002398423370E0
:1072E000237015DB14BF012000202B889F420ED095
:1072F00040F23A72A3F5AF730B490C4C02FB03F357
:1073000081FB0312DB17A3EB621332332360F8BD5A
:107310000749012218460A702270E6E7108BFF1F0A
:10732000819FFF1F269FFF1FB5814E1B048AFF1FF1
:107330000CA0FF1F014B187802F006BBF49FFF1F43
:10734000014B187802F01ABB2491FF1F134BB3F9BD
:10735000003030B583EAE374A4EBE374002BA0B2F1
:1073600018DB012300E0134603EB83025200944232
:10737000F9DA0B4D90FBF3F285FB03E403FB1200FB
:10738000DB173032D3EBA40380B201F8012BF1D12B
:107390000B7030BD2D230B700131E2E72491FF1FEC
:1073A00067666666144BB3F9003070B583EAE3751F
:1073B000A5EBE375002BACB21ADB012300E003461A
:1073C00003EB830040008542F9DA0C4E94FBF3F0A6
:1073D00086FB03E503FB1044DB173030D3EBA5033A
:1073E000A4B201F8010BF1D105480B70106070BD1B
:1073F0002D230B700131E0E7989CFF1F67666666DE
:10740000F8330100134BB3F9003030B583EAE3746D
:10741000A4EBE374002BA0B218DB012300E01346B9
:1074200003EB830252009442F9DA0B4D90FBF3F226
:1074300085FB03E403FB1200DB173032D3EBA4031C
:1074400080B201F8012BF1D10B7030BD2D230B70F0
:107450000131E2E7C089FF1F67666666134BB3F927
:10746000003030B583EAE374A4EBE374002BA0B2E0
:1074700018DB012300E0134603EB83025200944221
:10748000F9DA0B4D90FBF3F285FB03E403FB1200EA
:10749000DB173032D3EBA40380B201F8012BF1D11A
:1074A0000B7030BD2D230B700131E2E7E09CFF1F14
:1074B00067666666134BB3F9003030B583EAE37450
:1074C000A4EBE374002BA0B218DB012300E0134609
:1074D00003EB830252009442F9DA0B4D90FBF3F276
:1074E00085FB03E403FB1200DB173032D3EBA4036C
:1074F00080B201F8012BF1D10B7030BD2D230B7040
:107500000131E2E7FE9CFF1F67666666134BB3F925
:10751000003030B583EAE374A4EBE374002BA0B22F
:1075200018DB012300E0134603EB83025200944270
:10753000F9DA0B4D90FBF3F285FB03E403FB120039
:10754000DB173032D3EBA40380B201F8012BF1D169
:107550000B7030BD2D230B700131E2E7029FFF1F3E
:1075600067666666134BB3F9003030B583EAE3749F
:10757000A4EBE374002BA0B218DB012300E0134658
:1075800003EB830252009442F9DA0B4D90FBF3F2C5
:1075900085FB03E403FB1200DB173032D3EBA403BB
:1075A00080B201F8012BF1D10B7030BD2D230B708F
:1075B0000131E2E75E89FF1F67666666134BB3F928
:1075C000003030B583EAE374A4EBE374002BA0B27F
:1075D00018DB012300E0134603EB830252009442C0
:1075E000F9DA0B4D90FBF3F285FB03E403FB120089
:1075F000DB173032D3EBA40380B201F8012BF1D1B9
:107600000B7030BD2D230B700131E2E72089FF1F85
:1076100067666666134BB3F9003030B583EAE374EE
:10762000A4EBE374002BA0B218DB012300E01346A7
:1076300003EB830252009442F9DA0B4D90FBF3F214
:1076400085FB03E403FB1200DB173032D3EBA4030A
:1076500080B201F8012BF1D10B7030BD2D230B70DE
:107660000131E2E7148AFF1F67666666134BB3F9C0
:10767000003030B583EAE374A4EBE374002BA0B2CE
:1076800018DB012300E0134603EB8302520094420F
:10769000F9DA0B4D90FBF3F285FB03E403FB1200D8
:1076A000DB173032D3EBA40380B201F8012BF1D108
:1076B0000B7030BD2D230B700131E2E7608AFF1F94
:1076C00067666666134BB3F9003030B583EAE3743E
:1076D000A4EBE374002BA0B218DB012300E01346F7
:1076E00003EB830252009442F9DA0B4D90FBF3F264
:1076F00085FB03E403FB1200DB173032D3EBA4035A
:1077000080B201F8012BF1D10B7030BD2D230B702D
:107710000131E2E75C89FF1F6766666608B5702085
:1077200002F094F9044B1988884204D07020BDE817
:10773000084002F071B908BD589EFF1F08B57420BB
:1077400002F084F9044B1988884204D07420BDE803
:10775000084002F061B908BDF09EFF1F054B1B8871
:107760000846042213B904490AF008BB03490AF089
:1077700005BB00BFE29CFF1F00340100FC33010089
:107780000E4B1B88032B17D8DFE803F0110C070200
:10779000084604220A490AF0F1BA084604220949B7
:1077A0000AF0ECBA0846042207490AF0E7BA08468C
:1077B000042206490AF0E2BA704700BF669EFF1F26
:1077C000103401000C3401000834010004340100BD
:1077D00010B40A4B0A4C0A4693E8030083B023888E
:1077E00002AC04E9030004EB8303104653F8081CC1
:1077F000052203B010BC0AF0C1BA00BFEC2B010097
:10780000CC9EFF1F30B40A4B0A4D0C4693E807008C
:1078100084B02B8804AD05E9070005EB83032046FF
:1078200053F80C1C042204B030BC0AF0A7BA00BF05
:10783000F42B0100589EFF1FF0B40C4D0C4F0E4668
:107840000FCD8CB001AC0FC40FCD0FC495E807006D
:107850003B8884E807000CAA02EB8303304653F808
:107860002C1C04220CB0F0BC0AF088BA002C0100D9
:10787000B09EFF1F30B50A4B0A4D0C460FCB85B0AA
:107880000DF1100E0EE90F002B880EEB830320463E
:1078900053F8101C042205B0BDE830400AF06EBA5F
:1078A0003C2C0100CE9EFF1F30B50A4B0A4D0C4602
:1078B0000FCB85B00DF1100E0EE90F002B880EEBEB
:1078C0008303204653F8101C042205B0BDE8304065
:1078D0000AF054BA3C2C01005C9EFF1FF0B40B4D23
:1078E0000B4F0E460FCD86B06C460FC495E80300D3
:1078F0003B8884E8030006AA02EB8303304653F872
:10790000181C042206B0F0BC0AF038BA4C2C010056
:10791000669DFF1FF0B40A4D0A4F0E460FCD86B08C
:1079200001AC0FC42A683B88226006AA02EB8303DD
:10793000304653F8141C0C2206B0F0BC0AF01EBAF4
:10794000642C0100E49CFF1FF0B40B4D0B4F0E465E
:107950000FCD86B06C460FC495E803003B8884E8E1
:10796000030006AA02EB8303304653F8181C0422D6
:1079700006B0F0BC0AF002BA782C0100F09EFF1F9E
:10798000164B1B880BB31BB283EAE370A0EBE370CA
:10799000002B30B584B21DDB012300E0134603EB5E
:1079A000830252009042F9DA0D4894FBF3F280FB17
:1079B00003E503FB1244DB173032D3EBA503A4B27B
:1079C00001F8012BF1D10B7030BD084604220549A6
:1079D0000AF0D4B92D230B700131DDE72C9DFF1F78
:1079E0006766666614340100F0B40A4D0A4F0E460D
:1079F0000FCD86B001AC0FC42A683B88226006AA6E
:107A000002EB8303304653F8141C042206B0F0BC8A
:107A10000AF0B4B9902C01008C9CFF1F054B1B8809
:107A20001BB9054B186808607047084604220349D3
:107A30000AF0A4B9409DFF1FA4330100A033010048
:107A4000164B1B880BB31BB230B583EAE374A4EB6F
:107A5000E374002BA0B21CDB012300E0134603EB10
:107A6000830252009442F9DA0D4D90FBF3F285FB4C
:107A700003E403FB1200DB173032D3EBA40380B224
:107A800001F8012BF1D10B7030BD064B186808606E
:107A900070472D230B700131DEE700BFD49CFF1F20
:107AA00067666666A4330100164B1B880BB31BB2D6
:107AB00030B583EAE374A4EBE374002BA0B21CDBC3
:107AC000012300E0134603EB830252009442F9DAEB
:107AD0000D4D90FBF3F285FB03E403FB1200DB1773
:107AE0003032D3EBA40380B201F8012BF1D10B703B
:107AF00030BD064B1868086070472D230B700131AC
:107B0000DEE700BFBE9EFF1F67666666A433010006
:107B1000164B1B880BB31BB230B583EAE374A4EB9E
:107B2000E374002BA0B21CDB012300E0134603EB3F
:107B3000830252009442F9DA0D4D90FBF3F285FB7B
:107B400003E403FB1200DB173032D3EBA40380B253
:107B500001F8012BF1D10B7030BD064B186808609D
:107B600070472D230B700131DEE700BFA29CFF1F81
:107B70006766666618340100174B1B881BB31BB27F
:107B800070B583EAE375A5EBE375002BACB21EDBA1
:107B9000012300E0034603EB830040008542F9DA4D
:107BA0000E4E94FBF3F086FB03E503FB1044DB175A
:107BB0003030D3EBA503A4B201F8010BF1D1084892
:107BC0000B70106070BD074B1868086070472D235C
:107BD0000B700131DCE700BF489DFF1F67666666DA
:107BE0001C340100A4330100164B1B880BB31BB2DD
:107BF00030B583EAE374A4EBE374002BA0B21CDB82
:107C0000012300E0134603EB830252009442F9DAA9
:107C10000D4D90FBF3F285FB03E403FB1200DB1731
:107C20003032D3EBA40380B201F8012BF1D10B70F9
:107C300030BD064B1868086070472D230B7001316A
:107C4000DEE700BF3C9FFF1F67666666A433010046
:107C5000164B1B880BB31BB230B583EAE374A4EB5D
:107C6000E374002BA0B21CDB012300E0134603EBFE
:107C7000830252009442F9DA0D4D90FBF3F285FB3A
:107C800003E403FB1200DB173032D3EBA40380B212
:107C900001F8012BF1D10B7030BD064B186808605C
:107CA00070472D230B700131DEE700BF0C9FFF1FD3
:107CB00067666666A4330100164B1B880BB31BB2C4
:107CC00030B583EAE374A4EBE374002BA0B21CDBB1
:107CD000012300E0134603EB830252009442F9DAD9
:107CE0000D4D90FBF3F285FB03E403FB1200DB1761
:107CF0003032D3EBA40380B201F8012BF1D10B7029
:107D000030BD064B1868086070472D230B70013199
:107D1000DEE700BF389FFF1F67666666A433010079
:107D2000174B1B881BB31BB270B583EAE375A5EB39
:107D3000E375002BACB21EDB012300E0034603EB2E
:107D4000830040008542F9DA0E4E94FBF3F086FB87
:107D500003E503FB1044DB173030D3EBA503A4B2DB
:107D600001F8010BF1D108480B70106070BD074B92
:107D70001868086070472D230B700131DCE700BFE5
:107D80000A9FFF1F676666661C340100A43301006A
:107D9000054B1B881BB1054B186808607047044BE6
:107DA00018680860704700BF3A9DFF1F303401001B
:107DB0002C340100184B1A8852B3184A128830B577
:107DC0000A80B3F90030002B83EAE374A4EBE37478
:107DD000BCBF2D238B70A0B2ACBF02310331012395
:107DE00000E0134603EB830252009442F9DA0C4D93
:107DF00090FBF3F285FB03E403FB1200DB17303248
:107E0000D3EBA40380B201F8012BF1D10B7030BD8C
:107E1000044B186808607047EE9CFF1F3434010063
:107E200067666666A433010070B53C4D2B78064644
:107E3000002B35D11C4673780BB9204670BDFAF77C
:107E4000FFF8374A374B3848127831781B7800787A
:107E500002EB43034A1E03EB80030E2AEDD801A078
:107E600050F822F0CD7E0000EF7E00003B7E000047
:107E7000CD7E00003B7E00003B7E00003B7E00008C
:107E8000BB7E00003B7E00003B7E00003B7E00008E
:107E90003B7E00003B7E00003B7E0000B77E000082
:107EA000AE21224803F0FCFE204804F049F90023EB
:107EB0002B700124BFE706F0DFFBAF211B4803F066
:107EC000EFFE1B4A012313702B70B6E783B91948E4
:107ED000038804294FF6FF7103F1FF320CBF012321
:107EE0000B46134403F07F03013303800FE073B1AB
:107EF000013B114A32F813304BB10E4E0F48104976
:107F0000104A33800123002606700B701370084A54
:107F10000221012311702B70204670BD108BFF1FB2
:107F2000119FFF1F129FFF1F139FFF1F909FFF1F97
:107F30000CA0FF1FFC9EFF1F389EFF1F249DFF1FEC
:107F4000A59CFF1F0FA0FF1F10B5064B064C1A88FB
:107F50002046012101F04EFD21884220BDE810405D
:107F600001F05ABD089DFF1FC49CFF1F10B5064BB2
:107F7000064C1A882046022101F03CFD218842204F
:107F8000BDE8104001F048BD4A9DFF1FC49CFF1F83
:107F900010B5064B064C1A882046042101F02AFD34
:107FA00021884220BDE8104001F036BD6E9EFF1FC3
:107FB000C49CFF1F10B5064B064C1A8820460021B2
:107FC00001F018FD21884220BDE8104001F024BDD9
:107FD000BA9EFF1FC49CFF1F08B5122001F036FD9A
:107FE000054B1988884206D0122001F015FDBDE826
:107FF000084001F029BC08BDB09EFF1F08B55820FD
:1080000001F024FD054B1988884206D0582001F064
:1080100003FDBDE8084001F017BC08BDBE9EFF1F70
:1080200008B5142001F012FD054B1988884206D0CE
:10803000142001F0F1FCBDE8084001F005BC08BDCA
:10804000529DFF1FF0B480EAE075A5EBE0750028B3
:10805000ACB21FDB1DBF2B230B704E1C0E46012341
:1080600000E0134603EB830252009542F9DA0B4F0E
:1080700094FBF3F287FB030503FB1244DB1730325A
:10808000D3EBA503A4B206F8012BF1D13370084657
:10809000F0BC70472D230B704E1CE0E767666666E8
:1080A000084B188828B10D2807D00D3800B2FFF70B
:1080B000C9BF054A106808607047044A1068086024
:1080C000704700BF669FFF1FA433010038340100D2
:1080D000174B18880C2813D0192815D01A2817D038
:1080E0001B2819D01C281BD01D281DD01E2803D0EA
:1080F0000C3800B2FFF7A6BF0E4A10680860704740
:108100000D4A1068086070470C4A10680860704794
:108110000B4A1068086070470A4A10680860704788
:10812000094A106808607047084A1068086070477C
:10813000FA9EFF1F543401003C340100403401001A
:1081400044340100483401004C3401005034010033
:10815000034B1888A0EB8000400000B2FFF772BF0D
:10816000F49FFF1F024B1888033800B2FFF76ABF65
:10817000D29EFF1F024B18880C3800B2FFF762BF77
:108180009E9CFF1F024B1888183800B2FFF75ABF99
:10819000D09CFF1F024B1888183800B2FFF752BF5F
:1081A000CE9CFF1F024B1888183800B2FFF74ABF59
:1081B0000E9FFF1FC3681888183800B2FFF742BF30
:1081C000054B1B881BB9054B1868086070470846AB
:1081D0000422034909F0D2BDDC9EFF1FA433010035
:1081E000A0330100054B1B881BB9054B18680860BC
:1081F000704708460422034909F0C0BDD69CFF1F02
:10820000A4330100A033010030B5134C85B0012523
:108210002B463C2202212046009503F0B7FD204664
:1082200003F08EFF0022402180232046019100931D
:1082300011460A4B029504F031FC204604F08CF8FC
:1082400007480849084A0023036083800B608B803D
:108250001360938005B030BD909FFF1F0C2F01006D
:10826000749FFF1F889FFF1FFC9FFF1F10B500EB2F
:10827000C00000F10F02D2B293B284B09C1E981CD1
:108280003D2303918DE819003921024804F06AFB6F
:1082900004B010BD909FFF1F014B01221A70704760
:1082A000819FFF1FF0B5704B704C714F714E724D36
:1082B00085B004228DE80C00029320466F4B4022CB
:1082C000802103F06BFB20466D4C6E4A6E4908F02E
:1082D000CDFEA7616D486E4FE7616E4F87616E49B5
:1082E0006E4FC7616E4F8F616E4A6F4FCF616F4F98
:1082F00097616F4B6F4FD7616F4F9F616F4FDF611A
:108300006F4FB7616F4FF7616F4FAF616F4C704F39
:10831000EF61704FA7617048704FE761704F8761E0
:108320007049714FC761714F714A8F61714FCF6151
:10833000714F724B9761724FD761724F724E9F614E
:10834000724FDF61724F734DB761734FF761734FB7
:10835000734CAF61734FEF61734F7448A761744FF3
:10836000E761744F74498761744FC761744F8F61BF
:10837000744A754FCF61754F9761754B754FD761D3
:10838000754F9F61754E764FDF61764FB761764DC1
:10839000764FF761764FAF61764C774FEF61774F4D
:1083A000A7617748774FE761774F87617749784FC3
:1083B000C761784F8F61784A784FCF61784F976166
:1083C000784B794FD761794F9F61794E794FDF6153
:1083D000794F7A4DB7617A4FF7617A4F7A4CAF6136
:1083E0007A4FEF617A4F7B48A7617B4FE7617B4F04
:1083F0007B4987617B4FC7617B4F7C4A8F617C4F94
:10840000CF617C4F7C4B97617C4FD7617C4F7D4E19
:108410009F617D4FDF617D4F7D4DB7617D4FF7617E
:108420007D4F7E4CAF617E4F7E487F49EF617F4F2D
:108430007F4DA761E5617F4F7F4D804CDFF820E2E3
:108440007F4A804B8761C5618C617F4E7F4F804D35
:10845000804CC1F81CE0804880499761D5619C61DF
:10846000D861B16005B0F0BD40420F00909FFF1F82
:1084700075810000B88DFF1F288DFF1F7091FF1FB1
:10848000DC8DFF1F1C89FF1FF5B90000788FFF1FCF
:10849000F16D000065810000C48EFF1FFD6D0000BE
:1084A00085700000BC8CFF1F497F0000AD7000008C
:1084B0009C8FFF1F6D7F0000D5700000917F000032
:1084C000D17700000D6E0000FD700000948DFF1F3D
:1084D000B57F000051810000708DFF1F35730000D3
:1084E0004D730000548FFF1F41730000057800009A
:1084F000508CFF1F1D770000397800000890FF1F87
:10850000D97F0000A97A0000048DFF1FFD7F0000C5
:10851000A5730000108CFF1F1D6E00002571000068
:108520009890FF1F21800000117B0000E08CFF1F4E
:108530002D6E0000797B0000008EFF1F3D6E000055
:10854000E97B0000988CFF1F4D6E00000574000051
:10855000C88BFF1F5D6E0000757800005090FF1FF4
:108560006D6E00005D7400000C8FFF1F7D6E0000BB
:10857000A9780000808BFF1F8D6E0000B57400008D
:10858000388BFF1F9D6E0000DD780000C88AFF1F3A
:10859000AD6E00000D7500004C8DFF1FBD6E00001C
:1085A000B57D0000308FFF1FCD6E000015790000F3
:1085B0003491FF1FDD6E0000517C0000A08EFF1F74
:1085C000ED6E0000B97C00005C8BFF1FFD6E0000AB
:1085D000497900002C90FF1F3D770000217D0000AD
:1085E000E88EFF1F0D6F0000D1800000A48BFF1FDD
:1085F0001D6F000081790000148BFF1F2D6F00009C
:10860000E9790000808AFF1F3D6F0000A180000013
:108610000091FF1F4D6F000065750000748CFF1FF7
:108620005D6F0000EC8AFF1FEC8BFF1FBD75000023
:108630006D6F0000157600007D6F00006D76000004
:10864000C08FFF1FA48AFF1F2891FF1FC57600005F
:108650009D6F0000917D0000AD6F0000E98B000070
:108660008D6F0000F0B5461C83B00D460127032333
:1086700036B22AB2044631468DE888002448ADB2AD
:1086800004F006F90C23AA1C12B2009301970523EB
:1086900021B21F4804F0FCF81E4A1F4B12881B68C9
:1086A000BA422AD023D3022A10D11C4CA3F6CA0303
:1086B00084FB03241C44DB17C3EB24140A2CA8BF3F
:1086C0000A2424EAE474A2B223B202E000231A4688
:1086D0001C460D35AA1A01200093019012B23146B2
:1086E00003230B4804F052F8204603B0F0BD0C4CB5
:1086F000A3F6FC0384FB0324DDE7084CA3F69803F0
:1087000084FB03241C44DB17C3EBE404D6E700BF5F
:10871000909FFF1F589EFF1FC09EFF1F898888885B
:108720001F85EB512DE9F0438FB283B0DFF84C8009
:10873000BD1D461D2DB204B236B24FF001090AB27A
:108740002346314640460095CDF8049004F050F899
:108750002A463346214640468DE8200204F048F878
:1087600007F10C020095334612B22146CDF8049071
:10877000404604F03DF803B0BDE8F083909FFF1F32
:108780002DE9F043804685B0002956D101213048BB
:1087900004F0C4FB2F4998F8062098F8083011F827
:1087A0000290994522DA4FEA89064D460C24D8F802
:1087B0000C3027489B595F6822B2002104F0AAFBC5
:1087C000384609F01DFA39460246214804F03CFDBE
:1087D0001F4804F04FFD98F8083001350934AB42CA
:1087E000A4B206F1040601DD422CE0D1B9F1000F7C
:1087F00013D109F1060999450CDA3C2301213B22EA
:10880000039102930093019239233F223A211048A9
:1088100004F0A8F805B0BDE8F0830F2301213B2246
:10882000039102930093019239230C223A210848C4
:1088300004F098F898F80830DBE70021342300931F
:1088400001913F230C22024803F0A0FF9EE700BFE6
:10885000909FFF1F889FFF1F10B5104C01212046DD
:1088600004F062FB2046012104F058FB204634222C
:10887000552104F04FFB20460222094904F0E4FC94
:1088800020460522074904F0DFFC204604F0F2FCF4
:108890002046BDE8104003F05FBD00BF909FFF1F62
:1088A000A0340100A434010070B50D46064609F05D
:1088B000A7F900EB40008400002D36D0284609F0CF
:1088C0009FF900EB4000400023185B1003F16001AA
:1088D000091A282209B21748C3F1600404F01AFBF0
:1088E0000121144804F01AFB284609F089F92946A9
:1088F0000246104804F0A8FC0E4804F0BBFC02211C
:108900000C4804F00BFB21B221220A4804F002FBC0
:10891000304609F075F931460246064804F094FCE9
:108920000448BDE8704004F0A5BC6410C4F16004C4
:10893000E5E700BF909FFF1F184B70B5B3F90030FB
:1089400083EAE374A4EBE374002B82B0A1B21EDBD4
:1089500068466D46012300E0134603EB8302520094
:108960009442F9DA0E4E91FBF3F286FB03E403FB2B
:108970001211DB173032D3EBA40389B205F8012BB7
:10898000F1D119462B70FFF78FFF02B070BD2D2378
:108990008DF800300DF101056846DBE77C9EFF1F76
:1089A0006766666610B50D4B1B5C51F82340237853
:1089B00084B013B1012004B010BD04AA01A942F88B
:1089C000103D2046A3699847A38A9B07F2D401A8CB
:1089D0000099FFF769FF012004B010BD749FFF1FCD
:1089E0002DE9F04F2F4DDFF8CCB0DFF8C4A0DFF851
:1089F000C8900FCD91B003AC0FC40FCD0FC40FCDF5
:108A00000FC42B6823600025A8462F462E4600E0A1
:108A10009846BAF8003024495BF8232028461123F1
:108A2000F7F7E0FE00EBC00400EB840089FB0034A4
:108A30000444C017C0EB6434C4F13C00C6F13C02EE
:108A400007F14101012600B208F1410300901BB279
:108A5000019612B209B2154803F0CAFE08EB0603EC
:108A600005F211153C2B2646ADB24746D0D1342233
:108A70006B210E4804F04EFA00210C4804F04EFA27
:108A80000B4B1B8810AA02EB830353F8344C20468F
:108A900009F0B6F802460548214611B0BDE8F04F8E
:108AA00004F0D2BBA42C0100F0260100909FFF1F10
:108AB000B69CFF1F542501000900028010B5424CEE
:108AC000424882B003F03CFB2378C3B906213F48FB
:108AD00004F024FA2378012B37D90A22022B1146FD
:108AE0003A486BD004F016FA39490322374804F0AB
:108AF000ABFB364802B0BDE8104004F0BBBB354BC1
:108B00001A7801210523002A35D1019100931146DD
:108B10002E4803F0BDFE304B1A78002A36D00523CC
:108B200001220192009300220A21284803F02EFE20
:108B30002A4B1A78002A35D101210523019100938F
:108B40001421224803F0A4FEC0E7254C2388092BFA
:108B500032D9632B8CBF0A211F210A221B4804F043
:108B6000D9F92188194804F0D5FB184802B0BDE8AE
:108B7000104004F07FBB002201910093114613487E
:108B800003F004FE144B1A78002AC8D105230121F2
:108B9000019100930A210D4803F07AFE0F4B1A78D9
:108BA000002AC9D00122052301920093002214213A
:108BB000064803F0EBFD89E73021CEE704F0AAF97F
:108BC0000322084992E700BF0FA0FF1F909FFF1FDD
:108BD000B0340100119FFF1F129FFF1F139FFF1F43
:108BE000FC9EFF1FAC340100F8B56D4D287840B9EC
:108BF0006C4B1B6899425CD36B4A012313702B703A
:108C0000F8BD0C4600266948664F03F099FA04F651
:108C1000AC53324665483B6031212E7004F07AF93E
:108C200001216248624D04F07FF931465F4804F04B
:108C300075F905225F495D4804F006FB5B4804F0C6
:108C400019FB0C221021594804F064F90B225A49EF
:108C5000564804F0F9FA05225849544804F0F4FA49
:108C6000524804F007FB564B50481C68A4F6980382
:108C7000C3EB031385FB03251D441021DB172022C2
:108C8000C3EB652504F046F940F6CC339C4205F170
:108C900024054FF022014FF004000BDCFFF7E2FC4B
:108CA000484B1C88064674B3012C46D0022C41D098
:108CB0000120F8BDFFF736FD092243493B4804F087
:108CC000C3FA2A221021394804F024F93F4C3748CE
:108CD00084FB0534EB17C3EBA404214604F01AFB14
:108CE00001223B49314804F0AFFA04EB8401A5EBC3
:108CF00041012E4804F00EFB012236492B4804F0B6
:108D0000A3FA0120F8BD34491022284804F09CFA47
:108D1000264804F0AFFA2A221021244804F0FAF879
:108D20003146224804F0F6FA07222C491F4804F085
:108D30008BFACBE70C222A49E7E70C2229491B488A
:108D400004F082FA194804F095FA2A2210211748F3
:108D500004F0E0F8314615481C4E04F0DBFA072217
:108D60001E49124804F070FA86FB0536EB17C3EB78
:108D7000A60631460D4804F0CDFA224614490B48A8
:108D800004F062FA06EB8601A5EB4101074804F006
:108D9000C1FA22460F49054804F056FA2046F8BDAC
:108DA000108BFF1FF09FFF1F0CA0FF1F909FFF1F46
:108DB0003B773B98B4340100BC340100A43401007B
:108DC000C09EFF1F589EFF1FC8340100676666667D
:108DD000B03C0100203C0100D4340100E834010023
:108DE00000350100F03401002DE9F041754C227886
:108DF000002A05460F4614BF4FF001084FF0000847
:108E00004ED1714E3368CB1AB3F5FA6F04D86B7834
:108E1000A3B94046BDE8F0816C4B6D486D49DFF861
:108E2000D0E11A70012303700988237026208EF880
:108E3000002000F0F1FD6B78002BEAD03760F9F7E5
:108E4000FFF8654A654B6649127828781B780978DF
:108E500002EB4303421E03EB81030E2AD9D801A182
:108E600051F822F0558F0000218F0000138E000072
:108E7000558F0000138E0000138E0000138E00002B
:108E8000098F0000138E0000BB8E0000138E0000BF
:108E9000138E0000138E0000138E0000B78E0000AA
:108EA000AF215048484E02F0FBFEFFF707FE0023BB
:108EB00037602370ABE705F0DFFB4A4803F040F969
:108EC0000221484804F02AF80F222321454804F0E3
:108ED00021F805224449434804F0B6F9414804F01A
:108EE000C9F91E2223213F4804F014F805223F4906
:108EF0003C4804F0A9F93B4804F0BCF9394803F0B8
:108F00002BFA00F0ADFC84E7394D2B78012B50D9BA
:108F1000304B2620198800F07FFD00232B7078E766
:108F2000002B3FF476AF013B324A32F81330002B6E
:108F30003FF46FAF274C304825492D4A23804FF02E
:108F400001080023037081F8008082F80080FFF799
:108F5000B5FD5EE793B1013B264A32F8131019B311
:108F60001C4B254D1A4C224A19800026012326202D
:108F70002E702370137000F04FFD15E0154C1E4944
:108F800022880B7004284FF6FF7002F1FF310CBFEE
:108F9000012202460A440E4E154D02F07F020132B4
:108FA0000121228031702B70FFF788FD4FF00108FE
:108FB0002FE70649064A012300200870137023702A
:108FC000A6E700BF108BFF1F08A0FF1F0CA0FF1F0C
:108FD000A59CFF1FFC9EFF1F119FFF1F129FFF1FDD
:108FE000139FFF1F909FFF1F1035010018350100D0
:108FF0000FA0FF1F389EFF1F249DFF1F2DE9F04F7C
:1090000005468BB00F46AD480121164603F08CFF94
:10901000AA8812F0010440F0B080DFF8CC8298F802
:109020000030002B7DD1AB79A54AD15CA1B9DFF826
:10903000BCA279781AF8039041B33978013907292D
:1090400000F2B780DFE811F0F1005401B5006C01C7
:10905000B500B500B500E9007C78002C00F0CA80AE
:109060000139EC68387854F82170FC68411EB4F876
:109070000080072900F2A780DFE811F07401590190
:10908000A5006C01A500A500A5009F00DFF854A273
:10909000DAF80020B21AB2F5967F75D9894A1078AD
:1090A00001281ABF012010701170874A18BF0146AD
:1090B000D05CC0EB0900C0B2FFF7D8F80124CAF8B1
:1090C0000060AB889B0770D57B78002B6DD0F8F7DC
:1090D000B7FF7E4B7E4A7F481B781278397800783C
:1090E000022515FB02330A2903EB800300F04E81B1
:1090F0000C295AD1002B58D003F11900764E774A2B
:10910000013B0021400080B226F8131001231570A6
:1091100088F8003000F080FC714B032220461A7062
:109120002FE0664803F00CF80121644803F0F6FED6
:1091300062482246214603F0EDFEAB88580725D44D
:109140002C68204608F05CFD214602465B4804F08E
:109150007BF85A4804F08EF8092201238DE80C00B0
:1091600000217F23554803F043FB00212846FFF7E9
:1091700007FB002388F8003055E7AB6831463846D6
:1091800098470BB0BDE8F08F0846FAE72B6804A8B3
:10919000984704A808F034FD04A90246474804F0A3
:1091A00053F8464804F066F8D6E720460BB0BDE811
:1091B000F08F00240AF8039083E70021D154384649
:1091C000FB699847FC68A4F80080002725223C230F
:1091D0008DE8840041211822384803F0D7FAE96865
:1091E000A879FFF7DFFB374A3E4B17701E600BB0C4
:1091F000BDE8F08F3B490A68B21AB2F5967FD4D920
:10920000304F0E603E78012E00F0B480E9681846B9
:1092100001233B70FFF7C6FBB3E7304AE9791170D1
:10922000012288F800200024C4E72A7A013A4A453E
:10923000BFDD09F10104E4B2A145BAD0224E16F80F
:1092400003B0CBEB0900C0B20021FFF70FF82B7A77
:10925000052BD9461BD9CBEB0402042A40F3AE8080
:10926000A4F1040BBBF1000FC0F2B080063B5B45DC
:10927000A8BF5B465FFA83F9AA791348B15C9942AB
:1092800005D000F8029001212846FFF779FAC9EBD2
:109290000400C0B201210B4EFEF7E8FF0021342389
:1092A000019100930548317040230B223F21A146D4
:1092B00003F06CFA0124AB797CE700BF909FFF1F9D
:1092C000FC9FFF1F0DA0FF1F889FFF1F119FFF1F07
:1092D000129FFF1F139FFF1F389EFF1F0CA0FF1F31
:1092E0000FA0FF1FF89FFF1F108BFF1F749FFF1F12
:1092F0000FFA89F1E868604C50F821602168049108
:1093000034785E4904980860002C71D0012C7FF4F9
:1093100050AF5B4A317A88F800401170002449E769
:10932000B9F1000F50D009F1FF34E4B284E7B98AF3
:1093300001F0040189B200293FF440AF3B6A039277
:109340009847039A00283FF43DAFAB79FC680021B1
:10935000D15438E77B8A43453CD908F101081FFA0C
:1093600088F830E73B8A43453BD208F1FF381FFAC3
:1093700088F828E725238DE8180042483C703C23F4
:109380001822412103F002FA3046FAE6002B3FF49E
:109390000CAF3D4A3D4E1188394A03F11900013B9B
:1093A000400080B226F81310012388F800301570B1
:1093B00000F032FB364B20461D70E2E6002A3FF7F4
:1093C00055AF04F1FF3B4DE74C46F3E64FF0000983
:1093D0004B4651E7BB8ADA077FF5F5AEB7F8108048
:1093E000F1E6BB8AD9077FF5EEAEB7F81280EAE660
:1093F0002849C85CC0EB090009F1010EC0B2012187
:109400004FF0340B02F803E0FEF730FFB6681D485A
:10941000019440230B223F210124CDF800B003F03A
:10942000B5F940230B223F211648CDF800B0019436
:1094300003F02EFA2146134803F070FD304608F081
:10944000DFFBA0EB800000F15F0109B20F220D48A5
:1094500003F060FD304608F0D3FB31460246094870
:1094600003F0F2FE074803F005FFE968A879FFF76B
:1094700099FAAB799EE600BF4CA0FF1FF89FFF1F33
:109480000CA0FF1F909FFF1FFC9EFF1F389EFF1F19
:109490000FA0FF1F889FFF1F2DE9F047DFF80892FC
:1094A0006D4B99F800601B68DFF800A282B00036AF
:1094B00001934FF0030018BF0126019F9AF8008026
:1094C00004F092FD0546042004F08EFD04460520BC
:1094D00004F08AFD800040EA4404062004F084FD84
:1094E0002C4364B25D4944EAC0000A7880F00F035F
:1094F000DBB29A425A4A3CD01760002259480B709E
:1095000003788DF800808DF8012053B3564A126815
:109510004EF66021BA1A8A4219D8022B59D0012B73
:109520005FD0062B48D0032B63D0042B69D0052BCA
:1095300077D0072B7DD0082B00F08380092B68D0D3
:1095400016B14A4802F008FF02B0BDE8F087484A69
:10955000484C00230121237003701360938089F825
:1095600000103A4669464448FFF748FD3043C6B20A
:10957000E6E71268BA1A1E2A6BD99AF800209342BD
:1095800022D0394C3D488AF80030012B276082EA0E
:10959000030207609846B1D0042BAFD1374800686A
:1095A000381AB0F5C87FA9D9354C2068381A322846
:1095B000A4D927601A46A1E73A4669463148FFF721
:1095C0001DFD3043C6B2BBE7012B4FF00002E3D1D3
:1095D000E4E73A4669462C48FFF710FD3043C6B22F
:1095E000AEE73A4669462948FFF708FD3043C6B260
:1095F000A6E73A4669462648FFF700FD3043C6B263
:109600009EE73A4669462348FFF7F8FC3043C6B266
:1096100096E73A4669462048FFF7F0FC3043C6B269
:109620008EE73A4669461D48FFF7E8FC3043C6B26C
:1096300086E73A4669461A48FFF7E0FC3043C6B26F
:109640007EE73A4669461748FFF7D8FC3043C6B272
:1096500076E7002252E700BF4CA0FF1F10A0FF1FBB
:109660007C9FFF1F0CA0FF1F04A0FF1F909FFF1FE8
:10967000FC9FFF1F0EA0FF1FDC2E010014A0FF1F88
:10968000849FFF1F0C330100582E01006C2D010038
:10969000082D0100603B01005C2D0100C42D01007C
:1096A000A03B01002891FF1F108BFF1F809FFF1F11
:1096B00028B11028044BA8BF102018607047024B37
:1096C00001201860704700BF18A0FF1F38B50F4D6C
:1096D0002B78013B01381B02C4B203F470632004F1
:1096E00043F4404343F00C0300F4FE00184305F03C
:1096F000E3FD2868013860F03F00C0B204F00AFEC4
:109700002046BDE8384004F005BE00BF18A0FF1F8A
:1097100070B5124D2B78013B1B0203F470630646B3
:1097200043F430430806320400F0FE4043F00B03DC
:10973000034302F4FE0018430C4605F0BDFD286803
:10974000013860F04F00C0B204F0E4FD304604F090
:10975000E1FD2046BDE8704004F0DCBD18A0FF1F0D
:1097600070B5124D2B78013B1B0203F47063064663
:1097700043F410430806320400F0FE4043F00903AE
:10978000034302F4FE0018430C4605F095FD2868DB
:10979000013860F06F00C0B204F0BCFD304604F048
:1097A000B9FD2046BDE8704004F0B4BD18A0FF1F0D
:1097B00038B5104D2B78013B1B0203F4706304464F
:1097C00043F41043000443F0090300F4FE0018437F
:1097D00005F072FD2868013860F06F00C0B204F037
:1097E00099FD204604F096FD0020BDE8384004F0C5
:1097F00091BD00BF18A0FF1F38B50E4D2B78013B5F
:109800001B0203F47063044643F45043000443F026
:109810000D0300F4FE00184305F04EFD28680138E2
:1098200060F02F00C0B204F075FD2046BDE838405E
:1098300004F070BD18A0FF1F08B5002005F006FE5B
:109840000028FAD108BD00BF08B564210720FFF742
:109850005FFF7F210B20BDE80840FFF759BF00BF25
:1098600010B500217B20FFF753FF0024E0B2FFF783
:109870009FFF0134022004F0EDFB802CF6D110BDD7
:1098800010B504464FF4406004F0F4FC04F04CFDC5
:109890002CB1102C044BA8BF10241C6010BD024B2F
:1098A00001241C6010BD00BF18A0FF1F10B50446A6
:1098B00041F0E00004F02EFD04F07F0004F02AFDEA
:1098C000C4F3C610BDE8104004F024BD38B5134DF4
:1098D0002B78044641F6FF72A0F50050824203F156
:1098E000FF33A8BF02461B0202F5005203F4706367
:1098F000100443F4604343F00E0300F4FE005204EE
:10990000184302F0FE42104305F0D6FC29680139E5
:109910002046C9B2BDE83840FFF7C8BF18A0FF1FF6
:1099200038B504460D46F02004F0F4FC35B125446A
:1099300014F8010B04F0EEFCAC42F9D1F720BDE8BD
:10994000384004F0E7BC00BF00B50B4B83B00246C3
:10995000998818680090032AADF8041002D903B062
:109960005DF804FB684606218DF80520FFF7D8FF57
:1099700003B05DF804FB00BFE03B010000B50B4BFA
:10998000024683B0186899880090131F4C2BADF8DD
:10999000041002D903B05DF804FB684606218DF877
:1099A0000520FFF7BDFF03B05DF804FBE83B0100B5
:1099B000030203F4FE43C0F3C6101843704700BF10
:1099C00003784078DB0103F47E5300F07F001843F6
:1099D000704700BF82B002AA114642F8040D002071
:1099E00012F8013B03F07F03914243EA0020F7D1D4
:1099F00002B07047003210B403884FF0010404FA3B
:109A000001F418BF012202FA01F123EA04020A4319
:109A1000028010BC704700BF70B5CEB20C46054640
:109A200003F0AAFE864203D03146284603F0BEFE6C
:109A30000135284603F0A0FE240A844205D02146C1
:109A40002846BDE8704003F0B1BE70BD38B505468C
:109A500003F092FE4FF0000460F30704681C03F06B
:109A60008BFE60F30F24A0B238BD00BFF8B50446EA
:109A70000020FFF7EBFF002C00F09C854FF4AF6156
:109A80000220FFF7C9FF4FF47A610420FFF7C4FFFB
:109A90004FF496610620FFF7BFFF4FF4FA610820EC
:109AA000FFF7BAFF4FF4FA610A20FFF7B5FF40F65F
:109AB000B8310C20FFF7B0FF4FF42F612220FFF7E1
:109AC000ABFF40F6AC512420FFF7A6FF7D212A20F2
:109AD000FFF7A2FF0C210E20FFF79EFF01211020AF
:109AE000FFF79AFF02211220FFF796FF00211420B2
:109AF000FFF792FF00211620FFF78EFF02211820AA
:109B0000FFF78AFF01211A20FFF786FF01211C20A1
:109B1000FFF782FF04211E20FFF77EFF1421202083
:109B2000FFF77AFF01212620FFF776FF0321282087
:109B3000FFF772FF04212C20FFF76EFF14212E2067
:109B4000FFF76AFF00213020FFF766FF0C2132206B
:109B5000FFF762FF00213420FFF75EFF002136206F
:109B6000FFF75AFF00213820FFF756FF00213A2067
:109B7000FFF752FF00213C20FFF74EFF00213E205F
:109B8000FFF74AFF00214020FFF746FF0021422057
:109B9000FFF742FF1F214420FFF73EFF132146201D
:109BA000FFF73AFF0E214820FFF736FF11214A2028
:109BB000FFF732FF0A214C20FFF72EFF00214E2035
:109BC000FFF72AFF06215020FFF726FF022152202F
:109BD000FFF722FF0C215420FFF71EFF0021562023
:109BE000FFF71AFF00215820FFF716FF01215A2026
:109BF000FFF712FF08215C20FFF70EFF0A215E200D
:109C0000FFF70AFF00216020FFF706FF0421622012
:109C1000FFF702FF01216420FFF7FEFE002166200E
:109C2000FFF7FAFE0B216820FFF7F6FE7F216A207E
:109C3000FFF7F2FE00216C20FFF7EEFE00216E2000
:109C4000FFF7EAFE00217020FFF7E6FE00217220F8
:109C5000FFF7E2FE00217420FFF7DEFE1F217620D1
:109C6000FFF7DAFE13217820FFF7D6FE0E217A20C7
:109C7000FFF7D2FE11217C20FFF7CEFE0A217E20C5
:109C8000FFF7CAFE1F218020FFF7C6FE13218220A6
:109C9000FFF7C2FE0E218420FFF7BEFE11218620B1
:109CA000FFF7BAFE0A218820FFF7B6FE00218A20BE
:109CB000FFF7B2FE00218C20FFF7AEFE00219620B8
:109CC000FFF7AAFE00219820FFF7A6FE00219A20A8
:109CD000FFF7A2FE05219C20FFF79EFE06219E2095
:109CE000FFF79AFE0021A020FFF796FE7F21A22019
:109CF000FFF792FE40F2A461A420FFF78DFE4FF41F
:109D0000E161A620FFF788FE0021A820FFF784FE6E
:109D10000021AA20FFF780FE0221AC20FFF77CFE85
:109D20000121AE20FFF778FE0121B020FFF774FE7D
:109D30000B21B220FFF770FE2A210020FFF76CFEF6
:109D40000220FFF783FEB0F5805F034680F0F585C3
:109D5000D24A04201380FFF779FEB0F5805F0346F6
:109D600080F0E285CE4A06201380FFF76FFEA0F553
:109D70002F739BB2B3F57A6F024606D940F62821BD
:109D80000620FFF749FE40F62822C64B08201A801D
:109D9000FFF75CFEA0F52F739BB2B3F57A6F024616
:109DA00006D940F6E4410820FFF736FE40F6E442CB
:109DB000BD4B0A201A80FFF749FEA0F5FA739BB24B
:109DC00040F6AC518B42024606D94FF4FA610A20A4
:109DD000FFF722FE4FF4FA62B44B0C201A80FFF713
:109DE00035FEA0F5FA739BB240F6AC518B420246A9
:109DF00006D940F6B8310C20FFF70EFE40F6B83217
:109E0000AB4B0E201A80FFF721FE1828034600F204
:109E10008485A84A10201380FFF718FE431E9BB2CA
:109E20000F2B024604D901211020FFF7F5FD012276
:109E3000A14B12201A80FFF709FE0A28034600F200
:109E400065859E4A14201380FFF700FE0128034613
:109E500004D900211420FFF7DFFD0023984A1620C3
:109E60001380FFF7F3FD7F28034600F24885954AEB
:109E700018201380FFF7EAFD0528034600F2388515
:109E8000914A1A201380FFF7E1FD0C28034600F2E7
:109E900028858E4A1C201380FFF7D8FD042803462E
:109EA00000F218858A4A1E201380FFF7CFFD09288B
:109EB000034600F20885874A20201380FFF7C6FD7D
:109EC0004628034600F2F884834A22201380FFF7D5
:109ED000BDFDA0F5FA739BB240F6AC518B42024631
:109EE00006D94FF42F612220FFF796FD4FF42F6221
:109EF0007A4B24201A80FFF7A9FDA0F5FA739BB2D4
:109F000040F6AC54A342024604D921462420FFF770
:109F100083FD2246724B26201A80FFF797FD7F288B
:109F2000034600F2C2846F4A28201380FFF78EFD9B
:109F30000628034600F2B2846B4A2A201380FFF7FA
:109F400085FDA0F132039BB2B3F5967F024604D99A
:109F50007D212A20FFF760FD7D22644B2C201A8092
:109F6000FFF774FD0C28034600F29184604A2E200E
:109F70001380FFF76BFD1E28034600F281845D4AC3
:109F800030201380FFF762FD0928034600F2538456
:109F9000594A32201380FFF759FD1E28034600F26C
:109FA0004384564A34201380FFF750FD7F28034630
:109FB00000F23384524C36202380FFF747FD7F2880
:109FC000034600F2238438206380FFF73FFD7F289B
:109FD000034600F214843A20A380FFF737FD7F2860
:109FE000034600F205843C20E380FFF72FFD7F2825
:109FF000034600F2F7833E202381FFF727FD7F28E9
:10A00000034600F2E98340206381FFF71FFD7F28AC
:10A01000034600F2DB834220A381FFF717FD394D91
:10A0200028804420FFF712FD3028034600F2C88341
:10A03000354A46201380FFF709FD3028034600F219
:10A04000B983324C48202380FFF700FD30280346B7
:10A0500000F2AA834A206380FFF7F8FC3028034609
:10A0600000F29C834C20A380FFF7F0FC30280346CD
:10A0700000F28E834E20E380FFF7E8FC01280346C0
:10A0800004D900214E20FFF7C7FC0023204A5020AE
:10A090001380FFF7DBFC431E3CE000BF609DFF1F09
:10A0A0002C9FFF1F0A9DFF1FF89EFF1FC49EFF1FCE
:10A0B000CC9CFF1F9E9CFF1F7C9EFF1FB09EFF1F1E
:10A0C000529DFF1FA29CFF1F669DFF1FEE9CFF1F5E
:10A0D000E49CFF1FD49CFF1F0A9FFF1F749EFF1F5D
:10A0E000709EFF1FFC9EFF1FD29EFF1F269FFF1F1B
:10A0F000B69CFF1F489DFF1F3C9FFF1FFA9EFF1F3E
:10A10000389EFF1FC49CFF1F0E9FFF1FD49EFF1F82
:10A11000E29CFF1F9BB20B2B024604D90621502064
:10A12000FFF77AFC0622CF4B52201A80FFF78EFCF5
:10A130000428034600F22683CB4A54201380FFF7FD
:10A1400085FC431E9BB21D2B024604D90C215420D2
:10A15000FFF762FC0C22C54B56201A80FFF776FCF5
:10A160000128034604D900215620FFF755FC00239F
:10A17000BF4A58201380FFF769FC7F28034600F28E
:10A18000FB82BC4A5A201380FFF760FC431E9BB23F
:10A19000092B024604D901215A20FFF73DFC012278
:10A1A000B54B5C201A80FFF751FC431E9BB2102B6D
:10A1B000024604D908215C20FFF72EFC0822AF4B91
:10A1C0005E201A80FFF742FC431E9BB21D2B024605
:10A1D00004D90A215E20FFF71FFC0A22A84B602049
:10A1E0001A80FFF733FC0228034600F2BF82A54A1B
:10A1F00064201380FFF72AFC0128034604D90121BB
:10A200006420FFF709FC01239F4A62201380FFF7B7
:10A210001DFCC31E9BB2012B024604D904216220FF
:10A22000FFF7FAFB0422994B66201A80FFF70EFC19
:10A230007F28034600F29482954A68201380FFF736
:10A2400005FC7F28034600F28582924A6A2013802B
:10A25000FFF7FCFB7F28034600F276828E4A6C20D3
:10A260001380FFF7F3FB0428034600F267828B4A52
:10A270006E201380FFF7EAFB1928034600F258828C
:10A28000874A70201380FFF7E1FB0228034600F2A3
:10A290004982844A72201380FFF7D8FB06280346C0
:10A2A00000F23A82804A74201380FFF7CFFB052822
:10A2B000034600F22B827D4A8A201380FFF7C6FBFB
:10A2C0000A28034600F21C82794A8C201380FFF78B
:10A2D000BDFB0428034600F20D82764A98201380C5
:10A2E000FFF7B4FB0128034604D900219820FFF7AB
:10A2F00093FB0023704A9A201380FFF7A7FB0128E5
:10A30000034604D900219A20FFF786FB00236B4AFD
:10A3100096201380FFF79AFB0B28034600F2E48196
:10A32000674A9C201380FFF791FB831E9BB2032B8F
:10A33000024604D905219C20FFF76EFB0522614BE4
:10A3400076201A80FFF782FB3028034600F2C68190
:10A350005D4A78201380FFF779FB3028034600F22E
:10A36000B7815A4C7A202380FFF770FB30280346D0
:10A3700000F2A8817C206380FFF768FB3028034649
:10A3800000F29A817E20A380FFF760FB302803460D
:10A3900000F28C818020E380FFF758FB30280346D1
:10A3A00000F27E814A4A82201380FFF74FFB30285B
:10A3B000034600F26F81474C84202380FFF746FB61
:10A3C0003028034600F2608186206380FFF73EFB61
:10A3D0003028034600F252818820A380FFF736FB25
:10A3E0003028034600F24481A020E380FFF72EFBD3
:10A3F0000128034604D90021A020FFF70DFB00230C
:10A40000354A9E201380FFF721FBC31E9BB20C2B05
:10A41000024604D906219E20FFF7FEFA06222F4BA2
:10A42000A2201A80FFF712FB431E9BB27E2B02462E
:10A4300004D97F21A220FFF7EFFA7F22284BA42026
:10A440001A80FFF703FBA0F5AF639BB2B3F5167F4D
:10A45000024647D940F2A461A420FFF7DDFA40F29A
:10A46000A4623FE02089FF1F5E89FF1F148AFF1F3F
:10A470003A9DFF1FBE9EFF1F989CFF1F608AFF1F13
:10A480005C89FF1F6C9EFF1FCC9EFF1FF49CFF1F6B
:10A490000C9FFF1F2C9DFF1FD89CFF1F8C9CFF1F34
:10A4A000669FFF1F589EFF1F389FFF1FF09EFF1FD4
:10A4B0007E9EFF1F669EFF1FD69CFF1F409DFF1FB5
:10A4C000B89EFF1FBA9CFF1FCE9CFF1F489EFF1F18
:10A4D000D09CFF1F509EFF1FDC9EFF1FC089FF1FE7
:10A4E000029FFF1FD74BA6201A80FFF7AFFAA0F5F7
:10A4F000AF639BB2B3F5167F024606D94FF4E16114
:10A50000A620FFF789FA4FF4E162CF4BA8201A800A
:10A51000FFF79CFA0628034600F2A480CB4AAA2043
:10A520001380FFF793FA0328034600F29580C84A88
:10A53000AC201380FFF78AFA0328034600F28680D6
:10A54000C44AB0201380FFF781FA0328034677D866
:10A55000C14AAE201380FFF779FA7F28034669D8F5
:10A56000BE4AB2201380FFF771FA7F285CD82B888F
:10A57000DFF808E3BA4FBB4ABB4DBC4EBC4CBD49EB
:10A5800003F0010CAEF800C0C3F3400EA7F800E0E2
:10A59000C3F380071780C3F3C007B74A2F70C3F314
:10A5A0000017C3F34015C3F38013378025800B8059
:10A5B0001080F8BD4FF6FF7398423FF45FAA2A2837
:10A5C0003FF4BEAB17287FF659AA19287FF6C2AA16
:10A5D0001B287FF6DFAA1C283FF4F4AA1E287FF66A
:10A5E000F9AA1F283FF4FEAA20283FF417AB212820
:10A5F0003FF420AB22283FF425AB23283FF42EABB9
:10A6000024283FF45FAB25283FF464AB26283FF4B1
:10A6100065AB27283FF46AAB28283FF475AB29289F
:10A620007FF48AABFFF778BBB2200B21FFF7F4F978
:10A630000B209CE70121AE20FFF7EEF901238FE705
:10A640000121B020FFF7E8F9012381E70221AC20C6
:10A65000FFF7E2F9022373E70021AA20FFF7DCF9F4
:10A66000002364E70021A820FFF7D6F9002355E76F
:10A670000A218820FFF7D0F90A23B5E611218620A8
:10A68000FFF7CAF91123A7E60E218420FFF7C4F9CA
:10A690000E2399E613218220FFF7BEF913238AE6E1
:10A6A0001F218020FFF7B8F91F237BE60A217E20B7
:10A6B000FFF7B2F90A236DE611217C20FFF7ACF910
:10A6C00011235FE60E217A20FFF7A6F90E2351E64B
:10A6D00013217820FFF7A0F9132342E61F217620EB
:10A6E000FFF79AF91F2333E600219620FFF794F92C
:10A6F000002315E600218C20FFF78EF90023ECE5FE
:10A7000000218A20FFF788F90023DDE5002174206D
:10A71000FFF782F90023CEE500217220FFF77CF9D4
:10A720000023BFE500217020FFF776F90023B0E594
:10A7300000216E20FFF770F90023A1E500216C20B5
:10A74000FFF76AF9002392E57F216A20FFF764F999
:10A750007F2383E50B216820FFF75EF90B2374E567
:10A7600000216620FFF758F9002365E500216020ED
:10A77000FFF752F900233AE500215820FFF74CF982
:10A780000023FEE402215220FFF746F90223D3E41E
:10A790000A214C20FFF740F90A236BE411214A20DB
:10A7A000FFF73AF911235DE40E214820FFF734F951
:10A7B0000E234FE413214620FFF72EF9132340E424
:10A7C0001F214420FFF728F91F2331E400214020F6
:10A7D000FFF722F900231EE400213E20FFF71CF9B9
:10A7E000002310E400213C20FFF716F9002302E4C7
:10A7F00000213A20FFF710F90023FFF7F4BB0021F6
:10A800003820FFF709F90023FFF7E5BB00213620C8
:10A81000FFF702F90023FFF7D6BB00213420FFF732
:10A82000FBF80023FFF7C6BB0C213220FFF7F4F83A
:10A830000C23FFF7B6BB00213020FFF7EDF8002313
:10A84000FFF7A6BB649DFF1FE49EFF1F9A9CFF1F9E
:10A85000109DFF1FCE9EFF1F5C9EFF1FE09CFF1FF1
:10A86000089DFF1F4A9DFF1F5E9EFF1F6E9EFF1FDC
:10A87000D09EFF1F829EFF1FFE9CFF1FBA9EFF1FE0
:10A8800014212E20FFF7C8F81423FFF778BB04210A
:10A890002C20FFF7C1F80423FFF768BB0321282011
:10A8A000FFF7BAF80323FFF747BB01212620FFF784
:10A8B000B3F80123FFF737BB14212020FFF7ACF8D2
:10A8C0001423FFF701BB04211E20FFF7A5F8042382
:10A8D000FFF7F1BA01211C20FFF79EF80123FFF7D3
:10A8E000E1BA01211A20FFF797F80123FFF7D1BA47
:10A8F00002211820FFF790F80223FFF7C1BA0021C8
:10A900001620FFF789F80023FFF7B1BA02211220C1
:10A91000FFF782F80223FFF794BA0C210E20FFF70D
:10A920007BF80C23FFF775BA4FF47A610420FFF728
:10A9300073F84FF47A63FFF715BA4FF4AF61022052
:10A94000FFF76AF84FF4AF63FFF702BAF8B5C52016
:10A9500006F0C6FB204B214A054603CB1368C5F819
:10A9600003001A0CB420C5F807102B80AA70FFF75B
:10A970001FF82E46002426F80B0FA0B2FFF766F84A
:10A98000FFF716F80234B42C26F8020FF5D16C1E2E
:10A9900005F1C0064FF0FF3014F8013F082758407A
:10A9A0000F4B40F300017A1E0B4012F0FF0783EAC1
:10A9B0005000F5D1B442EFD1C043FFF70BF83A464F
:10A9C000C5F8C100C521284604F0C4FC2846BDE8EE
:10A9D000F84006F08DBB00BFF43B0100F03B0100E6
:10A9E0002083B8EDF0B50E4B0E4C054693E80700FA
:10A9F00085B024682E88AD7801AB83E80700270C6A
:10AA0000184600220B21ADF804408DF80670ADF811
:10AA10000C608DF80E5004F09DFC05B0F0BD00BF39
:10AA2000003C0100F03B0100F0B5124B124D1E68D6
:10AA3000124F0FCD87B06C460FC495E8030044F861
:10AA4000040B38683B79CDF80D00320C2A202180A8
:10AA50008DF802208DF81130ADF80060FEF7A8FFE8
:10AA60000022ADF80B001221684604F073FC07B019
:10AA7000F0BD00BFF03B01000C3C0100A43401001C
:10AA8000002004F0E3BC00BF02F02EBE70B5124CF3
:10AA900082B00025402306462946204600930195B2
:10AAA0008023202201F072FE20222946204602F057
:10AAB00031FA2046012102F037FA304607F0A0F8BB
:10AAC00031460246204602F0BFFB204602B0BDE8F8
:10AAD000704001F041BC00BF909FFF1FF0B5C4293A
:10AAE00083B075D90546441E00F1C0064FF0FF3013
:10AAF00014F8012F08275040404A40F300017B1E04
:10AB00000A4013F0FF0782EA5000F5D1B442EFD1BA
:10AB1000C043FEF75FFF0146D5F8C1000190019ADE
:10AB2000914202D0B2F17F2F0BD105F10B00FEF75D
:10AB300047FFB4280BD03248FFF7A8FF002003B02E
:10AB4000F0BD3048FFF7A2FF384603B0F0BD05F175
:10AB50000D00FEF735FF2A2840D1002440F6AC5600
:10AB600013E004281AD0062821D008281FD00A286C
:10AB700028D00C2822D1A1F5FA7292B2B24201D8A3
:10AB8000FEF74AFF0234B42C0ED004F10D00284425
:10AB9000FEF716FF022C0146A0B2E2D1B1F5805FAC
:10ABA000EED30234B42CF0D1012003B0F0BDA1F5F6
:10ABB0002F7292B2B2F57A6FE4D8E1E7222801D081
:10ABC000242811D1A1F5FA7292B2B242DAD8D7E7AD
:10ABD0000D48FFF75BFF002003B0F0BD0B48FFF707
:10ABE00055FF002003B0F0BD2A28C9D1A1F13202DF
:10ABF00092B2B2F5967FC5D8C2E700BF2083B8ED08
:10AC0000503C01003C3C0100243C0100643C01003C
:10AC100003290CD970B5461C82B005460C46304657
:10AC200003222A4907F05AF810B102B070BD7047EC
:10AC30000B2C05D905222649281D07F04FF840B1F5
:10AC40002448FFF723FF244802B0BDE87040FFF717
:10AC5000C9BE05F10901032201A807F08FF801A878
:10AC600003221E4907F03AF8D8B103221C4901A873
:10AC700007F034F808B301A803221A4907F02EF8A8
:10AC8000B0B91948FFF702FFA11E89B23046FFF79D
:10AC900025FF0028C9D0154802B0BDE87040FFF775
:10ACA000F5BE1348FFF7F2FEFFF750FE1148F3E739
:10ACB0001148FFF7EBFE1148C6E71148FFF7E6FE23
:10ACC00002B0BDE87040FFF7AFBE00BFF03B01002F
:10ACD0007C3C0100843C0100983C01009C3C01004C
:10ACE000C43C0100DC3C0100E03C0100F43C0100FC
:10ACF000A03C0100B43C0100083D01001C3D0100E6
:10AD0000C83C01002DE9F043174D2B6883B0814604
:10AD10000F469046F3B1154E34880A1992B2184680
:10AD20001146328006F05AFD28603A4649462044D2
:10AD300002F06CFDB8F1000F09D031882868FFF7E8
:10AD400067FF286806F0D4F900232B60338003B036
:10AD5000BDE8F083054E01930846318006F0C0F946
:10AD6000019B28601C46E0E720A0FF1F1CA0FF1FDE
:10AD700010B51F4C4FF4FA70FBF7B2FE204601F0FD
:10AD8000DFF900221146204602F0C4F820460121D6
:10AD900002F0CAF82046002102F0C0F80B22154943
:10ADA000204602F051FA204602F064FA0F221249BE
:10ADB000204602F049FA204602F05CFA0F490722C9
:10ADC000204602F041FA204602F054FA204601F0F3
:10ADD000C3FA0B4B0B4A1A604FF4FA70FBF780FE74
:10ADE000FFF722FE0848BDE81040FFF74FBE00BF46
:10ADF000909FFF1F203D01002C3D01003C3D0100C4
:10AE0000D8A1FF1F05AD0000443D010000207047A0
:10AE100090F8392090F83800101A704790F83830C0
:10AE200090F839209A4205D95A1C034480F83820FA
:10AE3000187E70474FF0FF30704700BF90F83830F1
:10AE400090F839209A4286BF1B18187E4FF0FF30C9
:10AE5000704700BF704700BF38B50546B0F85E00C8
:10AE600090B195F85D301446C3F1210294420CD89C
:10AE700005F13B001844224602F0C8FC95F85D300D
:10AE8000234485F85D30204638BD012014462871E2
:10AE9000EEE700BFB0F85E306BB190F85D30202B6C
:10AEA00007D8C218013380F85D30012082F83B10CA
:10AEB0007047012303710020704700BF00234269DF
:10AEC00080F8383080F8393080F85C3080F85D30B8
:10AED00080F85E3080F85F3006CA30B40D680469CF
:10AEE00043662A4383660A60A370426990F8613022
:10AEF0001649146813441D7A5B7B01EBC5051B02E0
:10AF00006D6803F4E06343F064032B6090F86230F3
:10AF100013449D7CDB7D01EBC5011B02496803F4F2
:10AF2000E06343F064030B6021685368194205D065
:10AF3000036927225A70036904229A710369202247
:10AF40005A71036980229A7030BC704778480100BA
:10AF500043690CCB12681A420CD0094B99420AD9AA
:10AF6000084B9942036994BF1A220D225A70036953
:10AF700004229A717047036927225A70F7E700BFCD
:10AF80007F1A06003F420F0010B50269D378DBB28A
:10AF9000D90604463DD510215806D17038D503F0A6
:10AFA000040303F0FF02002B51D03D49626E0023E1
:10AFB0000B7084F85D30002A5BD0904794F85D30C8
:10AFC000002B56D02369D0229A70236994F83B2035
:10AFD0001A712369012284F85C200222DA7010BD04
:10AFE000304B84F860009C424AD02F4B9C4252D098
:10AFF00094F8391013791F29DBB207D82848007854
:10B0000020B16018013184F8391003760223D3701F
:10B0100010BD5906C3D4917801F0100101F0FF0072
:10B020000029DDD013F001031ED194F85C1094F8D0
:10B030005D00884281BF4B1C091984F85C3091F88F
:10B040003B3013712369D0229A702269DEE72369AD
:10B0500084F83920C0229A702369114A1979012194
:10B0600011700222DA7010BDC02393702269137927
:10B07000CCE70122002384F85D2084F83B30A1E76F
:10B08000626994F86130094913440322187A02F086
:10B0900043FD2269ACE7626994F861300449F3E743
:10B0A00024A0FF1F7091FF1FDC91FF1F11B1000052
:10B0B0001DB100000369DB7803F0200373B190F841
:10B0C00060300133DBB2012B80F860301AD942695D
:10B0D00090F861301344187A02F09ABD70B5426955
:10B0E00003F0FF0590F8613013440446187A02F02B
:10B0F0008FFDA36E5BB184F8385094F83900BDE839
:10B100007040184790F85F30002BE0D0704770BD5A
:10B110000148FFF7CFBF00BF7091FF1F0148FFF745
:10B12000C9BF00BFDC91FF1F2DE9F047374FDFF8A3
:10B13000E0903B68026982B006460093DDF800802B
:10B140000021A025D3789B065BD53B680193019B2A
:10B15000C8EB03030F2BF5D949B1102BF2D0002017
:10B160009070336980229A7002B0BDE8F0877269EE
:10B1700096F8613013440521187A02F043FF726992
:10B1800096F861301344012193F812A0504602F062
:10B1900039FF09240021504602F020FF2B46013BD5
:10B1A000FDD10121504602F019FF2B46013BFDD194
:10B1B000013CEFD1706996F8611001444FF4A07220
:10B1C0000C7A4B7B09EBC4011B02496803F4E06372
:10B1D00043F064030B6096F862300344997CDB7D96
:10B1E00009EBC1011B02496803F4E06343F0640307
:10B1F0000B60013AFDD13269D3789B064FF0010113
:10B20000A3D4012002B0BDE8F08700BF4CA0FF1F0F
:10B2100078480100F0B503691222DA700269937868
:10B2200003F0200385B004460D46002B5ED0B42306
:10B2300093703C4922690B680093009E05E00B68FF
:10B240000193019B9B1B042B42D8D37803F020036E
:10B2500003F0FF00002BF2D094F85D30002B31D0CA
:10B260004FF0000E4FF0020C04EB0E0393F83B304E
:10B2700013710B680393039F206907E09B060DD5AC
:10B280000B680293029BDB1B052B28D8C378DBB22B
:10B2900003F0020202F0FF06002AEFD080F803C09C
:10B2A0002669F378DBB2DF0632462DD49F062BD514
:10B2B000DB0731D40EF1010E94F85D305FFA8EFE9B
:10B2C0007345D1D800201DBB002384F85E3004E014
:10B2D0009070236980229A70042005B0F0BD8670BA
:10B2E0002369802204209A7005B0F0BD03F0FF06A8
:10B2F000FFF71AFF10B9042005B0F0BD236984F8E8
:10B300005F60B0229A7094E78023B3700420DAE77C
:10B3100026698023B370D7E7BEF1000F0CBF02206F
:10B320000320F6E74CA0FF1F2DE9F0410669002538
:10B33000122780F8385080F83950F770D0F810C0D4
:10B340009CF802E00EF0200E88B0044688461546B0
:10B350001E46BEF1000F49D0B4238CF80230784B62
:10B3600021691A680092DDF800E006E01A6801928F
:10B370000198CEEB0000042830D8C87800F02000F7
:10B3800000F0FF070028F1D04FEA480242F0010226
:10B39000D2B20A711A680292DDF808E0206906E06C
:10B3A0001A6803920399CEEB010105292AD8C178C6
:10B3B00001F0020101F0FF070029F1D04FF0020C6B
:10B3C00080F803C02269D17811F0110722D12DBB7A
:10B3D000002E0CBFA0238023937003E08F7023699D
:10B3E00080229A70384608B0BDE8F0810EF0FF0761
:10B3F000FFF79AFE0028F5D0236984F85F70B02229
:10B400009A70ACE787702369802238469A7008B03A
:10B41000BDE8F081802393700027E3E7012D75D00C
:10B42000A021917021690A79BE4667464FF0A80CA9
:10B430001A680492049805E01A680592059A121A8F
:10B44000052A4AD8CA7802F0020202F0FF08002A50
:10B45000F2D0CF702169CA78D2B212F0100F08462C
:10B460005AD1920658D5013DEDB2012D49D0BEF119
:10B470001F0F3BD90A79012DDAD11A680692069D71
:10B4800005E01A680792079A521B052A46D8C27827
:10B4900002F0020202F0FF01002AF2D00223C37080
:10B4A0002269D378DBB2D9063AD49B0634D5B023CF
:10B4B000BEF11F0F93703FD8226904EB0E0312797F
:10B4C0001A760EF1010E5FFA8EFE16B12369802204
:10B4D0009A7084F839E0774684E781F8028023691E
:10B4E00080229A70774684F839E07BE704EB0E02FD
:10B4F00091F8048082F818800EF1010E5FFA8EFE3A
:10B50000B9E781F802C021690846B0E7A821917027
:10B510002069BE460279B0E7774663E78170DEE7CF
:10B520001021A023D170013BFDD12269937803F053
:10B53000F7037746937055E723691B79C5E700BF8A
:10B540004CA0FF1F0148FFF71FBD00BF7091FF1FF8
:10B550000148FFF719BD00BFDC91FF1F704700BF16
:10B5600038B5144C037801225B000546204684F868
:10B570003B3084F85E2084F85D20FFF78BFC20468A
:10B580000021FFF747FE0B4C2978012320461A467D
:10B59000FFF7CAFE0128F6D194F8383094F8392024
:10B5A0009A4205D9E218013384F83830107E38BD4C
:10B5B000FF2038BD7091FF1F38B51B4C0378012266
:10B5C0005B000546204684F83B3084F85E2084F812
:10B5D0005D20FFF75FFC20460021FFF71BFE124CA9
:10B5E0002978204601230222FFF79EFE0228F6D189
:10B5F00094F8382094F839108A420FD2531CDBB2E9
:10B60000A018994284F83830007E0AD923440232C7
:10B610001B7E84F8382040EA032038BD4FF6FF70C7
:10B6200038BD40F47F4038BD7091FF1F0C2901D90F
:10B63000002070470231490001F0FE01FFF7BCBF56
:10B6400070B50C4C0378164601255B00204684F843
:10B650003B3084F85E5084F85D50FFF71BFC3146A8
:10B660002046FFF717FC29462046BDE87040FFF74B
:10B67000D1BD00BF7091FF1FF8B505460F461646B5
:10B68000412421463A462846FFF7DAFF611C02347E
:10B69000C9B232462846E4B2FFF7D2FF592CF0D1A6
:10B6A000F8BD00BF38B504460D463548FFF706FC27
:10B6B0006322802120462570FFF7C2FF012002F09F
:10B6C000C9FC204600225E21FFF7BAFF20465D211B
:10B6D000FFF746FF242801D0002038BD204606226F
:10B6E0000C21FFF7C9FF204601222B21FFF7A8FFFD
:10B6F000204601222C21FFF7A3FF20460E222D21F8
:10B70000FFF79EFF204600222E21FFF799FF2046DB
:10B7100001222F21FFF794FF204605223021FFF759
:10B720008FFF204601223121FFF78AFF20460022A9
:10B730003221FFF785FF204600223321FFF780FFEB
:10B74000204600223421FFF77BFF204600223521CE
:10B75000FFF776FF204600225B21FFF771FF2046AE
:10B7600010225C21FFF76CFF204620225D21FFF7AD
:10B7700067FF20468F225E21FFF762FF012038BD60
:10B780007091FF1F10B4047F4160022CC26002D090
:10B7900010BC01F0D7BB836810BC184790E80C00C0
:10B7A000F0B41C6859682568164F174E294321606C
:10B7B000164D17491760D66015611160417A154A18
:10B7C0005C180A3194F8244053F8215002EBC4016C
:10B7D00049680D60017A5C1803EB8101247ECD6914
:10B7E00002EBC40149680D60817A581803EB8103AC
:10B7F00090F83000596B02EBC002F0BC536819603E
:10B80000704700BF01401F00011000380110007890
:10B8100000001F8078480100704700BFF0B50C1E83
:10B82000BDF8146034DBB0F906701919B942C4BF11
:10B830003B1B1BB2002BA6461CDD002A1146B8BFDD
:10B84000D11D02F00705CC10826A012007FB04E13C
:10B85000A840012E0A44C0B21ED00CD3022E09D13A
:10B86000013B12FA83F3013A12F8011F41409A4258
:10B870001170F9D1F0BDC043013B12FA83F3C0B29D
:10B88000013A12F8011F014093421170F9D1F0BD45
:10B8900023441BB20024C6E7013B12FA83F3013AAA
:10B8A00012F8011F01439A421170F9D1F0BD00BF97
:10B8B000F8B50D1E0EDB14461F46064601F03AFB96
:10B8C000A84207DD002C05DB304601F037FBA04223
:10B8D00001DCF8BDF8BD304601F02AFB022853D048
:10B8E00003284BD0012806D16540F3886C406540A1
:10B8F000013B5D1B2DB2012F03D02AD3022F14D0A0
:10B90000F8BD002C2246B6F90630B06AB8BFE21D79
:10B9100042F3CF0202FB035504F00704435D01210B
:10B9200001FA04F41C434455F8BD002C2246B6F934
:10B930000630B06AB8BFE21D42F3CF0202FB0355E6
:10B9400004F00704435D012101FA04F45C4044550E
:10B95000F8BD002C2246B6F90630B06AB8BFE21D29
:10B9600042F3CF0202FB035504F00704435D0121BB
:10B9700001FA04F423EA04044455F8BD3389013B79
:10B98000591B25460CB2B6E7F18832890139013AD4
:10B990004D1B141B2DB224B2ADE700BF2DE9F041C1
:10B9A000079E9DF91880089D04461F4600F0C0FFC1
:10B9B0000D4B0E480E4984F83380FF22002F08BF3C
:10B9C0001F4684F82F20002384F8302084F831208B
:10B9D00084F832202060A665E565676261652362B0
:10B9E000A3622046BDE8F0817091FF1FD03D0100A9
:10B9F0000110013810B50446806A034B236008B17A
:10BA000005F076FB204610BDD03D0100F8B5436A35
:10BA1000DBB190F82C200125AA4083F83B2083F865
:10BA20005E5083F85D500446406A03680E461B680A
:10BA300000219847606A036831461B689847294689
:10BA4000606ABDE8F840FFF7E5BBC26BC56C1368E0
:10BA5000046A23EA050313604CB122684FF00043E7
:10BA6000D3625163D36A002BFCDA936BF8BD836B0E
:10BA7000466B0825802410E03768426C3A433260F8
:10BA80001F68826C3A431A601A68876C013D22EA8B
:10BA900007024FEA54041A6007D02142ECD1326801
:10BAA000476C22EA07023260EAE7F8BD70B5044647
:10BAB000406A0D4600282BD0A16DFFF749FA002DF2
:10BAC00020460CBFA621A721FFF7A0FF606A20B186
:10BAD000E16DBDE87040FFF73BBA216C226D08684C
:10BAE000236A02430A6093B1DA7A82B1D00703D5A0
:10BAF000224A99691160DA7A910703D5204AD969F7
:10BB00001160DA7A520702D51E4A1B6A136070BDB3
:10BB1000236A002B2BD0D97A626DE1B172B6D97A43
:10BB2000CE0706D51848D96806683140996101608A
:10BB3000D97A880706D51548196906683140D96150
:10BB40000160D97A4E0705D5114859690668314018
:10BB50001962016062B61B68D968914207D00D482E
:10BB600018600D49DA6042F0804018611960226C5B
:10BB7000216D136823EA01031360A0E700E100E0F0
:10BB800004E100E008E100E080E100E084E100E0A1
:10BB900088E100E001403F0000003F80436A2DE95A
:10BBA000F04105460E469046002B3ED090F82C10F2
:10BBB0000124A14083F83B1083F85E4083F85D4088
:10BBC000406A036800211B6808F1FF379847FFB2FD
:10BBD000B8F1000F23D03744A046013E686A16F83A
:10BBE000011F03681B6898470134B742E4B216D0BE
:10BBF000202CF3D10121686AFFF70CFB95F82C206B
:10BC00006B6A520083F83B2083F85E8083F85D8086
:10BC1000686A036800211B6898470124DEE7686AA8
:10BC20000121BDE8F041FFF7F5BAC26BC16C1368A2
:10BC300023EA010306EB080413604FF00048A64214
:10BC40000ED02B6A16F801EB63B11A68C2F82C808B
:10BC5000C2F834E0D36A002BFCDAA642936BF0D131
:10BC6000BDE8F081AB6BD5F834C008208021DCF84A
:10BC700000206F6C1EEA010F14BF3A43BA43CCF8A0
:10BC800000201A68AF6C3A431A601A68AF6C01382A
:10BC900022EA07024FEA51011A60E8D1CFE700BF5C
:10BCA00070B50446406A0D46002828D0A16DFFF704
:10BCB0004FF920462946FFF7A9FE606A20B1E16DE1
:10BCC000BDE87040FFF744B9216C226D0868236A13
:10BCD00002430A6093B1DA7A82B1D00703D5234ACE
:10BCE00099691160DA7A910703D5214AD9691160FF
:10BCF000DA7A520702D51F4A1B6A136070BD236AA5
:10BD0000002B2BD0D97A626DE1B172B6D97ACE0709
:10BD100006D51948D9680668314099610160D97A19
:10BD2000880706D51548196906683140D961016050
:10BD3000D97A4E0705D5124859690668314019620B
:10BD4000016062B61B68D968914207D00D4818603F
:10BD50000D49DA6042F0804018611960226C216D53
:10BD6000136823EA01031360A3E700BF00E100E0CA
:10BD700004E100E008E100E080E100E084E100E0AF
:10BD800088E100E001403F0000003F802DE9F041E4
:10BD9000044686B0806A9DF830801E460F461546E0
:10BDA000B4F90830002800F04281DA1D48BF03F1E1
:10BDB0000E02B4F90630D21003FB02F2002105F0A6
:10BDC000BBFCB4F90820202A00F39280B4F90610D5
:10BDD000A34B0120203A733902EBD27201EBD171EF
:10BDE0004FF0200E029073208DE8014042F34F0285
:10BDF00041F34F01204600F051FE606A84F82D7037
:10BE0000002800F04D81002D40F08A80B4F9083000
:10BE1000202B14BF3D253C2584F82C50B8F1000F91
:10BE200040F0858006B394F93300002818DBC0B2D7
:10BE3000012102F0E7F8012194F8330002F0CEF876
:10BE4000012002F007F9002194F8330002F0C6F84F
:10BE50000A2002F0FFF8012194F8330002F0BEF846
:10BE6000606A002800F08280A16DFFF771F804225B
:10BE70007C492046FFF792FE217A0139C9B220465B
:10BE8000FFF7C4FD784904222046FFF787FE94F9A6
:10BE90002D30012B14BF142110212046FFF7B6FDD1
:10BEA000042272492046FFF779FEB4F90630802B50
:10BEB00000F09280602B00F0A680D9212046FFF789
:10BEC000A5FD94F92D30012B14BFF121222120462C
:10BED000FFF79CFD204606226549FFF75FFE606A7A
:10BEE00050B3E16DFFF734F8012006B0BDE8F081F2
:10BEF000B4F906105F4B0120403A52394FF0400E22
:10BF0000029002EBD272522001EBD1718DE8014018
:10BF100042F34F0241F34F01204600F0BFFD6CE7B2
:10BF20006DB284F82C50B8F1000F3FF47BAFFEF7F0
:10BF3000C5FF002E94D076E7216C226D0868236A35
:10BF400002430A6073B1DA7A62B1D00703D54A4A74
:10BF500099691160DA7A91077CD4520702D5474A71
:10BF60001B6A1360012006B0BDE8F081236A002B34
:10BF70002BD0D97A626DE1B172B6D97ACF0706D5E6
:10BF80003F48D9680568294099610160D97A8E07D0
:10BF900006D53C48196905682940D9610160D97AFC
:10BFA0004D0705D53848596905682940196201606F
:10BFB00062B61B68D968914207D03448186034498A
:10BFC000DA6042F0804018611960226C216D1368BC
:10BFD00023EA010313604AE7B4F90830202B00F08C
:10BFE0008680402B7FF469AF2A4920460322FFF761
:10BFF000D5FD94F92D30012B14BFCF219F21204670
:10C00000FFF704FD59E7B4F90830102B7FF455AF62
:10C01000214920460322FFF7C1FD94F92D30012B61
:10C0200014BFAF2110212046FFF7F0FC45E7DA1DD1
:10C0300048BF03F10E02B4F90630D21003FB02F23E
:10C040001046059205F04CF8A06200283FF44DAF71
:10C05000059AB3E6114AD9691160DA7A7DE700BF23
:10C06000283E0100084001000C4001001040010082
:10C07000144001001C40010000E100E008E100E084
:10C0800080E100E084E100E088E100E001403F0061
:10C0900000003F80243E0100DC42010004E100E09A
:10C0A000012194F83100244F01F0ACFF94F83200E4
:10C0B000012101F0A7FF94F9312094F9323057F8AB
:10C0C0003220E26357F83330206A23640125E564A7
:10C0D00025651A682A431A6078B1B8F1000F3FF459
:10C0E00028AFFFF75BFB002E3FF4BAAE9BE60422BD
:10C0F00012492046FFF752FDDFE6294694F82F004B
:10C1000001F080FF294694F8300001F07BFF94F99C
:10C110002F2094F9303057F83220626357F83330CB
:10C120006564A5641A68A36322F001021A60002EF8
:10C130003FF496AE77E600BF78480100203E01004C
:10C14000B0F90820D31D48BF02F10E03B0F9062054
:10C15000806ADB1002FB03F2002105F0EDBA00BF9C
:10C16000F0B50029BDF814502EDBB0F90660B142DD
:10C170002ADA002A59DBB0F9087014461C44BC4284
:10C18000C4BFBB1A1BB2002B1EDDD2B2D408D0F83C
:10C1900028E016FB041112F00702DBB20EEB0104DB
:10C1A00021D0C2F10807FAB2374F9342BF5C0CD2DC
:10C1B000C3EB020CFF2646FA0CF6012D07EA060730
:10C1C0003FD005D3022D36D0F0BD012D39D030D26D
:10C1D0001EF8016026EA07070EF801709342F3D3B8
:10C1E000B0F906100C449A1AD2B2072A10D9022DBF
:10C1F00036D0002D14BFFF26002613462670083BBC
:10C20000B0F90610DBB2072B0C44F7D802F0070296
:10C21000002AD9D01D4B012D9B5C1DD017D3022DB8
:10C22000D2D1227853402370F0BD13441BB20022B8
:10C23000A1E7022D25D11EF8016077400EF80170AC
:10C24000CCE71EF8016037430EF80170C6E722788C
:10C2500022EA03032370F0BD227813432370F0BD5C
:10C2600011462378DB4323700839B0F90630C9B290
:10C2700007291C44F5D812F00702A5D0034B9B5C9C
:10C28000CFE73444AFE700BFC03D0100B03D01003F
:10C2900070B4C47DBDF80C50022C18D0032C1FD0F4
:10C2A000012C0BD0002A03DBB0F90840944201DCDA
:10C2B00070BC7047039570BCFFF7B0BAC488039593
:10C2C000013CA41A0A4621B270BCFFF749BF068997
:10C2D000C488013E641AB21AE41A12B221B2E1E72C
:10C2E00004890395E41A641A114622B270BCFFF760
:10C2F00037BF00BF70B4C57DBDF80C60022D1AD0E9
:10C30000032D12D0012D03D0039670BCFFF728BF78
:10C31000C488E41AA41A0A4621B2002A03DBB0F941
:10C320000840944213DC70BC70470489013C641AD5
:10C33000114622B2F1E7C48805890396013CAD1A83
:10C34000ED1A621A11B22AB270BCFFF709BF039648
:10C3500070BCFFF763BA00BF2DE9F8430446406A9A
:10C36000002863D0A16DFEF7F3FD05227449204635
:10C37000FFF714FCA1790139C9B22046FFF746FB4B
:10C38000B4F90820E588A66AD31D48BF02F10E0360
:10C39000DB10626A15FB03F51FFA85F8002A7BD0D3
:10C3A00094F82C300125AB4082F83B3082F85E5087
:10C3B00082F85D50606A036840211B6808F1FF370E
:10C3C0009847BFB2B8F1000F23D03744A846013ECA
:10C3D000606A16F8011F03681B6898470135B74269
:10C3E000EDB216D0202DF3D10121606AFEF712FFC5
:10C3F00094F82C20636A520083F83B2083F85E8017
:10C4000083F85D80606A036840211B6898470125B6
:10C41000DEE70121606AFEF7FDFE606A002800F099
:10C420008D80E16DBDE8F843FEF792BD236A002BD5
:10C430002BD0D97A626DE1B172B6D97ACE0706D522
:10C440004048D9680568294099610160D97A8D070B
:10C4500006D53D48196905682940D9610160D97A36
:10C46000480705D5394859690568294019620160AE
:10C4700062B61B68D968914207D0354818603549C3
:10C48000DA6042F0804018611960226C216D1368F7
:10C4900023EA0103136068E7E26BE36C1168276A23
:10C4A0000B4306EB080913604FF0004E4E450DD0CC
:10C4B00016F801CB2FB33A68C2F82CE0C2F834C0AA
:10C4C000D36A002BFCDA4E45936BF1D1226C236DBD
:10C4D00011680B43136097B1FB7A83B1D90703D579
:10C4E0001D4BBA691A60FB7A9A0703D51B4BFA6990
:10C4F0001A60FB7A5B0702D5194B3A6A1A60BDE8ED
:10C50000F883A36BD4F8348008208021D8F8002069
:10C51000656C1CEA010F14BF2A43AA43C8F8002027
:10C520001A68A56C2A431A601A68A56C013822EAB9
:10C5300005024FEA51011A60E8D1B7E7276AC5E75B
:10C54000B83D010080E100E084E100E088E100E026
:10C5500001403F0000003F8000E100E004E100E016
:10C5600008E100E02DE9F04F85B09946BDF938703B
:10C57000BDF83CA0BB1AC1EB090B002BB8BF5B4256
:10C58000BBF1000FB8BFCBF1000B5B450D46164663
:10C590000093804648DC4D453A4633464CDC19460C
:10C5A00013460A46C5EB09019B1A89B2002B0CB24F
:10C5B000B8BF5B4204EBD474BE42ACBF4FF0FF3255
:10C5C00001224D45039102924FEA640429DC9BB29B
:10C5D00001930DE0D8F80070BF69B847019BE41AD9
:10C5E000A3B21CB20135002C2DB211DBA94518DB1A
:10C5F000009B5B452A46534631464046EADCD8F864
:10C60000002053469769294632464046B847E5E739
:10C61000029A1644039AA94502EB030436B224B2E7
:10C62000E6DA05B0BDE8F08F4A462B46B9463546F6
:10C630004D4517461E46B2DD304629463E464D461C
:10C6400007468946AEE700BF10B404682469A446D3
:10C6500010BC604730B40468BDF808500295A46B64
:10C66000A44630BC604700BF30B40468BDF8085031
:10C670000295E46BA44630BC604700BF70B4046808
:10C68000BDF90C60BDF8105003960495246CA446C7
:10C6900070BC6047704700BF10B582B0B0F90C2085
:10C6A00001910168009200220C6CB0F90A30114629
:10C6B000A04702B010BD00BF704700BF01F00301EA
:10C6C0000129C17506D0032904D0C288038942819B
:10C6D000838170470289C38842818381704700BF8C
:10C6E0002DE9F0410568134E6F6986B0B7420446E4
:10C6F000BDF8308010D1013B13441BB20093CDF83C
:10C7000004800B46AD6A2046A8472368DB6AB34223
:10C710000AD106B0BDE8F081059304920391B847B1
:10C7200003A925680EC9E6E7204606B0BDE8F0413A
:10C73000184700BF95C600002DE9F0410568124E6C
:10C740006F6986B0B7420446BDF830800FD1013B17
:10C75000CDF804800B4400921BB2AD6A2046A84776
:10C760002368DB6AB3420AD106B0BDE8F0810593C5
:10C7700004920391B84703A925680EC9E7E720464C
:10C7800006B0BDE8F041184795C600002DE9F04F0E
:10C790000568DFF858B06F6985B05F450646BDF99A
:10C7A0003890BDF83CA00C46904615D11F19BC42EC
:10C7B0000CDACDF800A0214601342D6A4B464246E2
:10C7C000304624B2A847BC423568F2DBEB6A5B45D1
:10C7D00007D105B0BDE8F08F0393B8473568039BD8
:10C7E000E4E7304605B0BDE8F04F184795C60000B5
:10C7F0002DE9F04387B099420546BDF93840BDF8B0
:10C800003C6025D0A24212D00768DFF88080D7F8BC
:10C810001490C14532D18DE850002846BC6AA0472B
:10C820002B68DB6A434524D107B0BDE8F083994209
:10C8300002DD08461946034628680E96C46B01338C
:10C840005B1A1BB22846A44607B0BDE8F043604718
:10C85000A24202DD134622461C4628680E96631C3F
:10C86000846B9B1A1BB22846A44607B0BDE8F04370
:10C870006047284607B0BDE8F04318470593049287
:10C880000391C84703A92F680EC9C4E795C60000E5
:10C890002DE9F04FD0F800E0DFF89090DEF814B00A
:10C8A00083B0CB450446BDF93080BDF834A00D46B9
:10C8B00017461E4631D1CDF800A0DEF824B0294637
:10C8C00033463A462046D8472368CDF800A008F101
:10C8D000FF323A44D3F824B0294612B233462046F8
:10C8E000D8472368CDF800A02946D3F820B03A46AF
:10C8F00043462046D8472068CDF800A0711E294441
:10C900004346056A09B23A462046A8472368DB6ACF
:10C910004B4506D103B0BDE8F08FD847D4F800E00E
:10C92000C9E7204603B0BDE8F04F184795C60000A0
:10C93000F0B4002401264FF6FF75094F076004711B
:10C94000C475C48104824476C46186750676858286
:10C950004582C180028141818281F0BC704700BF65
:10C96000E84201002DE9F04F85B00668BDF844505B
:10C97000BDF93880CDF8008004460195D6F848B05E
:10C980000392BDF93C60BDF9407089469A46D8478C
:10C9900023680195009742465146D3F848802046C7
:10C9A0003346C0472068039B0E930F95856C4B461A
:10C9B0003A4631462046AC4605B0BDE8F04F6047E8
:10C9C0002DE9F04F87B01746BDF94040009125464C
:10C9D000E91D059344BF2B4603F10E010268BDF823
:10C9E000486053690294C91003912B49BDF9444032
:10C9F00001968B42824645D1002C3CDD029B3C4493
:10CA00005E1EB6B24FF0000923B2049301364D46C4
:10CA1000029B002B28DD059B002403EB090806E0A0
:10CA2000EDB22B0604F1010411D4A6421CD0A1B230
:10CA300011F0070F23B24FEA4505F1D1002BB8BF23
:10CA40000733DB10013418F803502B06EDD5009B9B
:10CA5000D2F818B019443A4609B2019B5046D8475B
:10CA6000A642DAF80020E2D1039B01379944049BE7
:10CA70003FB2BB42CCD1D36A074A934206D107B03A
:10CA8000BDE8F08F9847DAF80020B5E7504607B0C8
:10CA9000BDE8F04F184700BF95C6000070B4BDF95F
:10CAA0000C60BDF91050BDF8144003960495059430
:10CAB00070BCFFF785BF00BF2DE9F04F93B09046E3
:10CAC0000591C1691090BDF870000790BDF8749091
:10CAD0009DF878A00493002900F0CD800A7A0AC955
:10CAE000894604998A1AD2B203EBC203BAF1010F44
:10CAF000DA780B9293F905201E8893F802B00F9212
:10CB000093F9064079D913B2099323B20C93109B81
:10CB10001A68A94B1193194653698B4240F0A680BD
:10CB20000B9B002B55D01FFA88F300210D93C846AC
:10CB30002344DDF8409006910E930F460C46BBF15E
:10CB4000000F3FD0BDF818100C9B03971FFA8AF016
:10CB5000CB1813FB00F304900E9801440D98034486
:10CB600009B21BB20A910893002505E00135EBB22A
:10CB700064009B45E4B222D9039B2B44590703D19F
:10CB8000731C18F806409EB22306EFD5099BBDF82A
:10CB90001000E91811FB00F10598BAF1010F0FFA26
:10CBA0008AF301441CD0079801900093D26909B21E
:10CBB00017464846089AB847D9F80020D6E7039F99
:10CBC0005F44FFB2069B0B9901330693DBB2994297
:10CBD000B5D8D36A119A934243D113B0BDE8F08F10
:10CBE0000F9B191893690A9A29441F4609B2079B9B
:10CBF0004846B847D9F80020B8E700230C930993BA
:10CC000085E70A9A0D9B0132013B52B213F0FF03F4
:10CC10000A920D936FD1DDF81890079BDDF83C80E8
:10CC2000DDF820A04B4517D0BAF1010F00F0C88005
:10CC30000B9A109DCDF804900BEB8B014FEACB03C0
:10CC40000A4400931146DEF81C405346424609B29E
:10CC50002846A047D5F800E0DEF82C30119A934220
:10CC6000BBD0109813B0BDE8F04F1847109D284670
:10CC700098472A6854E7109A0598B2F90A30834217
:10CC8000ABDDB2F90C304345A7DD062313FB0A03E5
:10CC9000002BA2DD08EBCA03002B9EDD537E2BB9CF
:10CCA000049BAF2B02D90133DBB20493109BD3F862
:10CCB00000E0414B11931A46DEF81430934240F0E5
:10CCC0008E801FFA88F30E9308339BB2BDF81420B0
:10CCD000059305230D9300230A93CDF83C800FFAAA
:10CCE0008AF3DDF84080CDF818900B921FFA8AFB8A
:10CCF000CDF820A099460A9ABDF810000B9C0E9D15
:10CD00000523194611FB00232C481146C75C0397E5
:10CD100002FB0B4214FA81F312B21BB209920C937C
:10CD20002C462E461CE0089B0999012B2AB24B4643
:10CD300040462DD0079F0197CDF80090DEF81CA04B
:10CD4000D047D8F800E0039B5B0801340393059BB0
:10CD5000A4B25D445E44A342ADB2B6B23FF451AF5B
:10CD6000039BD807DFD4079B069A9342EBD0089B1E
:10CD7000012B16D0069B0193CDF80090DEF81CA085
:10CD800009994B4632B24046D047D8F800E0DAE77E
:10CD9000DEF818A0079B0C9922B2D047D8F800E023
:10CDA000D1E7DEF818A00C991346404622B2D047CE
:10CDB000D8F800E0C7E700BF95C60000384301007F
:10CDC0000B99109DCDF800900531DEF8204009B296
:10CDD000424608232846A047D5F800E03CE7109CCF
:10CDE00020469847D4F800E06BE700BFF0B5C36970
:10CDF00085B004462BB30A2968D00D294AD01A7A87
:10CE0000914247D3587A884244D35D688A1A05EB29
:10CE1000C205AA78002A50D0E87800284DD0207E9C
:10CE200000283AD095F905E0B4F90E00A67DB4F9D2
:10CE30000A70724406FB0202BA4262DCB4F91020A6
:10CE400030E00A2956D00D2924D0027E002A4BD08A
:10CE5000B0F90E00A57DB4F90A60062212FB0502A6
:10CE6000B2423EDD228AE38102EBC50212B21846CD
:10CE70002282A78A668A02950B468DE8C000014689
:10CE80002046FFF719FEA37DE28903EB430302EB83
:10CE90004303E381012005B0F0BDA67DB4F90E0087
:10CEA000B4F91020B4F814E0678A02960B468DE8B6
:10CEB000804001462046FFF7FFFD2979E389A27DE6
:10CEC000012001FB0233E38105B0F0BD0022C281E5
:10CED0009A7A817D038A01FB02330382012005B027
:10CEE000F0BDB4F91020C4E7857DB4F91020B0F985
:10CEF0000E00BEE7028A817DC38102EBC10303827B
:10CF0000C8E70020E0819B7A228A03FB062212B246
:10CF10002282C7E7C1810282704700BF002908BF93
:10CF200001218175704700BF81824182704700BF37
:10CF3000C07D7047B0F90A00704700BFB0F90C001F
:10CF4000704700BF10B4EFF3108272B6437F33B95D
:10CF5000017F012907D003290FD00123437702B9AC
:10CF600062B610BC7047124C2168A1B111494361EF
:10CF70000B68836108605861EFE70F4C216881B14D
:10CF80000E4943610B688361086058610C4B4FF098
:10CF900080511960E1E7074B4161816120601860B1
:10CFA000DBE7064B4161816120601860EEE700BF5E
:10CFB00038A0FF1F34A0FF1F28A0FF1F2CA0FF1FB9
:10CFC00004ED00E070B5EFF3108272B60C4C2068EF
:10CFD00080B10C4E00254369236073B19D6102B995
:10CFE00062B6457783689847EFF3108272B620687F
:10CFF0000028F0D102B962B670BD3360EFE700BF20
:10D0000028A0FF1F2CA0FF1FFFF7DCBF184A30B479
:10D010001468002C27D0036821688B420ED2CB1AEB
:10D0200000218460C1602360E0601060022303750A
:10D0300030BC704711688B42144608D3A2685B1A53
:10D040000360002AF6D18260C460A060EEE7D26877
:10D05000C2608460E060C568CB1A0222A8602360C9
:10D06000027530BC70478460C4601060DEE700BFAA
:10D0700030A0FF1FF8B5224E34682CB32368002B74
:10D080003AD1204F1D4604E03468ECB12368002BF0
:10D0900032D1A36803B1DD60206933600368257570
:10D0A0001B68BB4221D1037F4560022BC46020D0A6
:10D0B000FFF748FF6368002BE6D023602046FFF7A8
:10D0C000A5FF3468002CE1D1EFF3108372B60E4A4D
:10D0D00000211068116003B962B628B18468FFF7B7
:10D0E00095FF20460028F9D1F8BD22460021984737
:10D0F000E0E783689847DDE7013B2360E4E700BF92
:10D1000030A0FF1F85B7000040A0FF1F024A136830
:10D1100001331360FFF7AEBF4CA0FF1F704700BF85
:10D120000368F0B4FBB1002501249D60DC601B4C5A
:10D130001A601C44241104F144056A11032692006C
:10D140009E60174F0679174B47F8241002F1604292
:10D1500002F5614205F01F05012000FA05F5E654CD
:10D160001560F0BC7047104C236843F40003236043
:10D1700000BF0E4B0E4DA4F58734A4F59E74012616
:10D180001E60234604609C68002CD0D01033AB4254
:10D190000360F8D1002303601846E2E7008FFCBF6C
:10D1A0004892FF1F44E400E03C80044000700340CC
:10D1B000407103400168A9B10B4BF0B40B441B1143
:10D1C0000A4E0B4F0B4D46F8237003F1440202F058
:10D1D0001F0401235211A340002445F822308C6023
:10D1E0000460F0BC704700BF008FFCBF4892FF1F77
:10D1F0001DD1000080E100E0024A034B01211160D3
:10D200001B6818470C7103404892FF1F024A034BEA
:10D21000012111605B6818471C7103404892FF1F91
:10D22000024A034B012111609B6818472C7103408F
:10D230004892FF1F024A034B01211160DB68184727
:10D240003C7103404892FF1FF8B50E4671B17AB1A8
:10D250000746144600253B6816F8011B1B68384634
:10D260009847013C0544F6D12846F8BD0846F8BD6C
:10D270001046F8BD00B5064A036812885B6883B0A3
:10D2800001A9ADF804200222984703B05DF804FB21
:10D2900038480100F0B507468BB0002A33D0012A88
:10D2A00008BF0A2251B3212400E0F4B2B1FBF2F529
:10D2B00002FB1511C8B2092900F1300198BFC8B2AC
:10D2C0000AA988BF3730214488BFC0B201F8240CB6
:10D2D000661E2946002DE8D133B1013CE4B20AAB09
:10D2E00023442D2203F8242C3B6801AA11195B6802
:10D2F0003846C4F1220298470BB0F0BD30228DF8B9
:10D3000025202124E8E70368C9B21B6898470BB0C1
:10D31000F0BD00BF0029BABF49422D2300230A22D5
:10D32000FFF7B8BF374A384913681B06FCD40B68AF
:10D3300013F08003F8D172B634490A78002A5FD01E
:10D34000334A3448F0B4344C176806682568D4680A
:10D350000C303E44143200681268304F35442C447F
:10D3600020440244C2F34E022D4E2E482E4D2F4C27
:10D3700042F400423A60376806682D682C4A2468F7
:10D380000C303E44006812682A4F35442C44204437
:10D390000244C2F34E02284E2848294D294C42F43B
:10D3A00000423A60376806682D68274A24680C30C6
:10D3B0003E4400681268254F35442C442044024402
:10D3C000C2F34E02224E2348234D244C42F4004225
:10D3D0003A60376806682D68214A24680C303E445C
:10D3E0000068126835442C4420440244C2F34E02C3
:10D3F0001C4842F4004202600B7062B6F0BC7047F9
:10D4000062B6704724B0034024B00B4045A0FF1F14
:10D4100038B003403CB0034040B003402CB0034060
:10D4200058B003405CB0034060B0034064B00340B8
:10D430006CB0034030B0034038B00B403CB00B4000
:10D4400040B00B4044B00B404CB00B402CB00B40F4
:10D4500058B00B405CB00B4060B00B4064B00B4068
:10D460006CB00B4030B00B4030B42948294A2A4BED
:10D470002A4D6024E121047011701B78284C082B80
:10D4800030D00A2B2748284937D00C2B0CBF352227
:10D490003D2212232A60236002600B60234B244943
:10D4A0001B78244ABBB101230B601360224B234934
:10D4B0001B78234A012B26D9042B0FD9082B1ED900
:10D4C000102B94BF862387230B6013601D4B012212
:10D4D0001A7030BC70470B601360E7E784230B6061
:10D4E0001360F3E700F58E200F4908300122132363
:10D4F0002A60236002600B60D0E73922F7E78523BA
:10D500000B601360E2E780230B601360DEE700BF6F
:10D5100000400740014007405892FF1F08B00340F9
:10D520000CB0034008B00B400CB00B4048A0FF1FEC
:10D5300020B0034020B00B405992FF1F24B003409D
:10D5400024B00B4045A0FF1F0C2830B417D910237E
:10D55000984228BF18461C46104A114D1178181AD7
:10D560008C42287018D00F4913700B7823B10E49E4
:10D570000E4A00230B60136030BCFFF775BF0A280A
:10D5800002D90C231C46E7E7082802D90A231C46C7
:10D59000E2E708231C46DFE730BC70475892FF1FC4
:10D5A00044A0FF1F45A0FF1F24B0034024B00B4040
:10D5B00028282FD8334B2DE9F0411E5CFF2E2BD0AD
:10D5C000314B1B78002B2AD132062CD472B62F4D4A
:10D5D0002F4C2F46012326602B7062B672B623684B
:10D5E0001B060CD43B781BB9F4E72B78002BF1D049
:10D5F00062B602F09BF972B623681806F5D5254B82
:10D600001B6800222A7062B6234A107843FA00F0A1
:10D61000BDE8F081002070470020BDE8F081FFF7F1
:10D6200081FE3206D2D572B61C4DDFF87C801C4CD0
:10D6300006F04007FFB206F03F06D8F80030DFB131
:10D6400023F01003C8F8003001232660134A2B7022
:10D6500062B672B6236819060CD413781BB9ECE7CE
:10D660002B78002BE9D062B602F060F972B623681D
:10D670001B06F5D50B4BC3E743F01003C8F8003089
:10D68000E2E700BF3C48010045A0FF1F47A0FF1F85
:10D6900000B0034010B0034044A0FF1F46A0FF1F8E
:10D6A00000B00B4010B00B400CB00B400A4A0B49C5
:10D6B000136843F4805313600B7843B9084BC022BE
:10D6C0001A70084B80F30C0000B218807047044BAE
:10D6D00080221A70F5E700BF2C80044048A0FF1F8D
:10D6E00021C00C4000C00C40F0B51B4B1B4E5968CC
:10D6F00018689A68DB6885B06C460FC43378990760
:10D700001DD5174A174C1378174913F0700318BF2B
:10D710001370164A164B80271770002633200322F9
:10D7200026706D4608701A7072B6043C45F001050B
:10D730002046A84762B6237813F0700309D10D4B39
:10D74000064901E0013B02D00A78D207FAD505B0BC
:10D75000F0BD237005B0F0BD684801000100024033
:10D7600000000240040002400B000240070002409B
:10D770000A000240410D0300B0F5006F0AD210B557
:10D78000094B1B78DB07044606D504F1A05000784E
:10D79000C0B210BD00207047FFF7A6FF04F1A050F3
:10D7A0000078C0B210BD00BF01000240B0F5006FAC
:10D7B00017D238B50F4B1B78DA070D46044611D542
:10D7C00004F1A0500378AB420AD00B4A137813F04F
:10D7D000700318BF1370074A05701378DB07FCD578
:10D7E00038BD7047FFF780FF04F1A0500378AB42CB
:10D7F000EBD1F5E7010002400000024008B5F4F764
:10D8000043FAF5F709F902F091F8FAE7844641EA9C
:10D81000000313F003036DD1403A41D351F8043BA8
:10D8200040F8043B51F8043B40F8043B51F8043BFA
:10D8300040F8043B51F8043B40F8043B51F8043BEA
:10D8400040F8043B51F8043B40F8043B51F8043BDA
:10D8500040F8043B51F8043B40F8043B51F8043BCA
:10D8600040F8043B51F8043B40F8043B51F8043BBA
:10D8700040F8043B51F8043B40F8043B51F8043BAA
:10D8800040F8043B51F8043B40F8043B51F8043B9A
:10D8900040F8043B51F8043B40F8043B403ABDD209
:10D8A000303211D351F8043B40F8043B51F8043BAB
:10D8B00040F8043B51F8043B40F8043B51F8043B6A
:10D8C00040F8043B103AEDD20C3205D351F8043B3A
:10D8D00040F8043B043AF9D2043208D0D2071CBF06
:10D8E00011F8013B00F8013B01D30B88038060462F
:10D8F000704700BF082A13D38B078DD010F00303A5
:10D900008AD0C3F10403D21ADB071CBF11F8013B14
:10D9100000F8013B80D331F8023B20F8023B7BE763
:10D92000043AD9D3013A11F8013B00F8013BF9D28E
:10D930000B7803704B7843708B7883706046704728
:10D9400008B5104C08E0236859050DD423681A0562
:10D950000FD42368DB0411D423685803F3D500F0F7
:10D960008DFE23685905F1D502F044F823681A05A5
:10D97000EFD502F0D5F82368DB04EDD500F0F0FC1C
:10D98000EAE700BF3480044008B5FFF7D9FF00BFC5
:10D99000014B10221A80704700200540704700BFDD
:10D9A000094908B50B6830B16A461844A2F580529F
:10D9B000904202D20860184608BD03F063FB0C23B6
:10D9C00003604FF0FF3008BD5C92FF1FFEE700BF11
:10D9D000EFF3138070B9EFF310836BB9EFF30582A7
:10D9E0005AB94FF48070EFF311832BB1984228BFDE
:10D9F000184670474FF0FF3070470F2A01D818467D
:10DA0000F1E7014BD05CEEE7F0E300E0F0B44D1E2F
:10DA10002E46002400E00134B0FBF2F302FB1300B9
:10DA2000092800F130078ABF3730F8B2C0B206F8D3
:10DA3000010F1846002BEED10A1953704CB1107823
:10DA400015F8016F28700133E01A834202F801696A
:10DA5000F5DB0846F0BC7047704700BF10B40F4BB1
:10DA600053F8302092F880422CB1012369B182F83A
:10DA7000803010BC704703EBC0035B681A6841B983
:10DA800022F002021A6010BC704782F8003110BC0C
:10DA9000704742F003021A6010BC704778480100DA
:10DAA0001C4A02EBC00301295B6811D004291BD07A
:10DAB00052F83000002280F8802229B1022920D0BB
:10DAC000032922D01A6070474FF480721A607047A1
:10DAD00052F830004FF4A27280F880121A601A686F
:10DAE00022F020021A60704752F830104FF4A272F0
:10DAF000012081F880021A601A6842F020021A6040
:10DB0000704740F203121A6070474FF481721A6036
:10DB1000704700BF78480100212848D8F8B5042A8A
:10DB200044D8DFE802F0484B4E0345004FF410267E
:10DB30002B4B03EBC0030D465C68216811F4E061D8
:10DB400048D0284B284A2949C3F89C2104F1404277
:10DB50002748C3F8A411A2F59221264FC3F8A001CB
:10DB60007C292548C3F8A871C3F8AC012CD9A2F5CB
:10DB700094237C2B2AD9A2F596237C2B28D9A2F5B5
:10DB800098237C2B29D9A2F59A227C2A27D81B48D6
:10DB900072B6236823F4702343F08072C4F38401C7
:10DBA0001643236040F82150266062B6F8BD7047E6
:10DBB0004FF43026BCE74FF40026B9E74FF4402677
:10DBC000B6E74FF42026B3E70D48E1E70D48DFE75D
:10DBD0000D48DDE7FFF764FFB3E70C48D8E7F8BD71
:10DBE000784801000082FF1FF188FF1F9988FF1FFE
:10DBF000C588FF1F6D88FF1F4188FF1F3893FF1FD7
:10DC00006092FF1F9892FF1FE892FF1F1893FF1F5B
:10DC10001A4B03EBC00010B4426802F14043A3F575
:10DC200092217C2923D9A3F594217C290DD9A3F530
:10DC300096217C291FD9A3F598217C2919D9A3F510
:10DC40009A237C2B11D80E4C00E00E4C72B6136850
:10DC50000D4823F08773C2F3840123F4803343F02B
:10DC60008073136044F8210062B610BC7047074C03
:10DC7000ECE7074CEAE7074CE8E700BF784801000B
:10DC80003893FF1F9892FF1F59DA00006092FF1F20
:10DC90001893FF1FE892FF1F30B4054B054D064C4B
:10DCA000002210211A602A602060196030BC704781
:10DCB00014D0034004D0034000D00340282838B5D6
:10DCC0002ED0002904464FDD5F4B1B78012505FA55
:10DCD00003F28A4202D8212837D938BD0338C2B2AC
:10DCE000012A3AD9202C4AD0192C48D0574A126818
:10DCF00002FB011222FA03F31D2800F29B80DFE8E9
:10DD000000F0928B847D9999766F99999999999958
:10DD100099999968615A53994C9999999999994502
:10DD2000494B1B780B2B08D90C2B1CBF0C3B194102
:10DD30000846BDE83840FFF7B9BCC3F10C03994071
:10DD40000846BDE83840FFF7B1BC2946FFF786FE1C
:10DD50002946BDE83840FFF7A3BE3D4A126802FBE2
:10DD6000011222FA03F3C7E72128B6D80021FFF7F2
:10DD700075FE20460121BDE83840FFF791BE354AC7
:10DD8000126802FB011222FA03F3B5E73249334A63
:10DD90000B604FF45173136038BD3149314A0B6049
:10DDA0004FF45173136038BD2F49304A0B6040F275
:10DDB0004443136038BD2E492E4A0B6040F2444361
:10DDC000136038BD2C492D4A0B6040F24443136068
:10DDD00038BD2B492B4A0B6040F24443136038BDD9
:10DDE00029492A4A0B6040F24443136038BD284950
:10DDF000284A0B6040F24443136038BD2649274A45
:10DE00000B6040F24443136038BD2549254A0B603E
:10DE100040F24443136038BD2349244A0B604FF459
:10DE20005173136038BD2249224A0B604FF451737D
:10DE3000136038BD212C3FF650AF7F29D4BF00219D
:10DE40000121204693E700BF4093FF1F0880034055
:10DE50000890034008800B4010800B4048A004400D
:10DE600018800B404CA004401880034008B00440C8
:10DE70001080034004B004404080034018C00440B8
:10DE80003880034014C004402880034010B0044090
:10DE9000208003400CB004403080034010C0044098
:10DEA000488003401CC00440189003403490044054
:10DEB000109003403090044038B1102828BF102043
:10DEC000044AC3B2107813707047024A01231078D5
:10DED000137070474093FF1F2DE9F8430E468046AC
:10DEE0003249334D304603F053F847F612230028E9
:10DEF0001ABF1D464FF002094FF00109002425FA10
:10DF000004F002F04FFE4FF05E51074602F0A2FE11
:10DF10000146304603F050F830B90134072CEED1F9
:10DF2000E80902F03FFE07463146384602F046FF58
:10DF30004FF07C5102F084FD03F078F84FF6FF7249
:10DF40009042A8F1030328BF1046012B29D9B8F14C
:10DF5000170F17D8174B23FA08F303F0010383F0C8
:10DF6000010223B9B8F1190F0FD0BDE8F883124BA5
:10DF7000124D13491A6044EAC9042A6008601C6003
:10DF8000BDE8F883B8F1200FECD10E4B0E4D0F49D0
:10DF9000002244EAC9041A602A6008601C60BDE8D7
:10DFA000F8830B4B0B4D0C49F2E700BF001BB74049
:10DFB000006CDC026006F000008003400480034037
:10DFC0000880034000800B4004800B4008800B4019
:10DFD000009003400490034008900340212801D89A
:10DFE000FFF73CBD704700BF212806D8044B53F80B
:10DFF000303093F80002C0B270470020704700BF75
:10E0000078480100212801D8FFF74ABD704700BFBA
:10E0100072B60C490C4B0D4A1B680868126862B650
:10E02000520102D5322B88BF01300949C3F5BB33F9
:10E030004FF47A72FF33A1FB031302FB00F000EBF5
:10E04000931070474CA0FF1F18E000E004ED00E0C3
:10E05000ABAAAAAA2DE9F843054672B6204F214B78
:10E06000214A1B683C68126862B6520102D5322B05
:10E0700088BF013495B3C3F5BB331C4EDFF8649001
:10E08000DFF86480FF334FF47A72A6FB031302FBC0
:10E0900004F404EB931472B6D9F800103A68D8F877
:10E0A00000E062B6C1F5BB33FF33A6FB03031EF0ED
:10E0B000806FC4EB93134FF47A7002D0322988BF7B
:10E0C000013200FB0233B3F57A7F04D3013D05D062
:10E0D00004F57A74DFE701F029FCDCE7BDE8F8839A
:10E0E0004CA0FF1F18E000E004ED00E0ABAAAAAAD4
:10E0F000F8B52D4B2D49DFF8D0E0DFF8D0C02C4E1D
:10E100002C4D2D4C2D4A2E4F4FF4000018604FF02F
:10E11000807018604FF0007018604FF080601860D9
:10E120004FF0006018600020086028234BF6FF7154
:10E13000CCF80010CEF80030336013602B60236001
:10E140003B60B3629362092245F8242CC4F8D80FCF
:10E1500005F57F65C7F8D41F07F5FF2707F5FA67B0
:10E16000C6F8F83F2B6006F5FF26C4F8D42F05F556
:10E17000FD2504F5FF24386006F2F476114831607D
:10E1800005F5FF6504F5FD642B6023600260FFF771
:10E190006BF91920FFF75EFF00F0B6FF40F2131095
:10E1A000BDE8F840FFF756BF08E100E004800340F7
:10E1B00014800340248003402C8003401C800340D3
:10E1C0003480034000800B400C80034008800340F3
:10E1D0002DE9F84F214B1B6807460BB101221A703D
:10E1E000DFF888901E4D99F80040DFF884801D4EBE
:10E1F0000134272C8ABF4FF0000A5FFA84FA544694
:10E20000AB462B78A34216D1FFF7E2FB40281FDC78
:10E2100033791B06F5D59BF800300133272B86BFD9
:10E2200000221346DAB218F80330DBB2F3712A7019
:10E230002B78A342E8D00C490A4BFFB208F80470CF
:10E240000120AC22087089F800A0DA70BDE8F88FD0
:10E25000FF28D6DD01F06AFBD3E700BFC4A0FF1F93
:10E26000C1A0FF1F00C00640C0A0FF1FC8A0FF1F25
:10E2700058A0FF1F1C4BDFF894C01A681B49F0B56B
:10E2800042F480521A4D1A60DFF884E0194F1A4E9A
:10E290001A4C00238CF800304FF451722B701F2859
:10E2A00040F213358EF800303B70337025600A6001
:10E2B00012D819460124124A124D11701248547096
:10E2C00000212C27402693724FF400349170117472
:10E2D000D7702E700460F0BDC0F34431C0F3471412
:10E2E00000F01F03E7E700BF348004400CC0044087
:10E2F00055A0FF1FC1A0FF1FC0A0FF1F08C0044002
:10E3000000C0064031E400E004E100E054A0FF1F3B
:10E31000C8A0FF1F034B1B68DB0401D5FFF758BFE4
:10E32000704700BF3480044010B5044C237823B1FB
:10E3300001F0FCFA2378002BFAD110BDC0A0FF1F1A
:10E34000054A064B10781B78C0B2DBB2984238BF42
:10E350004030C01A704700BF54A0FF1F55A0FF1FD8
:10E3600030B42B4B1A7994061FD52A48DA790378F2
:10E37000294901333F2B0978C8BF00238B42D2B211
:10E3800003D0264CD9B2E2540170254A116861B11C
:10E39000244A1278D2B2934236BFC2F140029B1A8D
:10E3A0009B18272BC4BF01230B70194AD378DBB20B
:10E3B000180611D45A060DD5154B1B795B0609D5E5
:10E3C000194B1A491B6800220A7003B11A70104BCE
:10E3D0002C22DA7030BC704711790906EAD514494D
:10E3E00010480C780178C9B28C420DD04A1C272AFB
:10E3F00084BF00210A460F4D054C98BFD1B2AA5CDC
:10E40000D2B2E2710170D5E76C21D170D2E700BFC2
:10E4100000C0064054A0FF1F55A0FF1F80A0FF1F93
:10E4200050A0FF1FC1A0FF1FC4A0FF1FC0A0FF1F5F
:10E43000C8A0FF1F58A0FF1F21282FD8184B195C18
:10E44000FF292BD0174B184ADFF870C003EBC00030
:10E45000F0B54368DFF868E0144F154D154E002401
:10E460001C60DEF80030012043F020038840CEF825
:10E47000003014604FF4A07338602E60C2F800C002
:10E48000013BFDD113689B05FCD42023013BFDD14A
:10E49000094B09B233F8110080B2F0BD002070477B
:10E4A00088490100784801000050044008500440A9
:10E4B00004500440000002030051044080014A005F
:10E4C00038800440431E032B14D872B60A4951F811
:10E4D000230068B170B4094C058834F813204668ED
:10E4E00041F82360521B24F8132062B670BC7047B9
:10E4F00062B670470020704724A1FF1F68A3FF1F6A
:10E50000013803280BD872B6074B53F8203043B1BB
:10E5100000205B680130002BFBD162B67047002001
:10E5200070471846F9E700BF78A1FF1F30B472B6F4
:10E530002B4A13781D0706D52A4B196A002936D0B5
:10E54000996A002941D053781C0706D5254B196CD0
:10E5500000293ED0996C002939D09378190705D548
:10E56000204B196E002936D0996E89B1D3781B07DC
:10E5700007D51C4BD3F880207AB3D3F8882011211B
:10E580003AB162B6184B00221A7030BC00F04ABE95
:10E590000D21154C154D227843F8315003EBC10382
:10E5A0000830013A5860227062B630BC70470422CD
:10E5B0000D4C0F4D217843F8325003EBC203083065
:10E5C0004A1E5860227062B6EFE70521E1E7092193
:10E5D000DFE70822ECE70C22EAE71022E8E700BFB9
:10E5E000AC4901000080FF1FA1A1FF1FC80040002F
:10E5F00088004000431E032B1DD81B4A400140F0F9
:10E60000100030B4104472B6184CE25C032A1BD8D8
:10E61000DFE802F00212151703220D88E25410F011
:10E62000080F14BFC823882343EA05430831036059
:10E63000416062B630BC704708300222EDE7052227
:10E64000EBE708300422E8E7094A52F8230038B122
:10E65000084A52F82300416042F8231062B6E9E705
:10E6600042F82310034AF7E70080FF1FB0A1FF1F05
:10E6700078A1FF1F88A1FF1F00BE70472DE9F04F52
:10E68000DFF818B3DFF818A387B044E0AD4F4FEAC6
:10E69000930807EBC809013ED9F8042003F00803EA
:10E6A000F6B2A2F1080003F0FF04002B40F0018154
:10E6B00057F838301B0C99B222F8081C002B00F0D8
:10E6C000EF80A14B22F8064C42F8044C53F8262068
:10E6D000002A00F0CF819D4D55F8263058609C4CA3
:10E6E00045F8260034F81630194424F8161000F0C6
:10E6F00079FD002800F0C281964A974B19F0080F67
:10E7000000F1080018BF1346C9F8040047F8383074
:10E7100008238BF800309BF80040E4B265071CD555
:10E720008E4B1B78B3B18E490A7802F0FF0322B1F9
:10E73000013BDBB20B7003B900BE8A490A7802F0D4
:10E74000FF032AB1013BDBB20B70002B00F06881A4
:10E7500000F066FE04238BF8003004F0080303F099
:10E76000FF02002B00F0C9809AF80030DBB21E09CE
:10E770008CD19A08DFF8CC9159F8321009EBC2001D
:10E78000C1F38301013940680C2900F28580DFE87C
:10E7900001F07A7A838383838383468383830700AC
:10E7A0000168714D4068714F714E6860296088B290
:10E7B00040F281610024674B49F832304FF0010E7E
:10E7C00088423C60C9F81040C9F8184086F800E05B
:10E7D0005C4A00F2E780B0F5D06F80F01B82B0F5A4
:10E7E000817F00F0D98100F26981802800F02A82BF
:10E7F000822840F0D781A98801F07F01042900F226
:10E80000D1815C485C4A89000844147054700178D6
:10E810008C0740F1608382F800E0022173E1534FDE
:10E820003A682AB3554B524E5548198834780578C2
:10E8300040298E4645F0020828BF4FF0400E002CBC
:10E8400084F001043470CEEB01010CBF8824C8248D
:10E8500009EBC80689B285F0010544EA0E447260EE
:10E86000198049F8384072440570002965D03A6033
:10E870003D4B1A88B2F5A06F0ED100219A785970DD
:10E88000404B1A7008E038493F4C0D68A54200F033
:10E890009880304949F832103C4A0123137037E719
:10E8A0002C4A2D4B19F0080F18BF134647F8383083
:10E8B0002EE700F0B7FC364A364952F82630002BD6
:10E8C00000F0E38058688C5D42F8260003F10802EE
:10E8D000C9F80420032C05D8DFE804F02C0229260F
:10E8E00002228A551A8819F0080F0CBF8823C82302
:10E8F00043EA024347F838300AE7E00700F1938023
:10E90000210600F1D180A20706D5234A23491378B6
:10E910000220DBB213700870E30602D51F4B1022F1
:10E920001A7007B0BDE8F08F04228A55DAE7052295
:10E930008A55D7E703228A55D4E7BEF1400F18BFA6
:10E94000002294E70080FF1F24A1FF1FD0A0FF1F1B
:10E9500068A3FF1FC800400088004000ACA1FF1F53
:10E9600035A1FF1F20A2FF1F98A1FF1FCCA0FF1FF2
:10E9700034A1FF1FC0200740A4A1FF1FE0A0FF1F7C
:10E98000A0A1FF1F98200740210900039420074001
:10E9900078A1FF1FB0A1FF1F8820074080200740FB
:10E9A00090200740B0F5106F00F07C8140F2A3800A
:10E9B00040F62112904240F07B82A54A0123137059
:10E9C0006AE74C68A3498C427FF463AF0178A929B8
:10E9D0007FF45FAF417845297FF45BAF8178C2292E
:10E9E0007FF457AFC1786B297FF453AF9A489B4EA1
:10E9F0000178347881F00105002C41F002010570A6
:10EA00000CBF8820C82084F0010449F8310009EBCC
:10EA1000C10193483470002505244D60047038E727
:10EA200000F064FF94E68F4B89488B491A614FF0E0
:10EA3000020E80F800E08C4F0A708C4919609960D2
:10EA40008B4E8C4D8C4C9A610D213970FF213170A9
:10EA5000DFF84CE229702270884D894A8EF8001048
:10EA60009F27012406F8047C5D600470DA6007B01B
:10EA7000BDE8F08F43F82600824D30E6824A47F821
:10EA8000380013780133137042E68B5D032B00F2DC
:10EA9000BA8001A252F823F011E7000011E700004C
:10EAA000F1EA0000EBEA00006F49724B80220D2072
:10EAB00008701A70A2077FF52FAF26E740F20232E6
:10EAC000904240F0ED81AA8802F07F02042A69D8C2
:10EAD0006D88002D66D16449CDF804E092001144A0
:10EAE0000A7842F002020A70C1E101238B550FE659
:10EAF00000238B550CE6B0F5086F53D16349644A87
:10EB0000097811707146ED888D4280F0E882524894
:10EB10000478402DAE4644F0020C28BF4FF0400E62
:10EB200002EB0E0309EBCC01029301234A604FEA8A
:10EB30000E48CEEB050101930025C82242EA0803E6
:10EB400084F0010249F83C3035700270DFF814C1DE
:10EB5000424BDFF8048149BBBEF1400F7FF42DAF7B
:10EB600042F0020C09EBCC03029ADFF8F8E05A609D
:10EB70008DBB0D0445F088059DF804304EF83C50DF
:10EB80000A4433700470134640297FF416AF002105
:10EB9000404A3B60118010E7AA8802F07F02042AF5
:10EBA00040F28B81304A0F23137006E74029D7D9F2
:10EBB00042F002020CEBC200029E4660BDB19DF81D
:10EBC000045035481D703346403988F800404033C2
:10EBD0004CF83200DCE79DF8043033700D04029BE2
:10EBE000047045F0C8050B444EF83C50CCE79DF846
:10EBF00004501D70029B1D4888F800404039403386
:10EC00004CF83200C4E719F0080F0CBF02230323AD
:10EC10008B557DE521494A68002AC3D06C88B5F838
:10EC200004E003E00C314A68002ABBD00B88A34201
:10EC3000F8D14B887345F5D1240A032C0CBF117809
:10EC4000098960E7124A0221147054705BE700BF23
:10EC50009420074001000400A0A1FF1F34A1FF1F62
:10EC600035A1FF1F0080FF1FC02007408800400023
:10EC7000882007408020074098200740E4A0FF1F1D
:10EC800038A1FF1FD0A0FF1FA1A1FF1FACA1FF1F34
:10EC9000A4A1FF1FE0A0FF1FC8004000B049010071
:10ECA0008C200740B248116AAC7804700C0600F161
:10ECB0009881D9F82820AF49100600F1DB81D9F8F6
:10ECC0003020AC49120600F1D081D9F83820A9498A
:10ECD000130600F1C581D9F84020A649150600F1B8
:10ECE000BA81D9F84820A349140600F1AF81D9F8B8
:10ECF0005020A049100600F1A481D9F858209D4960
:10ED0000120600F19981D9F860209A49130600F1A2
:10ED10008E81D9F868209749150600F18381D9F8CA
:10ED200070209449140600F17881D9F8782091492F
:10ED3000100600F16D81D9F880208E49120600F18D
:10ED40006181D9F888208B49130600F15581D9F8E3
:10ED500090208849150600F14981D9F89820854905
:10ED6000140600F1FF808448844A85490190854853
:10ED7000854D864C049700230596029580460F46E4
:10ED800016461D460394306828B1446800F04AFADC
:10ED90002046002CF9D100233360029B38681A46C4
:10EDA000002342F8253028B1446800F03BFA2046A1
:10EDB000002CF9D100223A60019A98F800301146EF
:10EDC000002241F8042B039A0191023B4FF000010D
:10EDD00022F81510032B07D8DFE803F05D025D026F
:10EDE0004FF0010388F800300135042D06F10406C8
:10EDF00007F1040708F10108C5D1654C654D22787B
:10EE0000654B049F059E0021100729701A7000F1C0
:10EE10009280624962780A700021C9F83010C9F8FE
:10EE200038101107DFF84C816ED4A2785C49DFF806
:10EE300044810A7000211207C9F85010C9F858100F
:10EE40004BD4E27857494B4C0A7013074FF000013E
:10EE5000C9F87010C9F8781000F1AE8033780193CA
:10EE6000002283F00105C9F89020C9F898200021FC
:10EE7000029188468E460A464B48047844F0020CBC
:10EE800009EBCC030393019B002B039B5A600CBF3F
:10EE90008822C82252E64FF0000388F80030A3E72A
:10EEA000B0F5A06F7FF47EAE012300250193DEE76D
:10EEB00040F621229042F7D074E66D88002D7FF451
:10EEC00071AE3A49CDF804E0920011440A7822F07C
:10EED00002020A70CBE7022115E600F083F9002850
:10EEE00000F0EB800830324AC8F86400C8F86020AF
:10EEF00000F078F9002800F0DA8008302D4AC9F8CF
:10EF00006C00C9F868209CE700F06CF9002800F05C
:10EF1000E0800830264AC8F84400C8F8402000F0D5
:10EF200061F9002800F0CF800830224AC9F84C006F
:10EF3000C9F8482079E700F055F9002800F0A580CD
:10EF400008301B4AC9F82400C9F8202000F04AF90B
:10EF5000002800F094800830164AC9F82C00C9F83F
:10EF6000282056E7D1F89C00083800F05BF9FAE653
:10EF7000ACA1FF1F0080FF1F88A1FF1F24A1FF1F5E
:10EF800078A1FF1FB0A1FF1FD0A0FF1F68A3FF1F24
:10EF9000AC490100A1A1FF1FC4200740C8200740C1
:10EFA000CC200740D0200740A0A1FF1FC020074071
:10EFB00088004000C800400000F014F9002870D01C
:10EFC00008304F4AC4F88400C4F8802000F00AF9E1
:10EFD000002860D008304B4AC9F88C00C9F8882056
:10EFE0003CE7506A083800F01DF962E6D1F8940059
:10EFF000083800F017F9B0E6D1F88C00083800F0B6
:10F0000011F9A4E6D1F88400083800F00BF998E66D
:10F01000C86F083800F006F98DE6486F083800F030
:10F0200001F982E6C86E083800F0FCF877E6486E11
:10F03000083800F0F7F86CE6C86D083800F0F2F810
:10F0400061E6486D083800F0EDF856E6C86C0838FF
:10F0500000F0E8F84BE6486C083800F0E3F840E6CA
:10F06000C86B083800F0DEF835E6486B083800F069
:10F07000D9F82AE6C86A083800F0D4F81FE62A78DA
:10F08000C9F8280001322A70C3E62A78C9F820009E
:10F0900001322A705AE72A78C9F8880001322A70AA
:10F0A000DCE62A78C4F8800001322A708EE72A78DC
:10F0B000C9F8680001322A70C3E62A78C8F86000EF
:10F0C00001322A7014E72A78C9F8480001322A7000
:10F0D000ABE62A78C8F8400001322A701FE74029C1
:10F0E0008E4628BF4FF0400E02EB0E030293012321
:10F0F000CEEB01014FEA0E4800250193BCE600BFAC
:10F1000088004000C8004000F8B500F08FFD294B92
:10F1100029482A4C2A4F2B4DDFF8BCC0DFF8BCE051
:10F12000294E00221A605A609A60DA601A615A61A8
:10F130009A61DA611A625A629A62DA621A635A63EF
:10F140009A63DA631A645A649A64DA641A655A65CF
:10F150009A65DA651A665A669A66DA661A675A67AF
:10F160009A67DA67C3F880200168C3F8842041F405
:10F1700080210160C3F307212170C3F307401349C5
:10F1800038701B0E2B70FF238CF80030104D8EF85A
:10F19000003010480B700123337084F8642070260F
:10F1A0004FF40074102207F82C3C2E70046081F894
:10F1B000F820F8BD0080FF1F348004409C200740E9
:10F1C000B0200740B420074094200740102007409B
:10F1D00049E400E008E100E0802007408820074083
:10F1E000704700BF72B60D480268B2FA82F30F2B67
:10F1F00010DC4FF00041D94022EA0102026062B601
:10F20000074803EBC303DB00C2180021C1501046BE
:10F210005160704762B60020704700BF4493FF1FE3
:10F22000BC83FF1F0D4B0E4AC31AA2FB03231B090D
:10F230000F2B0CD80B4A127852B972B60A484FF00D
:10F240000041026821FA03F31A43026062B6704774
:10F25000064A1278002AF0D0FFF768B9BC83FF1F76
:10F26000398EE338A1A1FF1F4493FF1FACA1FF1FFC
:10F2700038B50E4B0E4C1B68218805468BB1B1F595
:10F28000917F05D20B4A4B1C55549BB2238038BD4D
:10F290000022084898470021064A5554012323803C
:10F2A00038BDB1F5917FEDD338BD00BFD8A1FF1FA8
:10F2B00072A3FF1F78A3FF1F2DE9F843214E224FB1
:10F2C0003168012380463B70B1B1204D4B8801EB82
:10F2D0008302013300240F2BC2F808802C7004D85D
:10F2E0004B8000233B70BDE8F88340230B80032054
:10F2F000FFF780F93460F4E7DFF8549099F80030B4
:10F30000002BF0D0114D45F6215408E0013C12D0FD
:10F310002B7883B900F00AFB99F800307BB1032009
:10F32000FFF7EEF80528F1D8FFF75CFF01463060E3
:10F330000028EBD0CAE701232B70BDE8F883BDE8B5
:10F34000F88300BFF4A1FF1FC8A1FF1FF8A1FF1F92
:10F35000ACA1FF1F1201F8B5D5B2A1B3012943D06A
:10F360004378044600781B0643EA004040F47040AE
:10F3700045F004068F1E3043FFF79EFF022F04F175
:10F38000020314D9053414F8023C14F8032C14F8C1
:10F39000010C1B0443EA0223334343EA0060033FAA
:10F3A000FFF78AFF022F234604F10304EBD8022F54
:10F3B00023D0012F0DD045F4774040F00500BDE883
:10F3C000F840FFF779BF14482843BDE8F840FFF73D
:10F3D00073BF187845F4770545F0060545EA002027
:10F3E000BDE8F840FFF768BF03780C4845EA0345DD
:10F3F0002843BDE8F840FFF75FBF1A78587845F01A
:10F40000774545F0070545EA022545EA0040BDE895
:10F41000F840FFF751BF00BF06F0F70007F000F714
:10F4200038B5084B1C7824B9074D296809B14B88B9
:10F4300003B938BD9B000B800320FFF7DBF82C607D
:10F4400038BD00BFC8A1FF1FF4A1FF1F2DE9F04187
:10F45000AD4E33680746002B00F092801D885A8815
:10F46000910803EB81010432AA428C6842D25A808F
:10F4700004F00F064FEA1428A449A6F1080208F088
:10F480000F00C4F30313062A00F101050B701AD90B
:10F49000B31E012B5FFA88F04ED9052E48D0042EFA
:10F4A00000F0A481731F022B7FD90F2E0ED1F728F5
:10F4B00042D8F02802D0964B1B883BB1FFF7D8FE0C
:10F4C0000020BDE8F08127B1BD4202D00020BDE898
:10F4D000F081082EC4F3033300F08780092E11D089
:10F4E0000A2E40F094800A2BF0D18A4B8A4A1B687E
:10F4F000A02181E01846FFF795FE0420FEF7E2FF09
:10F500003060B5E7092BE1D1270E00F07B81834BFA
:10F51000814A1B689021C4F307461170EDB2FCB21A
:10F52000002B00F09D80224631462846984797E000
:10F53000F02843D9F72841D0F1380E28C6D801A3C6
:10F5400053F820F0FBF60000DFF60000CDF60000D7
:10F55000CDF40000CDF40000BFF60000CDF40000B3
:10F560009FF70000CDF4000069F7000083F700006A
:10F57000A7F60000CDF400008FF6000073F600003F
:10F58000674B1B78002BA1D00420FEF79BFF03469E
:10F59000306000289AD00588002D7FF460AFFFF717
:10F5A00041FE35602846BDE8F081FFF761FEC4F3F7
:10F5B0000740FFF75DFE072E02D1200EFFF758FE31
:10F5C000534B584A198858481468584D524A01708C
:10F5D00000270E0AF0201F802E7010700CB301223D
:10F5E0005348A0470120BDE8F081082B7FF46EAF9F
:10F5F000504B494A1B688021C4F307461170EDB295
:10F60000240E6BB3284622463146984728E00B2E3D
:10F6100011D10B2B7FF45AAF474B3F4A1B68B021E7
:10F62000EAE7464B1B68002B00F0FB8040489847F8
:10F630000120BDE8F0810C2E40F000810C2B7FF4FE
:10F6400045AF3F4B344A1B68C0211170EDB2C4F383
:10F650000746002B00F0C88028463146240E984704
:10F660003849314A314B0D7016701C700120BDE8CD
:10F67000F081354B1B68002B00F0D6809847C4F30F
:10F680000746254BEDB2240E83F80080E8E72F4BA8
:10F690001B68002BF2D12E4B1B68A3B1FE209847AC
:10F6A000C4F30746EDE72B4B1B68002BE6D1284B34
:10F6B0001B6843B1FC209847C4F30746E1E7264B9B
:10F6C0001B68002BDAD1C4F30746DAE7234B1B682B
:10F6D000C4F30746002BD4D030469847D1E7204BDF
:10F6E0001A68002AEFD0260C630C06F07F0003F4A2
:10F6F0007E531843F6B29047C3E71A4B1B68C4F316
:10F700000746002BE8D1BCE700A2FF1F76A3FF1F2E
:10F7100072A3FF1FDCA1FF1F70A3FF1F10A2FF1F1A
:10F72000ACA1FF1FD8A1FF1F74A3FF1F75A3FF1F6C
:10F7300078A3FF1F08A2FF1F0CA2FF1FF0A1FF1F4D
:10F74000CCA1FF1F77A3FF1FB8A1FF1FBCA1FF1F04
:10F75000C0A1FF1FFCA1FF1FECA1FF1F04A2FF1F00
:10F76000D4A1FF1FE8A1FF1F3F4B1B68002B85D1D1
:10F770003E4B1B68002BA6D0FA209847C4F30746DF
:10F780007FE73B4B1B68002B7FF478AF374B1B6840
:10F79000002B98D0FB209847C4F3074671E7354B00
:10F7A0001B68002B7FF46AAF304B1B68002B8AD09C
:10F7B000F8209847C4F3074663E70E2B7FF486AE24
:10F7C0002D4A2E4B1268E0211970002A47D0260CD2
:10F7D000610C06F07F0301F47E511943EDB2A1F5EF
:10F7E000005128469047F6B2240E39E7FFF740FD56
:10F7F000C4F30740FFF73CFD200EFFF739FD002062
:10F80000BDE8F0811E4B1D4A1B6880211170EDB2CE
:10F81000C4F3074683B1314628463A4698473C46EA
:10F820001EE70120BDE8F081104B1B68002B3FF460
:10F830004AAFFF20984746E71C4611E70D2EBCD182
:10F840000D2B7FF443AE0F4B0C4A1B68D021117077
:10F85000EDB2C4F30746002B7FF4FEAEC4E7C4F359
:10F860000746EDB2240EFBE6E4A1FF1FC0A1FF1F77
:10F87000C4A1FF1FB4A1FF1FD0A1FF1F70A3FF1FD2
:10F8800008A2FF1FE0A1FF1F38B5164D2868E0B1A0
:10F8900001884488A14213DD03191B7A83B104F166
:10F8A0000803C2180C1B002302E012F8011F21B14B
:10F8B0000133A342F9D1204638BD1C46204638BD4D
:10F8C000FFF7B0FC0020286038BD074B1B780BB950
:10F8D000002038BD0220FEF7F5FD28600028D7D1B2
:10F8E000F6E700BF1CA2FF1FACA1FF1F0D4B1B784A
:10F8F000BBB910B50C4C216803F0FF024B883F2BBD
:10F9000007DC07330B4401F1470003F8012F834262
:10F91000FBD140230B800120FEF76CFE0023236007
:10F9200010BD704714A2FF1F18A2FF1F38B5224C4C
:10F93000237803B138BD01232370FFF7A5FF70BB07
:10F9400000F048F840BB00F0DBF810BBFEF7F8FC15
:10F95000E0B900232370EFF30583002BEAD1EFF326
:10F96000108172B6154B1868E0B1154C2278CAB9EF
:10F9700045691D6001232370C5B1AA6101B962B652
:10F9800000254577836898472570D3E700F020F875
:10F99000DFE700F01BF8D9E700F016F8D3E7FFF730
:10F9A0001FFCCDE70029C5D162B638BD054B1D60EF
:10F9B0000029E5D1E3E700BF21A2FF1F38A0FF1F08
:10F9C0003CA0FF1F34A0FF1F704700BF704700BF5F
:10F9D000704700BF054A064B10781B78C0B2DBB2F7
:10F9E000984238BF4030C01A704700BF28A2FF1F9E
:10F9F00029A2FF1FF0B4384B1A7912F0300F2CD027
:10FA000072B6997D01F0FF0200293DD062B6334FF6
:10FA1000334938780D78334E1C46C0B2EDB2431CE2
:10FA2000402BE17928BF0023AB4202F1FF32C9B27B
:10FA30001CBFF154184612F0FF02F0D12A4B1B688C
:10FA4000C2B23A704BB1A84236BFC5F14005401B67
:10FA500040192728C4BF01221A701F49CA78D2B2A0
:10FA6000150616D452060DD51B4B1B795B0609D51E
:10FA70001E4B1F491B6800220A7003B11A70164BF7
:10FA80003C22DA70F0BC70474022D9795A7462B6D1
:10FA9000E3E70B791C06E5D5164B174E1C78337837
:10FAA000E4B2DBB29C420ED0144D01E0A3420AD076
:10FAB0000133402B28BF00230879E85CC0B2C8712D
:10FAC000087D0728F2D9DBB2034933700B79180699
:10FAD00044BF7C23CB70C5E700A0064028A2FF1FCF
:10FAE00029A2FF1F6CA2FF1F24A2FF1FB0A2FF1FAD
:10FAF000ACA2FF1FB4A2FF1FADA2FF1F2CA2FF1FCD
:10FB0000054A064B10781B78C0B2DBB2984238BF6A
:10FB10004030C01A704700BF28A3FF1FBDA2FF1FBF
:10FB2000F0B4384B1A7912F0300F2CD072B6997DA0
:10FB300001F0FF0200293DD062B6334F33493878D7
:10FB40000D78334E1C46C0B2EDB2431C402BE17918
:10FB500028BF0023AB4202F1FF32C9B21CBFF154EF
:10FB6000184612F0FF02F0D12A4B1B68C2B23A705D
:10FB70004BB1A84236BFC5F14005401B40192728AC
:10FB8000C4BF01221A701F49CA78D2B2150616D412
:10FB900052060DD51B4B1B795B0609D51E4B1F4921
:10FBA0001B6800220A7003B11A70164B3C22DA70EF
:10FBB000F0BC70474022D9795A7462B6E3E70B79FA
:10FBC0001C06E5D5164B174E1C783378E4B2DBB231
:10FBD0009C420ED0144D01E0A3420AD00133282BE1
:10FBE00028BF00230879E85CC0B2C871087D0728E7
:10FBF000F2D9DBB2034933700B79180644BF7C237A
:10FC0000CB70C5E700B0064028A3FF1FBDA2FF1FB1
:10FC1000E8A2FF1FB8A2FF1F2CA3FF1FBCA2FF1F5B
:10FC200030A3FF1F29A3FF1FC0A2FF1F70B584B020
:10FC300072B6194B194D1A48702241260F248021A3
:10FC40001A702E701A460470197013781B06FCD5B2
:10FC5000144B186862B6144B144C984298BF00EBD2
:10FC6000800001A998BF40000A22FDF7CFFE01A93C
:10FC70002046002311F8012B01333AB10A2B20F85A
:10FC8000022FF7D11623237004B070BD5B00DBB2E6
:10FC9000237004B070BD00BF0000024007000240A6
:10FCA00006000240080002407F9698001094FF1F53
:10FCB0002DE9F043DFF8EC808BB006460F4600F0EC
:10FCC00073F898F90030013304460D4637D03046BA
:10FCD000394600F0DFF9002831D02BA3D3E9002307
:10FCE0003046394600F026FE814668BB28A3D3E99A
:10FCF00000233046394600F0FFFD00B398F900308C
:10FD0000254ACDF82090042400200021022BCDE9C3
:10FD10000467CDE9026700940192CDE906012CD079
:10FD2000684600F0BDF940B3089B1BB101F0AAF989
:10FD3000089B0360DDE906010BB0BDE8F0832046B7
:10FD400029460BB0BDE8F083134A98F900300192C0
:10FD500003210022CDE90467CDE9026700910892F2
:10FD60002BB90E4B4FF06042CDE90623D8E70C4982
:10FD70000020022BCDE90601D2D101F083F9222324
:10FD80000360D1E7AFF30080EF39FAFE422E8640E0
:10FD900051302DD5104987C01C4A0100FFFFEF47A5
:10FDA0000000F07F2694FF1F2DE9F04FB04F21F0A7
:10FDB0000042BA4283B00C464FEAD17605460DD9CF
:10FDC000AC4FBA4225D9C1F31303034340F0EF808F
:10FDD0000EB10020014603B0BDE8F08FA64B9A4259
:10FDE00000F2CC80A54B9A4200F2DE808AA3D3E9D0
:10FDF000002300F05DF90022A14B00F09BFD0028DC
:10FE000000F005812846214600229D4B00F050F964
:10FE1000E1E783A3D3E9002300F08CFD002840F044
:10FE2000CB802846214680A3D3E9002300F064FD5F
:10FE30000028CED1934B284603EBC60821467CA36D
:10FE4000D3E9002300F0E6FAD8E9002300F030F906
:10FE500000F07AFD804600F077FA77A3D3E900231B
:10FE600006460F4600F0D6FA02460B4628462146C3
:10FE700000F01CF972A3D3E90023CDE9000130465C
:10FE8000394600F0C7FA82468B4652465B46DDE9AA
:10FE9000000100F00BF905460C462A462346284689
:10FEA000214600F0B7FA68A3D3E9002306460F46BF
:10FEB00000F0B0FA66A3D3E9002300F0F7F8324669
:10FEC0003B4600F0A7FA64A3D3E9002300F0F0F862
:10FED00032463B4600F09EFA61A3D3E9002300F0CE
:10FEE000E5F832463B4600F095FA5FA3D3E90023DC
:10FEF00000F0DEF832463B4600F08CFA02460B4634
:10FF00002846214600F0D2F806460F4628462146EC
:10FF100032463B46B8F1000F56D000F07BFA32462D
:10FF200004460D463B4600204FF0804100F0BEF8ED
:10FF300002460B462046294600F096FB02460B4639
:10FF40005046594600F0B2F8DDE9002300F0AEF863
:10FF50000B4602464A49002000F0A8F86FF47F7370
:10FF600098454FDA08F57A7801EB085100224FF0F6
:10FF7000B87300F04FFA03B0BDE8F08F424B9A42DD
:10FF80003FF658AF414BF4002344D3E9002300F07F
:10FF90008DF83F4BC6F101081C44CDE90001D4E9BE
:10FFA00000ABC6EB080870E74FF0000875E70246A3
:10FFB0000B4600F07DF80EE717A3D3E900231046A7
:10FFC000194600F027FA06E700F024FA00228046DE
:10FFD00089464FF080433046394600F067F80246C4
:10FFE0000B464046494600F03FFB2A46234600F0B8
:10FFF0005DF802460B460020214900F057F803B097
:020000021000EC
:10000000BDE8F08F01EB085103B0BDE8F08F8046EA
:1000100043E700BFAFF300809C7500883CE4377E67
:10002000EF39FAFE422E864051302DD5104987C057
:10003000FE822B654715F73F0000E0FE422EE63FAB
:10004000763C7935EF39EA3DD0A4BE726937663E19
:10005000F16BD2C541BDBB3E2CDE25AF6A56113FC8
:1000600093BDBE166CC1663F3E5555555555C53FAF
:10007000412E8640FFFFEF7F422ED63FFFFF2F3EEF
:100080000000F03F204A0100B1A2F03F404A0100C9
:10009000304A010041F0004101F58010C00F704767
:1000A0000020704781F0004102E000BF83F0004370
:1000B00030B54FEA41044FEA430594EA050F08BF03
:1000C00090EA020F1FBF54EA000C55EA020C7FEAC7
:1000D000645C7FEA655C00F0E2804FEA5454D4EB44
:1000E0005555B8BF6D420CDD2C4480EA020281EA0E
:1000F000030382EA000083EA010180EA020281EA46
:100100000303362D88BF30BD11F0004F4FEA013197
:100110004FF4801C4CEA113102D0404261EB4101A6
:1001200013F0004F4FEA03334CEA133302D052422C
:1001300063EB430394EA050F00F0A780A4F10104E8
:10014000D5F1200E0DDB02FA0EFC22FA05F2801822
:1001500041F1000103FA0EF2801843FA05F3594108
:100160000EE0A5F120050EF1200E012A03FA0EFC87
:1001700028BF4CF0020C43FA05F3C01851EBE371B1
:1001800001F0004507D54FF0000EDCF1000C7EEBCE
:1001900000006EEB0101B1F5801F1BD3B1F5001F0C
:1001A0000CD349085FEA30004FEA3C0C04F101042B
:1001B0004FEA445212F5800F80F09A80BCF1004F54
:1001C00008BF5FEA500C50F1000041EB045141EAD6
:1001D000050130BD5FEA4C0C404141EB010111F4D7
:1001E000801FA4F10104E9D191F0000F04BF014682
:1001F0000020B1FA81F308BF2033A3F10B03B3F160
:1002000020020CDA0C3208DD02F1140CC2F10C02EF
:1002100001FA0CF021FA02F10CE002F11402D8BF4D
:10022000C2F1200C01FA02F120FA0CFCDCBF41EA19
:100230000C019040E41AA2BF01EB0451294330BDE8
:100240006FEA04041F3C1CDA0C340EDC04F11404C5
:10025000C4F1200220FA04F001FA02F340EA03009C
:1002600021FA04F345EA030130BDC4F10C04C4F1E2
:10027000200220FA02F001FA04F340EA03002946C2
:1002800030BD21FA04F0294630BD94F0000F83F40C
:10029000801306BF81F480110134013D4EE77FEAEF
:1002A000645C18BF7FEA655C29D094EA050F08BF3B
:1002B00090EA020F05D054EA000C04BF194610461C
:1002C00030BD91EA030F1EBF0021002030BD5FEA60
:1002D000545C05D14000494128BF41F0004130BD88
:1002E00014F580043CBF01F5801130BD01F00045DC
:1002F00045F0FE4141F470014FF0000030BD7FEA4F
:10030000645C1ABF194610467FEA655C1CBF0B4649
:10031000024650EA013406BF52EA033591EA030F60
:1003200041F4002130BD00BF90F0000F04BF002158
:10033000704730B54FF4806404F132044FF000058B
:100340004FF0000150E700BF90F0000F04BF002104
:10035000704730B54FF4806404F1320410F000456A
:1003600048BF40424FF000013EE700BF42004FEA65
:10037000E2014FEA31014FEA02701FBF12F07F43E2
:1003800093F07F4F81F06051704792F0000F14BFDF
:1003900093F07F4F704730B54FF4607401F0004523
:1003A00021F0004120E700BF50EA010208BF70477A
:1003B00030B54FF000050AE050EA010208BF70476F
:1003C00030B511F0004502D5404261EB41014FF4D8
:1003D000806404F132045FEA915C3FF4DCAE4FF0DC
:1003E00003025FEADC0C18BF03325FEADC0C18BFC3
:1003F000033202EBDC02C2F1200300FA03FC20FA14
:1004000002F001FA03FE40EA0E0021FA02F1144460
:10041000C1E600BF70B54FF0FF0C4CF4E06C1CEA75
:1004200011541DBF1CEA135594EA0C0F95EA0C0FEA
:1004300000F0DEF82C4481EA030621EA4C5123EA5D
:100440004C5350EA013518BF52EA033541F480118C
:1004500043F4801338D0A0FB02CE4FF00005E1FB3F
:1004600002E506F00042E0FB03E54FF00006E1FB89
:1004700003569CF0000F18BF4EF0010EA4F1FF04CC
:10048000B6F5007F64F5407404D25FEA4E0E6D410C
:1004900046EB060642EAC62141EA55514FEAC5201D
:1004A00040EA5E504FEACE2EB4F1FD0C88BFBCF599
:1004B000E06F1ED8BEF1004F08BF5FEA500E50F14A
:1004C000000041EB045170BD06F0004646EA010110
:1004D00040EA020081EA0301B4EB5C04C2BFD4EB42
:1004E0000C0541EA045170BD41F480114FF0000E3B
:1004F000013C00F3AB8014F1360FDEBF002001F0A9
:10050000004170BDC4F10004203C35DA0C341BDC22
:1005100004F11404C4F1200500FA05F320FA04F0F4
:1005200001FA05F240EA020001F0004221F0004128
:1005300010EBD37021FA04F642EB06015EEA430E9B
:1005400008BF20EAD37070BDC4F10C04C4F12005CB
:1005500000FA04F320FA05F001FA04F240EA02007E
:1005600001F0004110EBD37041F100015EEA430E4F
:1005700008BF20EAD37070BDC4F1200500FA05F26F
:100580004EEA020E20FA04F301FA05F243EA0203EE
:1005900021FA04F001F0004121FA04F220EA0200FD
:1005A00000EBD3705EEA430E08BF20EAD37070BD43
:1005B00094F0000F0FD101F00046400041EB010123
:1005C00011F4801F08BF013CF7D041EA060195F005
:1005D000000F18BF704703F00046520043EB0303BF
:1005E00013F4801F08BF013DF7D043EA06037047AC
:1005F00094EA0C0F0CEA135518BF95EA0C0F0CD0B7
:1006000050EA410618BF52EA4306D1D181EA0301FC
:1006100001F000414FF0000070BD50EA410606BFF6
:100620001046194652EA430619D094EA0C0F02D13B
:1006300050EA013613D195EA0C0F05D152EA033680
:100640001CBF104619460AD181EA030101F000419E
:1006500041F0FE4141F470014FF0000070BD41F0E7
:10066000FE4141F4780170BD70B54FF0FF0C4CF4C1
:10067000E06C1CEA11541DBF1CEA135594EA0C0FE0
:1006800095EA0C0F00F0A7F8A4EB050481EA030E2D
:1006900052EA03354FEA013100F088804FEA033314
:1006A0004FF0805545EA131343EA12634FEA0222E2
:1006B00045EA111545EA10654FEA00260EF00041A3
:1006C0009D4208BF964244F1FD0404F5407402D2F5
:1006D0005B084FEA3202B61A65EB03055B084FEA86
:1006E00032024FF480104FF4002CB6EB020E75EB83
:1006F000030E22BFB61A754640EA0C005B084FEAAB
:100700003202B6EB020E75EB030E22BFB61A754627
:1007100040EA5C005B084FEA3202B6EB020E75EB72
:10072000030E22BFB61A754640EA9C005B084FEAEA
:100730003202B6EB020E75EB030E22BFB61A7546F7
:1007400040EADC0055EA060E18D04FEA051545EAE6
:1007500016754FEA06164FEAC30343EA52734FEA8F
:10076000C2025FEA1C1CC0D111F4801F0BD141EA08
:1007700000014FF000004FF0004CB6E711F4801F6D
:1007800004BF01430020B4F1FD0C88BFBCF5E06F4D
:100790003FF6AFAEB5EB030C04BFB6EB020C5FEA5D
:1007A000500C50F1000041EB045170BD0EF0004EB2
:1007B0004EEA113114EB5C04C2BFD4EB0C0541EAE4
:1007C000045170BD41F480114FF0000E013C90E6E1
:1007D00045EA060E8DE60CEA135594EA0C0F08BFA5
:1007E00095EA0C0F3FF43BAF94EA0C0F0AD150EAA4
:1007F00001347FF434AF95EA0C0F7FF425AF104637
:1008000019462CE795EA0C0F06D152EA03353FF45E
:10081000FDAE1046194622E750EA410618BF52EADB
:1008200043067FF4C5AE50EA41047FF40DAF52EAAF
:1008300043057FF4EBAE12E74FF0FF3C06E000BF4C
:100840004FF0010C02E000BF4FF0010C4DF804CD59
:100850004FEA410C7FEA6C5C4FEA430C18BF7FEA19
:100860006C5C1BD001B050EA410C0CBF52EA430C47
:1008700091EA030F02BF90EA020F0020704710F1C7
:10088000000F91EA030F58BF994208BF90422CBF56
:10089000D8176FEAE37040F0010070474FEA410C4F
:1008A0007FEA6C5C02D150EA013C07D14FEA430C6D
:1008B0007FEA6C5CD6D152EA033CD3D05DF8040BDE
:1008C000704700BF8446104662468C461946634610
:1008D00000E000BF01B5FFF7B7FF002848BF10F1E7
:1008E000000F01BD4DF808EDFFF7F4FF0CBF01202C
:1008F00000205DF808FB00BF4DF808EDFFF7EAFFA8
:1009000034BF012000205DF808FB00BF4DF808ED62
:10091000FFF7E0FF94BF012000205DF808FB00BF57
:100920004DF808EDFFF7CEFF94BF012000205DF8E1
:1009300008FB00BF4DF808EDFFF7C4FF34BF0120EE
:1009400000205DF808FB00BF4FEA410212F50012DB
:1009500015D211D56FF47873B3EB625212D94FEA06
:10096000C12343F0004343EA505311F0004F23FAF0
:1009700002F018BF404270474FF00000704750EA45
:10098000013005D111F0004008BF6FF00040704702
:100990004FF00000704700BF4FEA4102B2F1E04360
:1009A00024BFB3F5001CDCF1FE5C0DD901F0004C56
:1009B0004FEAC0024CEA5070B2F1004F40EB8300A6
:1009C00008BF20F00100704711F0804F21D113F1D2
:1009D0003872BCBF01F00040704741F480114FEA0B
:1009E0005252C2F11802C2F1200C10FA0CF320FA94
:1009F00002F018BF40F001004FEAC1234FEAD323B1
:100A000003FA0CFC40EA0C0023FA02F34FEA43031A
:100A1000CCE77FEA625307D150EA01331EBF4FF0A3
:100A2000FE4040F44000704701F0004040F0FE40BE
:100A300040F40000704700BF80F0004002E000BFBB
:100A400081F0004142001FBF5FEA410392EA030FB9
:100A50007FEA226C7FEA236C6AD04FEA1262D2EB03
:100A60001363C1BFD218414048404140B8BF5B4208
:100A7000192B88BF704710F0004F40F4000020F0A1
:100A80007F4018BF404211F0004F41F4000121F0B7
:100A90007F4118BF494292EA030F3FD0A2F1010201
:100AA00041FA03FC10EB0C00C3F1200301FA03F13F
:100AB00000F0004302D5494260EB4000B0F5000F62
:100AC00013D3B0F1807F06D340084FEA310102F121
:100AD0000102FE2A51D2B1F1004F40EBC25008BFD3
:100AE00020F0010040EA03007047490040EB00009D
:100AF00010F4000FA2F10102EDD1B0FA80FCACF1CC
:100B0000080CB2EB0C0200FA0CF0AABF00EBC250CA
:100B100052421843BCBFD0401843704792F0000FB8
:100B200081F4000106BF80F400000132013BB5E70B
:100B30004FEA41037FEA226C18BF7FEA236C21D081
:100B400092EA030F04D092F0000F08BF08467047E6
:100B500090EA010F1CBF0020704712F07F4F04D1B4
:100B6000400028BF40F00040704712F100723CBFC7
:100B700000F50000704700F0004343F0FE4040F4F1
:100B8000000070477FEA226216BF08467FEA2363AF
:100B90000146420206BF5FEA412390EA010F40F49A
:100BA000800070474FF0000304E000BF10F00043E6
:100BB00048BF40425FEA000C08BF704743F09643CD
:100BC00001464FF000001CE050EA010208BF7047E8
:100BD0004FF000030AE000BF50EA010208BF70476F
:100BE00011F0004302D5404261EB41015FEA010C84
:100BF00002BF84460146002043F0B64308BFA3F17C
:100C00008053A3F50003BCFA8CF2083AA3EBC2535D
:100C100010DB01FA02FC634400FA02FCC2F120027C
:100C2000BCF1004F20FA02F243EB020008BF20F0B3
:100C30000100704702F1200201FA02FCC2F1200219
:100C400050EA4C0021FA02F243EB020008BF20EA0E
:100C5000DC7070474FF0FF0C1CEAD0521EBF1CEA3C
:100C6000D15392EA0C0F93EA0C0F6FD01A4480EA2A
:100C7000010C400218BF5FEA41211ED04FF0006313
:100C800043EA501043EA5111A0FB01310CF000403F
:100C9000B1F5000F3EBF490041EAD3715B0040EA65
:100CA000010062F17F02FD2A1DD8B3F1004F40EB35
:100CB000C25008BF20F00100704790F0000F0CF008
:100CC000004C08BF49024CEA502040EA51207F3ACC
:100CD000C2BFD2F1FF0340EAC250704740F40000A7
:100CE0004FF00003013A5DDC12F1190FDCBF00F098
:100CF00000407047C2F10002410021FA02F1C2F146
:100D0000200200FA02FC5FEA310040F1000053EAE1
:100D10004C0308BF20EADC70704792F0000F00F02F
:100D2000004C02BF400010F4000F013AF9D040EA35
:100D30000C0093F0000F01F0004C02BF490011F4C9
:100D4000000F013BF9D041EA0C018FE70CEAD153C7
:100D500092EA0C0F18BF93EA0C0F0AD030F0004C47
:100D600018BF31F0004CD8D180EA010000F00040FB
:100D7000704790F0000F17BF90F0004F084691F0B9
:100D8000000F91F0004F14D092EA0C0F01D14202F3
:100D90000FD193EA0C0F03D14B0218BF084608D1BC
:100DA00080EA010000F0004040F0FE4040F4000006
:100DB000704740F0FE4040F4400070474FF0FF0C99
:100DC0001CEAD0521EBF1CEAD15392EA0C0F93EAE0
:100DD0000C0F69D0A2EB030280EA010C49024FEA32
:100DE000402037D04FF0805343EA111143EA1013EB
:100DF0000CF000408B4238BF5B0042F17D024FF4A3
:100E0000000C8B4224BF5B1A40EA0C00B3EB510F7D
:100E100024BFA3EB510340EA5C00B3EB910F24BF66
:100E2000A3EB910340EA9C00B3EBD10F24BFA3EBEB
:100E3000D10340EADC001B0118BF5FEA1C1CE0D1B3
:100E4000FD2A3FF650AF8B4240EBC25008BF20F066
:100E5000010070470CF0004C4CEA50207F32C2BFBA
:100E6000D2F1FF0340EAC250704740F400004FF057
:100E70000003013A37E792F0000F00F0004C02BF88
:100E8000400010F4000F013AF9D040EA0C0093F052
:100E9000000F01F0004C02BF490011F4000F013BAC
:100EA000F9D041EA0C0195E70CEAD15392EA0C0F14
:100EB00008D142027FF47DAF93EA0C0F7FF470AF4C
:100EC000084676E793EA0C0F04D14B023FF44CAF8F
:100ED00008466EE730F0004C18BF31F0004CCAD124
:100EE00030F000427FF45CAF31F000437FF43CAF60
:100EF0005FE700BF4FF0FF3C06E000BF4FF0010C82
:100F000002E000BF4FF0010C4DF804CD4FEA400263
:100F10004FEA41037FEA226C18BF7FEA236C11D0AD
:100F200001B052EA530C18BF90EA010F58BFB2EB60
:100F3000030088BFC81738BF6FEAE17018BF40F0E0
:100F4000010070477FEA226C02D15FEA402C05D194
:100F50007FEA236CE4D15FEA412CE1D05DF8040B19
:100F6000704700BF844608466146FFE70FB5FFF7AC
:100F7000C9FF002848BF10F1000F0FBD4DF808ED64
:100F8000FFF7F4FF0CBF012000205DF808FB00BF55
:100F90004DF808EDFFF7EAFF34BF012000205DF8AF
:100FA00008FB00BF4DF808EDFFF7E0FF94BF0120FC
:100FB00000205DF808FB00BF4DF808EDFFF7D2FFF9
:100FC00094BF012000205DF808FB00BF4DF808ED3C
:100FD000FFF7C8FF34BF012000205DF808FB00BF09
:100FE0004FEA4002B2F1FE4F0FD34FF09E03B3EB36
:100FF00012620DD94FEA002343F0004310F0004F76
:1010000023FA02F018BF404270474FF000007047CB
:1010100012F1610F01D1420205D110F0004008BF6A
:101020006FF0004070474FF00000704742000ED252
:10103000B2F1FE4F0BD34FF09E03B3EB126209D413
:101040004FEA002343F0004323FA02F070474FF0C9
:101050000000704712F1610F01D1420202D14FF03E
:10106000FF3070474FF00000704700BF0B4601464D
:10107000184600F001B800BF13460A460146022098
:1010800000F0B0BE014B1868704700BF5098FF1FBA
:1010900070B50F4E0F4D761BB61018BF002405D04B
:1010A000013455F8043B9847A642F9D10A4E0B4D3E
:1010B000761B03F0CFFCB61018BF002406D0013415
:1010C00055F8043B9847A642F9D170BD70BD00BFEA
:1010D000604A0100604A0100744A0100604A010050
:1010E000024B0146186800F00BB800BF5098FF1F74
:1010F000024B0146186800F039BF00BF5098FF1F2F
:101100002DE9F04F01F10B05162D83B0064640F294
:101110009F8035F0070500F1BF80A94200F2BC8036
:1011200000F058FBB5F5FC7FC0F09C826B0A00F024
:10113000BA80042B00F28381A80900F1390E4FEA2E
:101140004E033830C44F07EB8303A3F108015C68FA
:10115000A14207D1ACE0002A80F2AC80E468A14251
:1011600000F0A680636823F003035A1B0F2AF2DD08
:10117000B9493C6901F1080E744500F0B381636818
:1011800023F003035A1B0F2A00F39981002AC1F8A8
:1011900014E0C1F810E080F29E80B3F5007F80F08B
:1011A0006781DB0803F1010C01229B1002FA03F3B3
:1011B0004A6851F83C80C4F8088001EBCC091A4316
:1011C000A9F10803E3604A6041F83C40C8F80C40CC
:1011D000831001249C40944200F28A80144206D17C
:1011E00020F003006400144200F10400FAD007EB81
:1011F000C009CC468046DCF80C108C4507D173E161
:10120000002A80F28181C9688C4500F06D814B68AD
:1012100023F003035A1B0F2AF2DD0C46D1F80CC051
:1012200054F8088F4B1945F001054D6042F001015B
:10123000C8F80CC03046CCF808807B613B61C3F82D
:101240000CE0C3F808E059609A5000F0C5FA1FE0BE
:10125000102921D800F0BEFA1025062302207E4F67
:1012600007EB8303A3F108025C68944200F0458118
:101270006368E168A56823F00303234430465A6895
:10128000E96042F001028D605A6000F0A5FA08346E
:10129000204603B0BDE8F08F00240C2320463360C5
:1012A00003B0BDE8F08F80234FF0400E3F2049E7A8
:1012B00070465DE72344E1685A68A56842F0010280
:1012C000E96030468D605A6000F086FA08342046A6
:1012D00003B0BDE8F08F234430465A6842F0010263
:1012E0005A6000F079FA0834204603B0BDE8F08F68
:1012F000BC68636823F00308A84504D3C5EB080362
:101300000F2B00F38C80554BDFF860911A68D9F8E9
:10131000003001332A4404EB080A00F0608102F532
:1013200080520F3222F47F6222F00F0211463046C3
:10133000019200F04BFCB0F1FF3F8346019A00F0B0
:101340005881824500F2FC80454B1968DA4511440A
:10135000196000F05381D9F80000DFF810E1013086
:101360001BBFCAEB0B0A5144CEF800B019601BF04A
:10137000070100F01781C1F10800C1F580518344D5
:1013800008315A44C2F30B02C2EB01094946304608
:10139000019300F01BFC431C019B00F03F81CBEB51
:1013A00000024A4442F001021968C7F808B04944F3
:1013B000BC42CBF804201960DFF8A49016D0B8F135
:1013C0000F0F40F2FD806268A8F10C0323F00703C1
:1013D000E01802F001024FF0050E1A430F2B626075
:1013E000C0F804E0C0F808E000F21C811D4BBC68A6
:1013F0001A68914288BF19601B4B1A689142626853
:1014000088BF196022F003029542A2EB050301D8C0
:101410000F2B04DC304600F0DFF9002438E76219B6
:1014200043F0010345F0010565603046BA60536042
:1014300000F0D2F90834204603B0BDE8F08F142B39
:1014400071D9542B00F2A480280B00F16F0E4FEAE3
:101450004E036E3076E600BF5498FF1F3CA3FF1F7B
:1014600040A3FF1F38A3FF1F34A3FF1F609CFF1F73
:101470005A0A042A5ED9142A00F2B38002F15C01F0
:1014800049005B3207EB810C57F82110DFF8DC8153
:10149000ACF1080C8C4500F088804A6822F0030209
:1014A000934202D289688C45F7D1D1F80CC07A6892
:1014B000C4F80CC0A160CCF80840CC6088E6631981
:1014C00042F0010745F00105656030464B610B6154
:1014D000C3F80CE0C3F808E05F609A50083400F0ED
:1014E0007BF9D5E64A6873E608F1010818F0030FA6
:1014F0000CF1080C7FF47FAE30E0DC68A34208BF3B
:1015000002303FF435AEB3E60B440C465A68C96866
:1015100054F8085F42F001025A603046E9608D607D
:1015200000F05AF9B4E603F15C0E03F15B004FEAF8
:101530004E0307E69A0902F1390149003832A1E762
:10154000BC424A4B3FF400AF9C68626822F0030241
:101550005AE759F80839994540F0828010F0030F96
:1015600000F1FF30F5D17B6823EA04037B6064005F
:101570009C423FF6BDAE002C3FF4BAAE1C42404642
:101580007FF435AE64001C4200F10400FAD02EE670
:10159000B3F5AA7F18D8E80B00F1780E4FEA4E0396
:1015A0007730CFE54FF48051EBE60121D8F80430D5
:1015B000921001FA02F21A43C8F80420614677E754
:1015C0000123CBF8043025E740F25452934220D84F
:1015D000A80C00F17D0E4FEA4E037C30B2E51032CC
:1015E000A4E6542A26D81A0B02F16F0149006E3284
:1015F00048E7BC68626822F0030205E7CAF30B0003
:1016000000287FF4A8AE4244BB6842F001025A6051
:10161000ECE6FE234FF07F0E7E2093E501224FF093
:101620000009C1E604F10801304600F09FFCD9F83A
:101630000010DBE6B2F5AA7F05D8DA0B02F17801DB
:10164000490077321EE740F254518A4205D89A0C7D
:1016500002F17D0149007C3214E7FE217E2211E770
:101660007B6884E7E808431C5B00F8E55498FF1F9B
:101670008842F0B50DD98B1898420AD28118002AF9
:1016800051D09A1A13F8014D01F8014D9342F9D146
:10169000F0BD0F2A48D941EA00039B0746D100F16B
:1016A000100401F11003154653F8106C44F8106C47
:1016B00053F80C6C44F80C6C53F8086C44F8086C44
:1016C000103D53F8046C44F8046C0F2D03F1100323
:1016D00004F11004E8D8A2F1100323F00F0302F084
:1016E0000F0E1033BEF1030F1944034421D91E1FFE
:1016F0000D467446043C55F8047B46F8047F032CE1
:10170000F8D8AEF1040424F0030404342344214443
:1017100002F0030262B1013B0A4411F8014B03F8E5
:10172000014F8A42F9D1F0BD0346F3E70346F2E7E1
:10173000F0BD7246EEE700BF70B4840746D0541E79
:10174000002A41D0CDB2034602E0621EE4B3144643
:1017500003F8015B9A07F8D1032C2ED9CDB245EAE4
:1017600005250F2C45EA054519D903F11002264637
:10177000103E0F2E42F8105C42F80C5C42F8085CF8
:1017800042F8045C02F11002F2D8A4F1100222F037
:101790000F0204F00F041032032C13440DD91E461F
:1017A0002246043A032A46F8045BFAD8221F22F0A4
:1017B00003020432134404F003042CB1C9B21C44E4
:1017C00003F8011BA342FBD170BC704714460346CB
:1017D000C2E700BF704700BF704700BF024B0A4618
:1017E0000146186800F002B85098FF1F2DE9F04F2D
:1017F000174683B0002900F0C1800E46814607F1EC
:101800000B05FFF7E7FF56F804EC162D2EF0030446
:10181000A6F1080840D810221546AF4241D894429C
:1018200075DAC94B996808EB04008842416800F0FA
:10183000D98021F0010303445B68DB077DD51EF0EE
:10184000010F35D039464846FFF75AFC0746E0B14C
:1018500056F8043C23F001034344A0F108029A42E5
:1018600000F04481221F242A00F23181132A00F261
:1018700004810346324611681960516859609268C4
:101880009A603146484600F071FB4846FFF7A4FFD6
:10189000384603B0BDE8F08F25F00705002D2A4635
:1018A000BBDA0C230020C9F8003003B0BDE8F08F8C
:1018B00056F8083CC3EB080ADAF8043023F0030CAE
:1018C00004EB0C039342BDDB5746DAF80C1057F8D3
:1018D000080F221F242AC160886000F21781132A92
:1018E00040F212813168CAF808107168CAF80C1009
:1018F0001B2A00F22B8108360AF1100231681160B0
:1019000071685160B16891603E461C46D046631BC9
:101910000F2B1DD8D8F8043003F0010323434444AF
:10192000C8F80430636843F0010363604846FFF77A
:1019300053FF304603B0BDE8F08F21F0030121448E
:10194000914221DBC36882680C46D3609A60DEE76F
:10195000D8F8042008EB050102F00102154343F01A
:1019600001020B44C8F804504A605A6842F0010270
:1019700008315A60484600F0F9FAD7E7114603B03B
:10198000BDE8F04FFFF7BCBB1EF0010F7FF45AAF6C
:1019900056F8083CC3EB080ADAF8043023F0030CCD
:1019A00001EB0C0E96458BDBC36882685746D3600B
:1019B0009A6057F8081FDAF80C30CB60221F242AEF
:1019C000996000F29980132A62D93368CAF8083006
:1019D0007368CAF80C301B2A00F2A08008360AF19E
:1019E000100356E021F0030BA34405F110008345DA
:1019F00059DA1EF0010F7FF425AF56F8081CC1EB31
:101A0000080ADAF8041021F0030CE34458453FF7C4
:101A100057AF5746DAF80C1057F8080F221F242A40
:101A2000C160886000F2B480132A40F2A58031685A
:101A3000CAF808107168CAF80C101B2A00F2AF80AF
:101A400008360AF110023168116071685160B1689E
:101A500091600AEB0501C5EB0B0242F001029960AF
:101A60004A60DAF8043003F001031D434846CAF81F
:101A70000450FFF7B1FE38465CE7336803607368D3
:101A800043601B2A27D800F1080306F10802F2E69A
:101A90003B4632681A6072685A60B2689A603E4685
:101AA0007446D04633E708EB0501C5EB0B0B4BF052
:101AB000010299604A6056F8043C03F001031D439B
:101AC000484646F8045CFFF787FE304632E7314669
:101AD000FFF7CEFDD5E6B3688360F368C360242AC0
:101AE00028D000F1100306F11002C4E650F8043CBF
:101AF00023F003031C440AE7314638467446D046B7
:101B0000FFF7B6FD3E4602E73A46F7E6314638466D
:101B10001C46D046FFF7ACFD3E46F8E6B368CAF86F
:101B20001030F368CAF81430242A1BD010360AF19A
:101B30001803AEE7336903617369436106F1180264
:101B400000F1180397E600BF5498FF1FB168CAF868
:101B50001010F168CAF81410242A0FD010360AF1B8
:101B60001802CBE63369CAF818307369CAF81C301A
:101B700018360AF120038CE73A4664E73269CAF85E
:101B800018207269CAF81C2018360AF12002B5E63E
:101B9000314638460193FFF76BFD019B59E7B16869
:101BA000CAF81010F168CAF81410242A03D01036AD
:101BB0000AF1180247E73269CAF818207269CAF8B0
:101BC0001C2018360AF120023DE700BF38B5074C4B
:101BD0000023054608462360FBF7E2FE431C00D0C5
:101BE00038BD2368002BFBD02B6038BD9CA4FF1FA1
:101BF000FFFFFFFFFFFFFFFFFFFFFFFFFFFFFFFFF5
:101C000090F800F06DE9024520F007016FF0000C3C
